:020000040800F2
:1000000000060020E1010008E3010008E301000808
:10001000E3010008E3010008E3010008E301000830
:10002000E3010008E3010008E3010008652F000870
:10003000E3010008E3010008E3010008E301000810
:10004000E3010008E3010008E3010008E301000800
:10005000E3010008E30100080D3200083532000812
:100060005D32000885320008AD320008E301000867
:10007000E3010008E3010008E3010008E3010008D0
:10008000E3010008E3010008E3010008E3010008C0
:10009000E3010008E3010008E3010008D53200088D
:1000A000E3010008E3010008E3010008E3010008A0
:1000B000A9330008E3010008E3010008E301000898
:1000C000E3010008E3010008E3010008E301000880
:1000D000E3010008E3010008E3010008E301000870
:1000E00039330008E3010008E3010008E3010008D8
:1000F000E3010008E3010008E3010008E301000850
:10010000E3010008E3010008E3010008E30100083F
:10011000E3010008E3010008E3010008E30100082F
:10012000E3010008E3010008E3010008E30100081F
:10013000E3010008E3010008E3010008E30100080F
:10014000E3010008E3010008E301000819270008A3
:10015000E3010008E3010008E3010008E3010008EF
:10016000E3010008E3010008E3010008E3010008DF
:10017000E3010008E3010008E3010008E3010008CF
:10018000E3010008E3010008E3010008E3010008BF
:10019000E3010008E3010008E3010008E3010008AF
:1001A000E3010008E3010008E3010008E30100089F
:1001B000E3010008E3010008E3010008E30100088F
:1001C000E3010008E3010008E3010008E30100087F
:1001D000E3010008E3010008E3010008E30100086F
:1001E00002E000F000F8FEE772B6374880F30888B6
:1001F000364880F3098836483649086040F20000E6
:10020000CCF200004EF63471CEF200010860BFF36C
:100210004F8FBFF36F8F40F20000C0F2F0004EF638
:100220008851CEF200010860BFF34F8FBFF36F8F8C
:100230004FF00000E1EE100A4EF63C71CEF20001E4
:100240000860062080F31488BFF36F8F01F02CFF45
:1002500002F026FE4FF055301F491B4A91423CBF29
:1002600041F8040BFAE71D49184A91423CBF41F896
:10027000040BFAE71A491B4A1B4B9A423EBF51F83E
:10028000040B42F8040BF8E700201849184A914281
:100290003CBF41F8040BFAE701F00AFF02F054FEFC
:1002A000144C154DAC4203DA54F8041B8847F9E7A7
:1002B00000F042F8114C124DAC4203DA54F8041B22
:1002C0008847F9E701F0F2BE000600200022002076
:1002D0000000000808ED00E00000002000060020FB
:1002E0006837000800220020402200204022002021
:1002F000602E0020E0010008E0010008E001000895
:10030000E00100082DE9F04F2DED108AC1F80CD066
:10031000C3689D46BDEC108ABDE8F08F002383F3CF
:1003200011882846A047002001F072FAFEE701F08C
:1003300001FA00DFFEE7000038B500F0BBFB01F07A
:1003400083FE054601F0A6FE0446C8B90E4B9D4249
:1003500018D001339D4218BF044641F2883504BFCE
:1003600001240025002001F079FE0CB100F074F8A2
:1003700000F000FD284600F0BFF800F06DF8F9E746
:100380000025EFE70546EDE7010007B008B500F0EE
:1003900063FBA0F120035842584108BD07B541F264
:1003A0001203022101A8ADF8043000F073FB03B082
:1003B0005DF804FB38B5302383F3118817480368D0
:1003C0000BB101F0F1FA164A144800234FF47A7188
:1003D00001F0E0FA002383F31188124C236813B173
:1003E0002368013B2360636813B16368013B63606A
:1003F0000D4D2B7833B963687BB9022000F024FCE3
:10040000322363602B78032B07D163682BB902205A
:1004100000F01AFC4FF47A73636038BD402200206C
:10042000B50300086023002058220020084B1870F4
:1004300003280CD8DFE800F008050208022000F0CD
:10044000F9BB022000F0ECBB024B00225A6070475F
:100450005822002060230020234B244A10B51C465C
:10046000196801313FD004339342F9D16268A24246
:1004700039D31F4B9B6803F1006303F540439A4255
:1004800031D2002000F030FB0220FFF7CFFF194BE4
:100490001A6C00221A64196E1A66196E596C5A6425
:1004A000596E5A665A6E5A6942F080025A615A6908
:1004B00022F080025A615A691A6942F000521A61A8
:1004C0001A6922F000521A611B6972B64FF0E023DC
:1004D0003021C3F8084DD4E9003281F311889D46DC
:1004E00083F30888104710BD00C0000820C0000832
:1004F00000220020003802402DE9F04F93B0AA4BB3
:1005000000902022FF210AA89D6800F0DDFBA74A89
:100510001378A3B9A648012103601170302383F337
:10052000118803680BB101F03FFAA24AA0480023EA
:100530004FF47A7101F02EFA002383F31188009BA7
:1005400013B19D4B009A1A609C4A009C1378032BB0
:100550001EBF00231370984A4FF0000A18BF536063
:10056000D3465646D146012000F064FB24B1924B9D
:100570001B68002B00F01182002000F06DFA039040
:10058000039B002BF2DB012000F04AFB039B213B85
:10059000162BE8D801A252F823F000BFF905000895
:1005A00021060008B5060008670500086705000871
:1005B000670500083F0700080F0900082908000820
:1005C0008B080008B3080008D90800086705000870
:1005D000EB080008670500085D0900089906000897
:1005E00067050008A109000805060008990600082B
:1005F000670500088B0800080220FFF7C7FE0028E7
:1006000040F0F581009B0221BAF1000F08BF1C46A3
:1006100005A841F21233ADF8143000F03BFAA2E71E
:100620004FF47A7000F018FA071EEBDB0220FFF798
:10063000ADFE0028E6D0013F052F00F2DA81DFE8A9
:1006400007F0030A0D10133605230593042105A8AE
:1006500000F020FA17E054480421F9E75848042133
:10066000F6E758480421F3E74FF01C08404600F035
:100670003DFA08F104080590042105A800F00AFAE3
:10068000B8F12C0FF2D1012000FA07F747EA0B0B63
:100690005FFA8BFB4FF0000900F062FB26B10BF014
:1006A0000B030B2B08BF0024FFF778FE5BE74648DF
:1006B0000421CDE7002EA5D00BF00B030B2BA1D10D
:1006C0000220FFF763FE074600289BD0012000F0C0
:1006D0000BFA0220FFF7AAFE00261FFA86F8404612
:1006E00000F012FA044690B10021404600F01CFAD6
:1006F00001360028F1D1BA46044641F21213022114
:1007000005A8ADF814303E4600F0C4F92BE70120EF
:10071000FFF78CFE2546244B9B68AB4207D9284641
:1007200000F0E4F9013040F067810435F3E7234B32
:1007300000251D70204BBA465D603E46ACE7002E9A
:100740003FF460AF0BF00B030B2B7FF45BAF022089
:10075000FFF76CFE322000F07FF9B0F10008FFF6E1
:1007600051AF18F003077FF44DAF0F4A926808EBC2
:10077000050393423FF646AFB8F5807F3FF742AF9F
:10078000124B0193B84523DD4FF47A7000F064F901
:100790000390039A002AFFF635AF019B039A03F8F2
:1007A000012B0137EDE700BF002200205C23002071
:1007B00040220020B50300086023002058220020BA
:1007C00004220020082200200C2200205C220020AD
:1007D000C820FFF7DBFD074600283FF413AF1F2DAD
:1007E00011D8C5F1200242450AAB25F0030028BF0D
:1007F000424683490192184400F040FA019A804829
:10080000FF2100F061FA4FEAA8037D490193C8F384
:100810008702284600F060FA064600283FF46DAFD4
:10082000019B05EB830537E70220FFF7AFFD0028AA
:100830003FF4E8AE00F0A4F900283FF4E3AE00274F
:10084000B846704B9B68BB4218D91F2F11D80A9B22
:1008500001330ED027F0030312AA134453F8203CAF
:1008600005934046042205A900F0AEFA04378046FD
:10087000E7E7384600F03AF90590F2E7CDF8148042
:10088000042105A800F006F906E70023642104A866
:10089000049300F0F5F800287FF4B4AE0220FFF7CF
:1008A00075FD00283FF4AEAE049800F051F90590B4
:1008B000E6E70023642104A8049300F0E1F800288F
:1008C0007FF4A0AE0220FFF761FD00283FF49AAE4E
:1008D000049800F04DF9EAE70220FFF757FD0028E1
:1008E0003FF490AE00F05CF9E1E70220FFF74EFD27
:1008F00000283FF487AE05A9142000F057F9042121
:100900000746049004A800F0C5F83946B9E732203C
:1009100000F0A2F8071EFFF675AEBB077FF472AEBB
:10092000384A926807EB090393423FF66BAE022008
:10093000FFF72CFD00283FF465AE27F003074F4476
:10094000B9453FF4A9AE484600F0D0F8042105901F
:1009500005A800F09FF809F10409F1E74FF47A7057
:10096000FFF714FD00283FF44DAE00F009F9002810
:1009700044D00A9B01330BD008220AA9002000F0C2
:10098000ABF900283AD02022FF210AA800F09CF9F8
:10099000FFF704FD1C4800F041FF13B0BDE8F08FE5
:1009A000002E3FF42FAE0BF00B030B2B7FF42AAE7F
:1009B0000023642105A8059300F062F8074600288B
:1009C0007FF420AE0220FFF7E1FC804600283FF4D0
:1009D00019AEFFF7E3FC41F2883000F01FFF0598E5
:1009E00000F0F0F9464600F0BBF93C46BBE5064690
:1009F00052E64FF0000905E6BA467EE637467CE649
:100A00005C22002000220020A086010070B50F4B60
:100A10001B780133DBB2012B0C4611D80C4D296831
:100A20004FF47A730E6AA2FB03320146224628462F
:100A3000B047844204D1074B00221A70012070BDD8
:100A40004FF4FA7000F0EAFE0020F8E710220020D0
:100A5000082600209423002007B500230246012128
:100A60000DF107008DF80730FFF7D0FF20B19DF89A
:100A7000070003B05DF804FB4FF0FF30F9E700001A
:100A80000A4608B50421FFF7C1FF80F00100C0B29B
:100A9000404208BD30B4054C2368DD69044B0A466A
:100AA000AC460146204630BC604700BF0826002007
:100AB000A086010070B501F0CDF9094E094D3080D6
:100AC000002428683388834208D901F0BDF92B68D7
:100AD00004440133B4F5404F2B60F2D370BD00BF26
:100AE000962300206823002001F062BA00F1006024
:100AF00000F540400068704700F10060920000F58A
:100B0000404001F0EDB90000054B1A68054B1B8809
:100B10009B1A834202D9104401F096B90020704715
:100B2000682300209623002038B5084D044629B1DB
:100B300028682044BDE8384001F0A6B92868204460
:100B400001F08AF90028F3D038BD00BF68230020E7
:100B500010F003030AD1B0F5047F05D200F1005074
:100B6000A0F51040D0F80038184670470023FBE786
:100B700000F10050A0F51040D0F8100A70470000B6
:100B8000064991F8243033B10023086A81F82430F3
:100B90000822FFF7B1BF0120704700BF6C2300207F
:100BA000014B1868704700BF002004E070B5194B76
:100BB0001D68194B0138C5F30B0408442D0C0422A1
:100BC0001E88A6420BD15C680A46013C824213464D
:100BD0000FD214F9016F4EB102F8016BF6E7013A3A
:100BE00003F10803ECD181420B4602D22C2203F818
:100BF000012B0A4A05241688AE4204D1984284BFCC
:100C0000967803F8016B013C02F10402F3D1581A03
:100C100070BD00BF002004E08C3400087834000868
:100C2000022802BF024B4FF000429A61704700BF9A
:100C300000080240022802BF024B4FF400429A61B2
:100C4000704700BF00080240022801BF024A5369F2
:100C500083F40043536170470008024070B50446B6
:100C60004FF47A764CB1412C254628BF412506FB2E
:100C700005F000F0D3FD641BF4E770BD10B5002350
:100C8000934203D0CC5CC4540133F9E710BD00009B
:100C900010B5013810F9013F3BB191F900409C4279
:100CA00003D11AB10131013AF4E71AB191F90020E8
:100CB000981A10BD1046FCE703460246D01A12F9F6
:100CC000011B0029FAD1704702440346934202D027
:100CD00003F8011BFAE770472DE9F8431F4D14464E
:100CE00095F824200746884652BBDFF870909CB3E5
:100CF00095F824302BB92022FF2148462F62FFF7B8
:100D0000E3FF95F82400C0F10802A24228BF224662
:100D1000D6B24146920005EB8000FFF7AFFF95F891
:100D20002430A41B1E44F6B2082E17449044E4B2AB
:100D300085F82460DBD1FFF723FF0028D7D108E036
:100D40002B6A03EB82038342CFD0FFF719FF002801
:100D5000CBD10020BDE8F8830120FBE76C23002005
:100D6000024B1A78024B1A70704700BF9423002080
:100D70001022002010B5104C104800F0B5F82146A4
:100D80000E4800F0DDF82468626DD2F8043843F0B4
:100D90000203C2F804384FF47A70FFF75FFF084986
:100DA000204600F0D3F9626DD2F8043823F0020334
:100DB000C2F8043810BD00BF5835000808260020CE
:100DC000603500087047000030B5094D0A44914273
:100DD0000DD011F8013B5840082340F30004013BBB
:100DE0002C4013F0FF0384EA5000F6D1EFE730BD4A
:100DF0002083B8ED026843681143016003B11847CE
:100E00007047000013B5446BD4F894341A68117815
:100E1000042915D1217C022912D1197912890123C3
:100E20008B4013420CD101A904F14C0001F0F4FEF7
:100E3000D4F89444019B21790246206800F0D0F94F
:100E400002B010BD143001F077BE00004FF0FF3348
:100E5000143001F071BE00004C3001F049BF0000B9
:100E60004FF0FF334C3001F043BF0000143001F06D
:100E700045BE00004FF0FF31143001F03FBE0000CE
:100E80004C3001F015BF00004FF0FF324C3001F044
:100E90000FBF00000020704710B5D0F894341A68D6
:100EA00011780429044617D1017C022914D15979FB
:100EB000528901238B4013420ED1143001F0D8FD2A
:100EC000024648B1D4F894444FF4807361792068A5
:100ED000BDE8104000F072B910BD0000406BFFF794
:100EE000DBBF0000704700007FB5124B036000239A
:100EF0004360C0E90233012502260F4B0574044606
:100F00000290019300F18402294600964FF4807309
:100F1000143001F089FD094B0294CDE9006304F51A
:100F200023724FF48073294604F14C0001F050FE07
:100F300004B070BDAC340008DD0E0008050E0008DA
:100F40000B68302282F311880A7903EB82029061E8
:100F50004A79093243F822008A7912B103EB8203FD
:100F600098610223C0F894140374002080F3118860
:100F70007047000038B5037F044613B190F8543031
:100F8000ABB9201D01250221FFF734FF04F1140045
:100F900025776FF0010100F069FC84F8545004F1EA
:100FA0004C006FF00101BDE8384000F05FBC38BD77
:100FB00010B5012104460430FFF71CFF00232377FE
:100FC00084F8543010BD000038B5044600251430B4
:100FD00001F042FD04F14C00257701F011FE201DC7
:100FE00084F854500121FFF705FF2046BDE8384042
:100FF000FFF752BF90F8443003F06003202B07D175
:1010000090F84520212A4FF0000303D81F2A06D864
:1010100000207047222AFBD1C0E90E3303E0034AC7
:1010200082630722C26303640120704711220020FB
:1010300037B5D0F894341A681178042904461AD1C7
:10104000017C022917D11979128901238B4013429F
:1010500011D100F14C05284601F092FE58B101A9CA
:10106000284601F0D9FDD4F89444019B2179024629
:10107000206800F0B5F803B030BD0000F0B500EB1B
:10108000810385B09E6904460D46FEB1302383F38B
:10109000118804EB8507301D0821FFF7ABFEFB68C4
:1010A0005B691B6806F14C001BB1019001F0C2FDA9
:1010B000019803A901F0B0FD024648B1039B2946FF
:1010C000204600F08DF8002383F3118805B0F0BDB1
:1010D000FB685A691268002AF5D01B8A013B13404D
:1010E000F1D104F14402EAE7093138B550F8214062
:1010F000DCB1302383F31188D4F894241368527937
:1011000003EB8203DB689B695D6845B104216018CD
:10111000FFF770FE294604F1140001F0B3FC2046ED
:10112000FFF7BAFE002383F3118838BD7047000033
:1011300001F012B8012303700023C0E90133C36139
:1011400083620362C36243620363704738B5044637
:10115000302383F311880025C0E90355C0E9055504
:10116000416001F009F80223237085F311882846B5
:1011700038BD000070B500EB810305465069DA60A8
:101180000E46144618B110220021FFF79DFDA069FC
:1011900018B110220021FFF797FD31462846BDE81F
:1011A000704001F0B3B80000826802F00112826062
:1011B0000022C0E90422826101F034B9F0B400EBEE
:1011C00081044789E4680125A4698D403D43458138
:1011D00023600023A2606360F0BC01F04FB90000FF
:1011E000F0B400EB81040789E468012564698D404F
:1011F0003D43058123600023A2606360F0BC01F0E1
:10120000C9B9000070B50223002504460370C0E987
:101210000255C0E90455C564856180F8345001F079
:1012200011F863681B6823B129462046BDE8704069
:10123000184770BD0378052B10B504460AD080F816
:1012400050300523037043681B680BB10421984795
:101250000023A36010BD00000178052906D190F895
:101260005020436802701B6803B1184770470000A4
:1012700070B590F83430044613B1002380F8343050
:1012800004F14402204601F0EFF863689B68B3B9AB
:1012900094F8443013F0600535D00021204601F069
:1012A0008FFB0021204601F081FB63681B6813B1AE
:1012B000062120469847062384F8343070BD204626
:1012C00098470028E4D0B4F84A30E26B9A4288BFCD
:1012D000E36394F94430E56B002B4FF0300380F268
:1012E0000381002D00F0F280092284F8342083F37A
:1012F00011880021D4E90E232046FFF771FF002357
:1013000083F31188DAE794F8452003F07F0343EA7A
:10131000022340F20232934200F0C58021D8B3F597
:10132000807F48D00DD8012B3FD0022B00F0938056
:10133000002BB2D104F14C02A2630222E2632364C7
:10134000C1E7B3F5817F00F09B80B3F5407FA4D166
:1013500094F84630012BA0D1B4F84C3043F002038E
:1013600032E0B3F5006F4DD017D8B3F5A06F31D090
:10137000A3F5C063012B90D8636894F846205E689B
:1013800094F84710B4F848302046B047002884D07D
:101390004368A3630368E3631AE0B3F5106F36D0C4
:1013A00040F6024293427FF478AF5C4BA363022382
:1013B000E3630023C3E794F84630012B7FF46DAF5D
:1013C000B4F84C3023F00203C4E90E55A4F84C30B5
:1013D000256478E7B4F84430B3F5A06F0ED194F8E3
:1013E000463084F84E30204600F084FF63681B6866
:1013F00013B1012120469847032323700023C4E939
:101400000E339CE704F14F03A3630123C3E7237862
:10141000042B10D1302383F311882046FFF7C4FE3C
:1014200085F311880321636884F84F5021701B688D
:101430000BB12046984794F84630002BDED084F854
:101440004F300423237063681B68002BD6D0022121
:1014500020469847D2E794F848301D0603F00F0164
:1014600020460AD500F0F2FF012804D002287FF4BC
:1014700014AF2B4B9AE72B4B98E700F0D9FFF3E71B
:1014800094F84630002B7FF408AF94F8483013F0FE
:101490000F01B3D01A06204602D501F0A5FAADE738
:1014A00001F098FAAAE794F84630002B7FF4F5AEE5
:1014B00094F8483013F00F01A0D01B06204602D547
:1014C00001F07EFA9AE701F071FA97E7142284F8A6
:1014D000342083F311882B462A4629462046FFF7FD
:1014E0006DFE85F31188E9E65DB1152284F834209C
:1014F00083F311880021D4E90E232046FFF75EFE16
:10150000FDE60B2284F8342083F311882B462A460B
:1015100029462046FFF764FEE3E700BFDC340008FD
:10152000D4340008D834000838B590F83430044674
:10153000002B3ED0063BDAB20F2A34D80F2B32D81C
:10154000DFE803F0373131082232313131313131C6
:1015500031313737C56BB0F84A309D4214D2C36879
:101560001B8AB5FBF3F203FB12556DB9302383F3ED
:1015700011882B462A462946FFF732FE85F311884B
:101580000A2384F834300EE0142384F834303023F6
:1015900083F3118800231A4619462046FFF70EFEF2
:1015A000002383F3118838BD036C03B198470023EF
:1015B000E7E70021204601F003FA0021204601F070
:1015C000F5F963681B6813B1062120469847062386
:1015D000D7E7000010B590F83430142B044629D01A
:1015E00017D8062B05D001D81BB110BD093B022B23
:1015F000FBD80021204601F0E3F90021204601F04C
:10160000D5F963681B6813B1062120469847062365
:1016100019E0152BE9D10B2380F83430302383F304
:10162000118800231A461946FFF7DAFD002383F3D9
:101630001188DAE7C3689B695B68002BD5D1036C1E
:1016400003B19847002384F83430CEE700230375B4
:10165000826803691B6899689142FBD25A680360EB
:101660004260106058607047002303758268036908
:101670001B6899689142FBD85A6803604260106009
:101680005860704708B50846302383F311880B7DF6
:10169000032B05D0042B0DD02BB983F3118808BD83
:1016A0008B6900221A604FF0FF338361FFF7CEFF92
:1016B0000023F2E7D1E9003213605A60F3E700003B
:1016C000FFF7C4BF054BD9680875186802681A602F
:1016D000536001220275D860FEF714BE98230020E3
:1016E00030B50C4BDD684B1C87B004460FD02B4641
:1016F000094A684600F04EF92046FFF7E3FF009BD9
:1017000013B1684600F050F9A86907B030BDFFF783
:10171000D9FFF9E79823002085160008044B1A68C2
:10172000DB6890689B68984294BF00200120704756
:1017300098230020084B10B51C68D86822681A60EE
:10174000536001222275DC60FFF78EFF01462046C0
:10175000BDE81040FEF7D6BD9823002038B5074CF1
:1017600007490848012300252370656001F040FB0C
:101770000223237085F3118838BD00BF00260020A6
:10178000E43400089823002000F044B9034A51686B
:1017900053685B1A9842FBD8704700BF001000E006
:1017A0008B60022308618B82084670478368A3F12F
:1017B000840243F8142C026943F8442C426943F82C
:1017C000402C094A43F8242CC26843F8182C022202
:1017D00003F80C2C002203F80B2C044A43F8102CBD
:1017E000A3F12000704700BF1D03000898230020CC
:1017F00008B5FFF7DBFFBDE80840FFF761BF000059
:10180000024BDB6898610F20FFF75CBF9823002034
:10181000302383F31188FFF7F3BF000008B50146BA
:10182000302383F311880820FFF75AFF002383F346
:10183000118808BD064BDB6839B1426818605A60F0
:10184000136043600420FFF74BBF4FF0FF30704739
:10185000982300200368984206D01A6802605060FE
:1018600099611846FFF72CBF7047000038B5044651
:101870000D462068844200D138BD036823605C6057
:101880008561FFF71DFFF4E710B503689C68A2426D
:101890000CD85C688A600B604C6021605960996864
:1018A0008A1A9A604FF0FF33836010BD1B68121BC9
:1018B000ECE700000A2938BF0A2170B504460D463E
:1018C0000A26601901F08EFA01F07AFA041BA5428B
:1018D00003D8751C2E460446F3E70A2E04D9BDE84A
:1018E0007040012001F0C4BA70BD0000F8B5144B7F
:1018F0000D46D96103F1100141600A2A196982601D
:1019000038BF0A22016048601861A818144601F027
:101910005BFA0A2701F054FA431BA342064606D39A
:101920007C1C281901F05EFA27463546F2E70A2F9B
:1019300004D9BDE8F840012001F09ABAF8BD00BF13
:1019400098230020F8B506460D4601F039FA0F4AF3
:10195000134653F8107F9F4206D12A46014630466F
:10196000BDE8F840FFF7C2BFD169BB68441A2C1923
:1019700028BF2C46A34202D92946FFF79BFF2246E7
:1019800031460348BDE8F840FFF77EBF98230020AA
:10199000A823002010B4C0E9032300235DF8044B02
:1019A0004361FFF7CFBF000010B5194C236998427F
:1019B0000DD0D0E90032816813605A609A680A44F9
:1019C0009A60002303604FF0FF33A36110BD2346EC
:1019D000026843F8102F53600022026022699A4285
:1019E00003D1BDE8104001F0F7B9936881680B445A
:1019F000936001F0E5F92269E1699268441AA24214
:101A0000E4D91144BDE81040091AFFF753BF00BFE5
:101A1000982300202DE9F047DFF8BC8008F110077B
:101A20002C4ED8F8105001F0CBF9D8F81C40AA6819
:101A3000031B9A423ED81444D5E900324FF0000906
:101A4000C8F81C4013605A60C5F80090D8F81030F0
:101A5000B34201D101F0C0F989F31188D5E903310E
:101A600028469847302383F311886B69002BD8D020
:101A700001F0A6F96A69A0EB04094A4582460DD235
:101A8000022001F0F5F90022D8F81030B34208D155
:101A900051462846BDE8F047FFF728BF121A2244F6
:101AA000F2E712EB090938BF4A4629463846FFF7E4
:101AB000EBFEB5E7D8F81030B34208D01444211A31
:101AC000C8F81C00A960BDE8F047FFF7F3BEBDE809
:101AD000F08700BFA8230020982300200020704733
:101AE000FEE70000704700004FF0FF307047000035
:101AF00002290CD0032904D00129074818BF00206F
:101B00007047032A05D8054800EBC2007047044817
:101B100070470020704700BFBC350008202200201D
:101B20007035000870B59AB00546084601A91446FC
:101B300000F0C2F801A8FFF7BFF8431C5B00C5E93D
:101B400000340022237003236370C6B201AB023459
:101B50001046D1B28E4204F1020401D81AB070BD11
:101B600013F8011B04F8021C04F8010C0132F0E721
:101B700008B5302383F311880348FFF759FA00238F
:101B800083F3118808BD00BF0826002090F8443078
:101B900003F01F02012A07D190F845200B2A03D138
:101BA0000023C0E90E3315E003F06003202B08D1B9
:101BB000B0F848302BB990F84520212A03D81F2AC5
:101BC00004D8FFF717BA222AEBD0FAE7034A826358
:101BD0000722C26303640120704700BF182200205F
:101BE00007B5052917D8DFE801F0191603191920E0
:101BF000302383F31188104A01900121FFF7BAFACC
:101C000001980E4A0221FFF7B5FA0D48FFF7DCF9FB
:101C1000002383F3118803B05DF804FB302383F3C2
:101C200011880748FFF7A6F9F2E7302383F31188FC
:101C30000348FFF7BDF9EBE710350008343500081D
:101C40000826002038B50C4D0C4C0D492A4604F1ED
:101C50000800FFF767FF05F1CA0204F11000094907
:101C6000FFF760FF05F5CA7204F118000649BDE8E8
:101C70003840FFF757BF00BFD02A002020220020A5
:101C8000F0340008FA3400080535000870B5044641
:101C900008460D46FFF710F8C6B220460134037817
:101CA0000BB9184670BD32462946FEF7F1FF0028F1
:101CB000F3D10120F6E700002DE9F84F05460C4668
:101CC000FEF7FAFF2949C6B22846FFF7DFFF08B141
:101CD000013EF6B226492846FFF7D8FF08B1103674
:101CE000F6B2632E0DD8DFF88490DFF884A0214F80
:101CF000DFF888B0DFF888802E7846B92670BDE816
:101D0000F88F29462046BDE8F84F01F097BB252EF5
:101D100028D1072249462846FEF7BAFF40B9D8F82D
:101D200000302360B8F80430A38007350634E3E7B9
:101D3000082251462846FEF7ABFF98B90E4BA21C6D
:101D4000197809090232C95D02F8041C13F8011B55
:101D500001F00F015B45C95D02F8031CF0D1183496
:101D60000835C9E704F8016B0135C5E7DC35000823
:101D700005350008EB350008107AFF1F1C7AFF1F9D
:101D8000E4350008BFF34F8F024AD368DB03FCD46D
:101D9000704700BF003C024008B5094B1B7873B97F
:101DA000FFF7F0FF074B1A69002ABFBF064A5A60C7
:101DB00002F188325A601A6822F480621A6008BD03
:101DC0002E2D0020003C02402301674508B50B4B37
:101DD0001B7893B9FFF7D6FF094B1A6942F000420E
:101DE0001A611A6842F480521A601A6822F480520A
:101DF0001A601A6842F480621A6008BD2E2D002015
:101E0000003C02400B28F0B516D80C4C0C49237846
:101E10007BB90C4D0E460C234FF0006255F8047B45
:101E200046F8042B013B13F0FF033A44F6D101239B
:101E3000237051F82000F0BD0020FCE7602D002049
:101E4000302D0020FC350008014B53F8200070476E
:101E5000FC3500080C2070470B2810B5044601D94A
:101E6000002010BDFFF7CEFF064B53F82430184476
:101E7000C21A0BB90120F4E712680132F0D1043B19
:101E8000F6E700BFFC3500080B2810B5044621D842
:101E9000FFF778FFFFF780FF0F4AF323D360C300FB
:101EA000DBB243F4007343F002031361136943F49C
:101EB00080331361FFF766FFFFF7A4FF074B53F86A
:101EC000241000F0D9F8FFF781FF2046BDE810404C
:101ED000FFF7C2BF002010BD003C0240FC350008E7
:101EE000F8B512F00103144642D18218B2F1016F25
:101EF00057D82D4B1B6813F0010352D02B4DFFF721
:101F00004BFFF323EB60FFF73DFF40F20127032C6B
:101F100015D824F001046618244C401A40F2011729
:101F2000B142236900EB010524D123F001032361B1
:101F3000FFF74CFF0120F8BD043C0430E7E78307BE
:101F4000E7D12B6923F440732B612B693B432B6151
:101F500051F8046B0660BFF34F8FFFF713FF036860
:101F60009E42E9D02B6923F001032B61FFF72EFF7E
:101F70000020E0E723F44073236123693B4323619E
:101F80000B882B80BFF34F8FFFF7FCFE2D8831F8B5
:101F9000023BADB2AB42C3D0236923F001032361FE
:101FA000E4E71846C7E700BF00380240003C0240A3
:101FB000084908B50B7828B11BB9FFF7EDFE0123DE
:101FC0000B7008BD002BFCD0BDE808400870FFF77F
:101FD000FDBE00BF2E2D002010B50244064BD2B22C
:101FE000904200D110BD441C00B253F8200041F8CB
:101FF000040BE0B2F4E700BF502800400F4B30B5AF
:102000001C6F240407D41C6F44F400741C671C6FFD
:1020100044F400441C670A4C236843F48073236033
:102020000244084BD2B2904200D130BD441C00B2F1
:1020300051F8045B43F82050E0B2F4E70038024066
:10204000007000405028004007B5012201A900207F
:10205000FFF7C2FF019803B05DF804FB13B5044617
:10206000FFF7F2FFA04205D0012201A90020019450
:10207000FFF7C4FF02B010BD70470000034B1A68A1
:102080001AB9034AD2F874281A607047642D0020E8
:102090000030024008B5FFF7F1FF024B1868C0F3AB
:1020A000407008BD642D002070470000FEE700006E
:1020B0000A4B0B480B4A90420BD30B4BDA1C121AFB
:1020C000C11E22F003028B4238BF00220021FEF71E
:1020D000FBBD53F8041B40F8041BECE7A8370008CD
:1020E000602E0020602E0020602E002070B5D0E908
:1020F00015439E6800224FF0FF3504EB4213510157
:10210000D3F800090028BEBFD3F8000940F0804092
:10211000C3F80009D3F8000B0028BEBFD3F8000BAA
:1021200040F08040C3F8000B013263189642C3F8B8
:102130000859C3F8085BE0D24FF00113C4F81C380B
:1021400070BD0000890141F02001016103699B0617
:10215000FCD41220FFF71ABB10B5054C2046FEF741
:10216000E9FF4FF0A0436365024BA36510BD00BFBC
:10217000682D00205036000870B50378012B054605
:1021800050D12A4B446D98421BD1294B5A6B42F0D7
:1021900080025A635A6D42F080025A655A6D5A693C
:1021A00042F080025A615A6922F080025A610E217F
:1021B00043205B6900F022FC1E4BE3601E4BC4F819
:1021C00000380023C4F8003EC02323606E6D4FF436
:1021D0000413A3633369002BFCDA012333610C2061
:1021E000FFF7D4FA3369DB07FCD41220FFF7CEFAED
:1021F0003369002BFCDA0026A6602846FFF776FF3D
:102200006B68C4F81068DB68C4F81468C4F81C680C
:102210004BB90A4BA3614FF0FF336361A36843F0EE
:102220000103A36070BD064BF4E700BF682D0020DA
:10223000003802404014004003002002003C30C03F
:10224000083C30C0F8B5446D054600212046FFF734
:1022500079FFA96D00234FF001128F68C4F834385C
:102260004FF00066C4F81C284FF0FF3004EB431217
:1022700001339F42C2F80069C2F8006BC2F8080936
:10228000C2F8080BF2D20B686A6DEB65636210232B
:102290001361166916F01006FBD11220FFF776FACB
:1022A000D4F8003823F4FE63C4F80038A36943F47B
:1022B000402343F01003A3610923C4F81038C4F885
:1022C00014380A4BEB604FF0C043C4F8103B084B86
:1022D000C4F8003BC4F81069C4F80039EB6D03F191
:1022E000100243F48013EA65A362F8BD2C3600089F
:1022F00040800010426D90F84E10D2F8003823F460
:10230000FE6343EA0113C2F8003870472DE9F84331
:1023100000EB8103456DDA68166806F00306731E4C
:10232000022B05EB41130C4680460FFA81F94FEA68
:1023300041104FF00001C3F8101B4FF0010104F1F0
:10234000100398BFB60401FA03F391698EBF334EB0
:1023500006F1805606F5004600293AD0578A04F166
:102360005801490137436F50D5F81C180B43C5F885
:102370001C382B180021C3F8101953690127611E5E
:10238000A7409BB3138A928B9B08012A88BF5343B3
:10239000D8F85C20981842EA034301F1400205EBAB
:1023A0008202C8F85C00214653602846FFF7CAFE47
:1023B00008EB8900C3681B8A43EA845348346401EC
:1023C0001E432E51D5F81C381F43C5F81C78BDE8B4
:1023D000F88305EB4917D7F8001B21F40041C7F833
:1023E000001BD5F81C1821EA0303C0E704F13F03E2
:1023F00005EB83030A4A5A6028462146FFF7A2FEEE
:1024000005EB4910D0F8003923F40043C0F8003937
:10241000D5F81C3823EA0707D7E700BF0080001073
:1024200000040002826D1268C265FFF75FBE000003
:102430005831436D49015B5813F4004004D013F444
:10244000001F0CBF02200120704700004831436D7F
:1024500049015B5813F4004004D013F4001F0CBF73
:10246000022001207047000000EB8101CB68196A4F
:102470000B6813604B6853607047000000EB8103EA
:1024800030B5DD68AA691368D36019B9402B84BFE1
:10249000402313606B8A1468426D1C44013CB4FBFA
:1024A000F3F46343033323F0030302EB411043EAE5
:1024B000C44343F0C043C0F8103B2B6803F0030350
:1024C000012B09B20ED1D2F8083802EB411013F4F7
:1024D000807FD0F8003B14BF43F0805343F000539B
:1024E000C0F8003B02EB4112D2F8003B43F004433A
:1024F000C2F8003B30BD00002DE9F041244D6E6D67
:1025000006EB40130446D3F8087BC3F8087B380772
:102510000AD5D6F81438190706D505EB84032146E9
:10252000DB6828465B689847FA071FD5D6F8143849
:10253000DB071BD505EB8403D968CCB98B69488AC6
:102540005A68B2FBF0F600FB16228AB91868DA68FE
:1025500090420DD2121AC3E90024302383F311886C
:102560000B482146FFF78AFF84F31188BDE8F0810C
:10257000012303FA04F26B8923EA02036B81CB681F
:10258000002BF3D021460248BDE8F041184700BFB8
:10259000682D002000EB810370B5DD68436D6C6928
:1025A0002668E6604A0156BB1A444FF40020C2F880
:1025B00010092A6802F00302012A0AB20ED1D3F8E8
:1025C000080803EB421410F4807FD4F8000914BF0C
:1025D00040F0805040F00050C4F8000903EB421274
:1025E000D2F8000940F00440C2F80009D3F83408DA
:1025F000012202FA01F10143C3F8341870BD19B980
:10260000402E84BF4020206020682E8A8419013C1F
:10261000B4FBF6F440EAC44040F000501A44C6E768
:102620002DE9F8433B4D6E6D06EB40130446D3F89D
:102630000889C3F8088918F0010F4FEA40171AD02B
:10264000D6F81038DB0716D505EB8003D9684B693F
:102650001868DA68904230D2121A4FF000091A60F6
:10266000C3F80490302383F3118821462846FFF7EE
:1026700091FF89F3118818F0800F1CD0D6F83438F8
:102680000126A640334216D005EB84036D6DD3F8C6
:102690000CC0DCF814200134E4B2D2F800E005EB01
:1026A00004342F445168714515D3D5F8343823EAE2
:1026B0000606C5F83468BDE8F883012303FA04F27E
:1026C0002B8923EA02032B818B68002BD3D0214670
:1026D00028469847CFE7BCF81000AEEB01038342D1
:1026E00028BF0346D7F8180980B2B3EB800FE2D8B1
:1026F0009068A0F1040959F8048FC4F80080A0EB99
:1027000009089844B8F1040FF5D818440B449060B8
:102710005360C7E7682D00202DE9F74FA24C656D87
:102720006E69AB691E4016F480586E6107D0204672
:10273000FEF768FD03B0BDE8F04F00F047BC002E87
:1027400012DAD5F8003E98489B071EBFD5F8003E28
:1027500023F00303C5F8003ED5F8043823F0010345
:10276000C5F80438FEF778FD370505D58E48FFF724
:10277000BDFC8D48FEF75EFDB0040CD5D5F80838D9
:1027800013F0060FEB6823F470530CBF43F410539F
:1027900043F4A053EB6031071BD56368DB681BB9BA
:1027A000AB6923F00803AB612378052B0CD1D5F876
:1027B000003E7D489A071EBFD5F8003E23F0030374
:1027C000C5F8003EFEF748FD6368DB680BB176484C
:1027D0009847F30274D4B70227D5D4F85490DFF8A1
:1027E000C8B100274FF0010A09EB4712D2F8003BAD
:1027F00003F44023B3F5802F11D1D2F8003B002B16
:102800000DDA62890AFA07F322EA0303638104EB13
:102810008703DB68DB6813B1394658469847A36DD8
:1028200001379B68FFB29F42DED9F00617D5676D6E
:102830003A6AC2F30A1002F00F0302F4F012B2F582
:10284000802F00F08580B2F5402F08D104EB830380
:102850000022DB681B6A07F5805790426AD130037B
:10286000D5F8184813D5E10302D50020FFF744FE40
:10287000A20302D50120FFF73FFE630302D5022029
:10288000FFF73AFE270302D50320FFF735FE750355
:102890007FF550AFE00702D50020FFF7C1FEA1078A
:1028A00002D50120FFF7BCFE620702D50220FFF728
:1028B000B7FE23077FF53EAF0320FFF7B1FE39E7F0
:1028C000636DDFF8E4A0019300274FF00109A36DC9
:1028D0009B685FFA87FB9B453FF67DAF019B03EB4F
:1028E0004B13D3F8001901F44021B1F5802F1FD10B
:1028F000D3F8001900291BDAD3F8001941F09041F0
:10290000C3F80019D3F800190029FBDB5946606DA4
:10291000FFF718FC218909FA0BF321EA030323814D
:1029200004EB8B03DB689B6813B15946504698470C
:102930000137CCE7910708BFD7F80080072A98BF76
:1029400003F8018B02F1010298BF4FEA182884E7CF
:10295000023304EB830207F580575268D2F818C09F
:10296000DCF80820DCE9001CA1EB0C0C00218842FB
:102970000AD104EB830463689B699A6802449A60F5
:102980005A6802445A606AE711F0030F08BFD7F88B
:1029900000808C4588BF02F8018B01F1010188BFDE
:1029A0004FEA1828E3E700BF682D0020436D03EBD2
:1029B0004111D1F8003B43F40013C1F8003B7047CC
:1029C000436D03EB4111D1F8003943F40013C1F812
:1029D00000397047436D03EB4111D1F8003B23F4FC
:1029E0000013C1F8003B7047436D03EB4111D1F870
:1029F000003923F40013C1F80039704700F1604337
:102A000003F561430901C9B283F80013012200F004
:102A10001F039A4043099B0003F1604303F56143A0
:102A2000C3F880211A60704730B5039C01720433EB
:102A300004FB0325C0E90653049B03630021059BA7
:102A4000C160C0E90000C0E90422C0E90842C0E951
:102A50000A11436330BD0000416A0022C0E904113D
:102A6000C0E90A22C2606FF00101FEF7FFBE00005C
:102A7000D0E90432934201D1C2680AB9181D7047E7
:102A80000020704703691960C2680132C260C269E0
:102A9000134482690361934224BF436A03610021A6
:102AA000FEF7D8BE38B504460D46E3683BB162690F
:102AB000131D1268A3621344E362002007E0237A27
:102AC00033B929462046FEF7B5FE0028EDDA38BDB9
:102AD0006FF00100FBE70000C368C269013BC360FF
:102AE0004369134482694361934224BF436A43614B
:102AF00000238362036B03B11847704770B530231E
:102B0000044683F31188866A3EB9FFF7CBFF05467A
:102B100018B186F31188284670BDA36AE26A13F8DB
:102B2000015BA362934202D32046FFF7D5FF002347
:102B300083F31188EFE700002DE9F84F04460E46B5
:102B4000174698464FF0300989F311880025AA46A8
:102B5000D4F828B0BBF1000F09D141462046FFF759
:102B6000A1FF20B18BF311882846BDE8F88FD4E986
:102B70000A12A7EB050B521A934528BF9346BBF1E7
:102B8000400F1BD9334601F1400251F8040B43F8C2
:102B9000040B9142F9D1A36A40334036A362403519
:102BA000D4E90A239A4202D32046FFF795FF8AF31D
:102BB0001188BD42D8D289F31188C9E730465A46F8
:102BC000FEF75CF8A36A5B445E44A3625D44E7E7FA
:102BD00010B5029C0172043303FB0421C0E9061303
:102BE0000023C0E90A33039B0363049BC460C0E96C
:102BF0000000C0E90422C0E90842436310BD0000A0
:102C0000026AC260426AC0E904220022C0E90A22C4
:102C10006FF00101FEF72ABED0E904239A4201D1E8
:102C2000C26822B9184650F8043B0B607047002375
:102C30001846FAE7C368C2690133C36043691344A5
:102C400082694361934224BF436A43610021FEF7D6
:102C500001BE000038B504460D46E3683BB1236968
:102C60001A1DA262E2691344E362002007E0237A9E
:102C700033B929462046FEF7DDFD0028EDDA38BDE0
:102C80006FF00100FBE7000003691960C268013AB8
:102C9000C260C269134482690361934224BF436ADC
:102CA000036100238362036B03B118477047000080
:102CB00070B530230D460446114683F31188866AA9
:102CC0002EB9FFF7C7FF10B186F3118870BDA36A54
:102CD0001D70A36AE26A01339342A36204D3E169DF
:102CE00020460439FFF7D0FF002080F31188EDE77C
:102CF0002DE9F84F04460D46904699464FF0300AAC
:102D00008AF311880026B346A76A4FB94946204680
:102D1000FFF7A0FF20B187F311883046BDE8F88F98
:102D2000D4E90A073A1AA8EB0607974228BF1746C4
:102D3000402F1BD905F1400355F8042B40F8042B14
:102D40009D42F9D1A36A4033A3624036D4E90A23F5
:102D50009A4204D3E16920460439FFF795FF8BF3CB
:102D600011884645D9D28AF31188CDE729463A46DB
:102D7000FDF784FFA36A3B443D44A3623E44E5E77C
:102D8000D0E904239A4217D1C3689BB1836A8BB1FF
:102D9000043B9B1A0ED01360C368013BC360C36938
:102DA0001A44836902619A4224BF436A0361002383
:102DB00083620123184670470023FBE700F030B917
:102DC0004FF08043586A70474FF0804300225863A9
:102DD0001A610222DA6070474FF080430022DA6005
:102DE000704700004FF0804358637047FEE70000D3
:102DF00070B51B4B01630025044686B058608562A0
:102E00000E4600F0BFF804F11003C4E904334FF09C
:102E1000FF33C4E90635C4E90044A560E562FFF765
:102E2000CFFF2B460246C4E9082304F134010D4AC2
:102E3000256580232046FEF7B3FC0123E0600A4AA3
:102E40000375009272680192B268CDE90223074BC4
:102E50006846CDE90435FEF7CBFC06B070BD00BF77
:102E6000002600205C36000861360008ED2D0008C1
:102E7000024AD36A1843D062704700BF98230020EB
:102E80004B6843608B688360CB68C3600B694361A8
:102E90004B6903628B6943620B68036070470000F3
:102EA00008B5264B26481A6940F2FF110A431A61F9
:102EB0001A6922F4FF7222F001021A611A691A6B70
:102EC0000A431A631A6D0A431A651E4A1B6D11469E
:102ED000FFF7D6FF02F11C0100F58060FFF7D0FF7D
:102EE00002F1380100F58060FFF7CAFF02F15401DA
:102EF00000F58060FFF7C4FF02F1700100F580600B
:102F0000FFF7BEFF02F18C0100F58060FFF7B8FF0C
:102F100002F1A80100F58060FFF7B2FF02F1C401E1
:102F200000F58060FFF7ACFF02F1E00100F5806082
:102F3000FFF7A6FFBDE8084000F0EEB800380240F9
:102F4000000002406836000808B500F059FAFEF7A4
:102F500005FCFFF793F8BDE80840FEF773BE0000DC
:102F600070470000EFF3098305494A6B22F0010224
:102F70004A63683383F30988002383F31188704719
:102F800000EF00E0302080F3118862B60C4B0D4A50
:102F9000D96821F4E0610904090C0A43DA60D3F826
:102FA000FC20094942F08072C3F8FC200A6842F014
:102FB00001020A602022DA7783F82200704700BFFE
:102FC00000ED00E00003FA05001000E010B530232A
:102FD00083F311880E4B5B6813F4006314D0F1EE99
:102FE000103AEFF30984683C4FF08073E361094BBA
:102FF000DB6B236684F30988FEF790FB10B1064B68
:10300000A36110BD054BFBE783F31188F9E700BF0F
:1030100000ED00E000EF00E02F030008320300089D
:103020000F4B1A6C42F001021A641A6E42F0010250
:103030001A660C4A1B6E936843F0010393604FF0CD
:10304000804353229A624FF0FF32DA6200229A6183
:103050005A63DA605A6001225A611A60704700BFF1
:1030600000380240002004E04FF0804208B51169AA
:10307000D3680B40D9B2C9439B07116107D53023F0
:1030800083F31188FEF780FB002383F3118808BDCA
:103090001F4B1A696FEAC2526FEAD2521A611A695B
:1030A000C2F308021A614FF0FF301A695A69586179
:1030B00000215A6959615A691A6A62F080521A628B
:1030C0001A6A02F080521A621A6A5A6A58625A6A76
:1030D00059625A6A1A6C42F080521A641A6E42F0AF
:1030E00080521A661A6E0B4A106840F480701060A5
:1030F000186F00F44070B0F5007F1EBF4FF48030B1
:1031000018671967536823F40073536000F054B9CB
:103110000038024000700040334B4FF080521A6478
:10312000324A4FF4404111601A6842F001021A60BD
:103130001A689107FCD59A6822F003029A602A4B1C
:103140009A6812F00C02FBD1196801F0F9011960BC
:103150009A601A6842F480321A601A689203FCD5A9
:103160005A6F42F001025A671F4B5A6F9007FCD505
:103170001F4A5A601A6842F080721A601B4A5368EC
:103180005904FCD5184B1A689201FCD5194A9A606B
:10319000194B1A68194B9A42194B21D1194A1168D7
:1031A000194A91421CD140F205121A60144A136860
:1031B00003F00F03052BFAD10B4B9A6842F0020281
:1031C0009A609A6802F00C02082AFAD15A6C42F40A
:1031D00080425A645A6E42F480425A665B6E70476F
:1031E00040F20572E1E700BF003802400070004085
:1031F0000854400700948838002004E0116400203F
:10320000003C024000ED00E041C20F41074A08B512
:10321000536903F00103536123B1054A13680BB1ED
:1032200050689847BDE80840FFF7D0BE003C014019
:10323000E02D0020074A08B5536903F002035361EB
:1032400023B1054A93680BB1D0689847BDE80840A0
:10325000FFF7BCBE003C0140E02D0020074A08B546
:10326000536903F00403536123B1054A13690BB199
:1032700050699847BDE80840FFF7A8BE003C0140F0
:10328000E02D0020074A08B5536903F00803536195
:1032900023B1054A93690BB1D0699847BDE808404E
:1032A000FFF794BE003C0140E02D0020074A08B51E
:1032B000536903F01003536123B1054A136A0BB13C
:1032C000506A9847BDE80840FFF780BE003C0140C7
:1032D000E02D0020164B10B55C6904F478725A6139
:1032E000A30604D5134A936A0BB1D06A98476006C7
:1032F00004D5104A136B0BB1506B9847210604D5C7
:103300000C4A936B0BB1D06B9847E20504D5094A80
:10331000136C0BB1506C9847A30504D5054A936C08
:103320000BB1D06C9847BDE81040FFF74FBE00BF0F
:10333000003C0140E02D0020194B10B55C6904F4FD
:103340007C425A61620504D5164A136D0BB1506D6B
:103350009847230504D5134A936D0BB1D06D984758
:10336000E00404D50F4A136E0BB1506E9847A104C8
:1033700004D50C4A936E0BB1D06E9847620404D505
:10338000084A136F0BB1506F9847230404D5054AC0
:10339000936F0BB1D06F9847BDE81040FFF716BE92
:1033A000003C0140E02D002008B5FFF75DFEBDE8C0
:1033B0000840FFF70BBE0000062108B50846FFF7DE
:1033C0001DFB06210720FFF719FB06210820FFF748
:1033D00015FB06210920FFF711FB06210A20FFF744
:1033E0000DFB06211720FFF709FB06212820FFF718
:1033F00005FBBDE8084007211C20FFF7FFBA0000CD
:1034000008B5FFF745FE00F00BF8FDF791FEFDF75C
:1034100069FDFFF7A5FDBDE80840FFF7CFBC000040
:103420000023054A19460133102BC2E9001102F1AD
:103430000802F8D1704700BFE02D0020034611F8C4
:10344000012B03F8012B002AF9D1704753544D3357
:1034500032463F3F3F0053544D33324634307800BC
:1034600053544D3332463432780053544D33324640
:103470003434365858000000012033000010410059
:1034800001105A000310590007103100000000001D
:103490004C340008130400005634000819040000DE
:1034A00060340008210400006A34000800000000B5
:1034B000610E00084D0E0008890E0008750E000808
:1034C000810E00086D0E0008590E0008450E000818
:1034D000950E000800000000010000000000000040
:1034E00063300000E0340008F023002000260020B4
:1034F0004172647550696C6F740025424F415244AB
:10350000252D424C002553455249414C25000000D1
:1035100002000000000000007D100008E910000813
:1035200040004000A02A0020B02A00200200000035
:103530000000000003000000000000002D11000842
:103540000000000010000000C02A00200000000061
:103550000100000000000000682D002001010200B1
:10356000E11B0008F11A00088D1B0008711B000800
:10357000430000007835000809024300020100C042
:1035800032090400000102020100052400100105B7
:10359000240100010424020205240600010705821B
:1035A000030800FF09040100020A000000070501EA
:1035B00002400000070581024000000012000000E8
:1035C000C4350008120110010200004009124157E1
:1035D00000020102030100000403090425424F41D7
:1035E00052442500574647303031003031323334B1
:1035F00035363738394142434445460000400000E3
:1036000000400000004000000040000000000100F9
:1036100000000200000002000000020000000200A2
:103620000000020000000200000002000000000094
:103630007112000829150008D51500084000400047
:10364000C82D0020C82D002001000000D82D00202A
:103650008000000040010000030000006D61696E01
:103660000069646C650000000000802A0000000012
:10367000AAAAAAAA00000024FFFF00000000000080
:1036800000A00A000000000000000000AAAAAAAAE8
:1036900000000000FFFF000000000000000000002C
:1036A0000000004000000000AAAAAAAA0000000032
:1036B000FF7F00000000000000000000000000008C
:1036C00000000000AAAAAAAA00000000FFFF000054
:1036D00000000000000000000000000000000000EA
:1036E000AAAAAAAA00000000FFFF00000000000034
:1036F000000000000000000000000000AAAAAAAA22
:1037000000000000FFFF00000000000000000000BB
:103710000000000000000000AAAAAAAA0000000001
:10372000FFFF00000000000000000000000000009B
:10373000000000000A00000000000000030000007C
:103740000000000000000000000000000000000079
:103750000000000000000000000000000000000069
:103760000000000000000000FE0700000000000054
:1037700000400F0000000000FF009600000000085D
:10378000009600000000080004000000D835000882
:103790000000000000000000000000000000000029
:1037A0000000000000000000FFFFFFFFFFFFFFFF21
:1037B000FFFFFFFFFFFFFFFFFFFFFFFFFFFFFFFF19
:1037C000FFFFFFFFFFFFFFFFFFFFFFFFFFFFFFFF09
:1037D000FFFFFFFFFFFFFFFFFFFFFFFFFFFFFFFFF9
:1037E000FFFFFFFFFFFFFFFFFFFFFFFFFFFFFFFFE9
:10C000000006002089D20008E954080845540808B1
:10C01000B1540808455408087D5408088BD200081C
:10C020008BD200088BD200088BD20008E15B0A0893
:10C030008BD200088BD200088BD200088BD200086C
:10C040008BD200088BD200088BD200088BD200085C
:10C050008BD200088BD20008FD6D0A08256E0A08F5
:10C060004D6E0A08756E0A089D6E0A08991A0A082C
:10C07000C11A0A08ED1A0A08191B0A08451B0A0802
:10C080006D1B0A08991B0A081D1A0A088BD20008A2
:10C090008BD200088BD200088BD20008C56E0A082C
:10C0A000FD6F0A0801700A0815700A0819700A085D
:10C0B0001D700A0831700A0845700A0825210A080F
:10C0C000CD220A088BD200088BD200088BD2000840
:10C0D0008BD20008996F0A08AD6F0A08C16F0A0871
:10C0E000296F0A088BD200088BD2000869700A08F1
:10C0F0006D700A0881700A0885700A08C51B0A0855
:10C100008BD200088BD2000859700A088BD2000825
:10C11000D56F0A08E96F0A088BD200088BD2000895
:10C12000F11B0A08191C0A08451C0A08711C0A0898
:10C130009D1C0A088BD200088BD200088BD2000805
:10C140008BD200088BD200088BD200080D630A083E
:10C15000C51C0A08F11C0A081D1D0A088BD200081C
:10C160008BD200088BD200088BD200088BD200083B
:10C170008BD200088BD200088BD200088BD200082B
:10C180008BD200088BD200088BD200088BD200081B
:10C190008BD200088BD200088BD200088BD200080B
:10C1A0008BD200088BD200088BD200088BD20008FB
:10C1B0008BD200088BD200088BD200088BD20008EB
:10C1C0008BD200088BD200088BD200088BD20008DB
:10C1D0008BD200088BD200088BD200088BD20008CB
:10C1E0002102010861DE0108C94A030829FB04088D
:10C1F00031010508956B050879B805083DC00508AB
:10C2000075C305088D240608F9430608B5D5060848
:10C21000F13D0708BD4D0808C13F0908E1A0090824
:10C22000F9C6090849D20908C1FF090889050A08A1
:10C2300081F0004102E000BF83F0004330B54FEAD7
:10C2400041044FEA430594EA050F08BF90EA020F44
:10C250001FBF54EA000C55EA020C7FEA645C7FEAD7
:10C26000655C00F0E2804FEA5454D4EB5555B8BFFA
:10C270006D420CDD2C4480EA020281EA030382EA6B
:10C28000000083EA010180EA020281EA0303362DFD
:10C2900088BF30BD11F0004F4FEA01314FF4801CD0
:10C2A0004CEA113102D0404261EB410113F0004FE2
:10C2B0004FEA03334CEA133302D0524263EB430399
:10C2C00094EA050F00F0A780A4F10104D5F1200E37
:10C2D0000DDB02FA0EFC22FA05F2801841F1000192
:10C2E00003FA0EF2801843FA05F359410EE0A5F166
:10C2F00020050EF1200E012A03FA0EFC28BF4CF097
:10C30000020C43FA05F3C01851EBE37101F000454C
:10C3100007D54FF0000EDCF1000C7EEB00006EEB59
:10C320000101B1F5801F1BD3B1F5001F0CD34908E3
:10C330005FEA30004FEA3C0C04F101044FEA44523A
:10C3400012F5800F80F09A80BCF1004F08BF5FEAC1
:10C35000500C50F1000041EB045141EA050130BDA1
:10C360005FEA4C0C404141EB0101013C28BFB1F5B3
:10C37000801FE9D291F0000F04BF01460020B1FAFE
:10C3800081F308BF2033A3F10B03B3F120020CDAD1
:10C390000C3208DD02F1140CC2F10C0201FA0CF0AF
:10C3A00021FA02F10CE002F11402D8BFC2F1200C14
:10C3B00001FA02F120FA0CFCDCBF41EA0C019040CA
:10C3C000E41AA2BF01EB0451294330BD6FEA040413
:10C3D0001F3C1CDA0C340EDC04F11404C4F12002FE
:10C3E00020FA04F001FA02F340EA030021FA04F310
:10C3F00045EA030130BDC4F10C04C4F1200220FA67
:10C4000002F001FA04F340EA0300294630BD21FAA4
:10C4100004F0294630BD94F0000F83F4801306BF6A
:10C4200081F480110134013D4EE77FEA645C18BF5E
:10C430007FEA655C29D094EA050F08BF90EA020FF5
:10C4400005D054EA000C04BF1946104630BD91EAED
:10C45000030F1EBF0021002030BD5FEA545C05D1F0
:10C460004000494128BF41F0004130BD14F580042F
:10C470003CBF01F5801130BD01F0004545F0FE41A3
:10C4800041F470014FF0000030BD7FEA645C1ABFD8
:10C49000194610467FEA655C1CBF0B46024650EA0F
:10C4A000013406BF52EA033591EA030F41F400213B
:10C4B00030BD00BF90F0000F04BF0021704730B5C1
:10C4C0004FF4806404F132044FF000054FF0000196
:10C4D00050E700BF90F0000F04BF0021704730B557
:10C4E0004FF4806404F1320410F0004548BF40422C
:10C4F0004FF000013EE700BF42004FEAE2014FEA81
:10C5000031014FEA02701FBF12F07F4393F07F4F5B
:10C5100081F06051704732F07F4208BF704793F05E
:10C520007F4F04BF41F40021704730B54FF4607471
:10C5300001F0004521F000411CE700BF50EA010274
:10C5400008BF704730B54FF000050AE050EA01021D
:10C5500008BF704730B511F0004502D5404261EB8D
:10C5600041014FF4806404F132045FEA915C3FF4CE
:10C57000D8AE4FF003025FEADC0C18BF03325FEA6B
:10C58000DC0C18BF033202EBDC02C2F1200300FA1C
:10C5900003FC20FA02F001FA03FE40EA0E0021FA41
:10C5A00002F11444BDE600BF70B54FF0FF0C4CF42F
:10C5B000E06C1CEA11541DBF1CEA135594EA0C0FE1
:10C5C00095EA0C0F00F0DEF82C4481EA030621EA1C
:10C5D0004C5123EA4C5350EA013518BF52EA033557
:10C5E00041F4801143F4801338D0A0FB02CE4FF009
:10C5F0000005E1FB02E506F00042E0FB03E54FF039
:10C600000006E1FB03569CF0000F18BF4EF0010E30
:10C61000A4F1FF04B6F5007F64F5407404D25FEA2C
:10C620004E0E6D4146EB060642EAC62141EA5551DF
:10C630004FEAC52040EA5E504FEACE2EB4F1FD0C21
:10C6400088BFBCF5E06F1ED8BEF1004F08BF5FEA9F
:10C65000500E50F1000041EB045170BD06F0004651
:10C6600046EA010140EA020081EA0301B4EB5C04FE
:10C67000C2BFD4EB0C0541EA045170BD41F48011F6
:10C680004FF0000E013C00F3AB8014F1360FDEBF1B
:10C69000002001F0004170BDC4F10004203C35DAF7
:10C6A0000C341BDC04F11404C4F1200500FA05F37A
:10C6B00020FA04F001FA05F240EA020001F000421B
:10C6C00021F0004110EBD37021FA04F642EB060191
:10C6D0005EEA430E08BF20EAD37070BDC4F10C04BB
:10C6E000C4F1200500FA04F320FA05F001FA04F27F
:10C6F00040EA020001F0004110EBD37041F100016B
:10C700005EEA430E08BF20EAD37070BDC4F1200575
:10C7100000FA05F24EEA020E20FA04F301FA05F2DD
:10C7200043EA020321FA04F001F0004121FA04F285
:10C7300020EA020000EBD3705EEA430E08BF20EA55
:10C74000D37070BD94F0000F0FD101F0004640008F
:10C7500041EB010111F4801F08BF013CF7D041EA11
:10C76000060195F0000F18BF704703F00046520015
:10C7700043EB030313F4801F08BF013DF7D043EAE6
:10C780000603704794EA0C0F0CEA135518BF95EA9C
:10C790000C0F0CD050EA410618BF52EA4306D1D123
:10C7A00081EA030101F000414FF0000070BD50EA42
:10C7B000410606BF1046194652EA430619D094EACC
:10C7C0000C0F02D150EA013613D195EA0C0F05D1B6
:10C7D00052EA03361CBF104619460AD181EA03010A
:10C7E00001F0004141F0FE4141F470014FF00000C2
:10C7F00070BD41F0FE4141F4780170BD70B54FF05D
:10C80000FF0C4CF4E06C1CEA11541DBF1CEA1355DC
:10C8100094EA0C0F95EA0C0F00F0A7F8A4EB0504BE
:10C8200081EA030E52EA03354FEA013100F08880B5
:10C830004FEA03334FF0805545EA131343EA12637E
:10C840004FEA022245EA111545EA10654FEA002633
:10C850000EF000419D4208BF964244F1FD0404F5EC
:10C86000407402D25B084FEA3202B61A65EB030548
:10C870005B084FEA32024FF480104FF4002CB6EB05
:10C88000020E75EB030E22BFB61A754640EA0C0085
:10C890005B084FEA3202B6EB020E75EB030E22BFC5
:10C8A000B61A754640EA5C005B084FEA3202B6EB06
:10C8B000020E75EB030E22BFB61A754640EA9C00C5
:10C8C0005B084FEA3202B6EB020E75EB030E22BF95
:10C8D000B61A754640EADC0055EA060E18D04FEA53
:10C8E000051545EA16754FEA06164FEAC30343EAF3
:10C8F00052734FEAC2025FEA1C1CC0D111F4801FC0
:10C900000BD141EA00014FF000004FF0004CB6E7B8
:10C9100011F4801F04BF01430020B4F1FD0C88BF57
:10C92000BCF5E06F3FF6AFAEB5EB030C04BFB6EB62
:10C93000020C5FEA500C50F1000041EB045170BD55
:10C940000EF0004E4EEA113114EB5C04C2BFD4EB82
:10C950000C0541EA045170BD41F480114FF0000E06
:10C96000013C90E645EA060E8DE60CEA135594EA82
:10C970000C0F08BF95EA0C0F3FF43BAF94EA0C0F85
:10C980000AD150EA01347FF434AF95EA0C0F7FF4FA
:10C9900025AF104619462CE795EA0C0F06D152EA4E
:10C9A00003353FF4FDAE1046194622E750EA410632
:10C9B00018BF52EA43067FF4C5AE50EA41047FF443
:10C9C0000DAF52EA43057FF4EBAE12E74FF0FF3CA8
:10C9D00006E000BF4FF0010C02E000BF4FF0010C79
:10C9E0004DF804CD4FEA410C7FEA6C5C4FEA430CF2
:10C9F00018BF7FEA6C5C1BD001B050EA410C0CBF41
:10CA000052EA430C91EA030F02BF90EA020F0020A2
:10CA1000704710F1000F91EA030F58BF994208BF09
:10CA200090422CBFD8176FEAE37040F001007047C6
:10CA30004FEA410C7FEA6C5C02D150EA013C07D11D
:10CA40004FEA430C7FEA6C5CD6D152EA033CD3D068
:10CA50005DF8040B704700BF8446104662468C4662
:10CA60001946634600E000BF01B5FFF7B7FF002895
:10CA700048BF10F1000F01BD4DF808EDFFF7F4FFBE
:10CA80000CBF012000205DF808FB00BF4DF808ED49
:10CA9000FFF7EAFF34BF012000205DF808FB00BF6C
:10CAA0004DF808EDFFF7E0FF94BF012000205DF88E
:10CAB00008FB00BF4DF808EDFFF7CEFF94BF012043
:10CAC00000205DF808FB00BF4DF808EDFFF7C4FF3C
:10CAD00034BF012000205DF808FB00BF4FEA410C85
:10CAE0007FEA6C5C02D150EA013C0AD14FEA430C68
:10CAF0007FEA6C5C02D152EA033C02D14FF00000A5
:10CB000070474FF0010070474FEA410212F50012E2
:10CB100015D211D56FF47873B3EB625212D94FEA84
:10CB2000C12343F0004343EA505311F0004F23FA6E
:10CB300002F018BF404270474FF00000704750EAC3
:10CB4000013005D111F0004008BF6FF00040704780
:10CB50004FF00000704700BF4A0011D212F50012DA
:10CB600011D20DD56FF47873B3EB62520ED44FEA45
:10CB7000C12343F0004343EA505323FA02F07047C5
:10CB80004FF00000704750EA013002D14FF0FF3003
:10CB900070474FF0000070474FEA4102B2F1E043A6
:10CBA00024BFB3F5001CDCF1FE5C0DD901F0004C94
:10CBB0004FEAC0024CEA5070B2F1004F40EB8300E4
:10CBC00008BF20F00100704711F0804F21D113F110
:10CBD0003872BCBF01F00040704741F480114FEA49
:10CBE0005252C2F11802C2F1200C10FA0CF320FAD2
:10CBF00002F018BF40F001004FEAC1234FEAD323EF
:10CC000003FA0CFC40EA0C0023FA02F34FEA430358
:10CC1000CCE77FEA625307D150EA01331EBF4FF0E1
:10CC2000FE4040F44000704701F0004040F0FE40FC
:10CC300040F40000704700BF80F0004002E000BFF9
:10CC400081F0004142001FBF5FEA410392EA030FF7
:10CC50007FEA226C7FEA236C6AD04FEA1262D2EB41
:10CC60001363C1BFD218414048404140B8BF5B4246
:10CC7000192B88BF704710F0004F40F4000020F0DF
:10CC80007F4018BF404211F0004F41F4000121F0F5
:10CC90007F4118BF494292EA030F3FD0A2F101023F
:10CCA00041FA03FC10EB0C00C3F1200301FA03F17D
:10CCB00000F0004302D5494260EB4000B0F5000FA0
:10CCC00013D3B0F1807F06D340084FEA310102F15F
:10CCD0000102FE2A51D2B1F1004F40EBC25008BF11
:10CCE00020F0010040EA03007047490040EB0000DB
:10CCF000013A28BFB0F5000FEDD2B0FA80FCACF1DC
:10CD0000080CB2EB0C0200FA0CF0AABF00EBC25008
:10CD100052421843BCBFD0401843704792F0000FF6
:10CD200081F4000106BF80F400000132013BB5E749
:10CD30004FEA41037FEA226C18BF7FEA236C21D0BF
:10CD400092EA030F04D092F0000F08BF0846704724
:10CD500090EA010F1CBF0020704712F07F4F04D1F2
:10CD6000400028BF40F00040704712F100723CBF05
:10CD700000F50000704700F0004343F0FE4040F42F
:10CD8000000070477FEA226216BF08467FEA2363ED
:10CD90000146420206BF5FEA412390EA010F40F4D8
:10CDA000800070474FF0000304E000BF10F0004324
:10CDB00048BF40425FEA000C08BF704743F096430B
:10CDC00001464FF000001CE050EA010208BF704726
:10CDD0004FF000030AE000BF50EA010208BF7047AD
:10CDE00011F0004302D5404261EB41015FEA010CC2
:10CDF00002BF84460146002043F0B64308BFA3F1BA
:10CE00008053A3F50003BCFA8CF2083AA3EBC2539B
:10CE100010DB01FA02FC634400FA02FCC2F12002BA
:10CE2000BCF1004F20FA02F243EB020008BF20F0F1
:10CE30000100704702F1200201FA02FCC2F1200257
:10CE400050EA4C0021FA02F243EB020008BF20EA4C
:10CE5000DC7070477BB972B90029BEBF00204FF06B
:10CE6000004106E008BF00281CBF6FF000414FF0F2
:10CE7000FF3000F007BAADF1080C6DE904CE0029CF
:10CE800009DB002B1ADB00F095F8DDF804E0DDE9A2
:10CE9000022304B07047404261EB4101002B1BDBD1
:10CEA00000F088F8DDF804E0DDE9022304B0404238
:10CEB00061EB4101524263EB43037047524263EB23
:10CEC000430300F077F8DDF804E0DDE9022304B065
:10CED000404261EB41017047524263EB430300F073
:10CEE00069F8DDF804E0DDE9022304B0524263EBA7
:10CEF0004303704753B94AB9002908BF00281CBF33
:10CF00004FF0FF314FF0FF3000F0BCB9ADF1080C2D
:10CF10006DE904CE00F04EF8DDF804E0DDE902230F
:10CF200004B07047430803F05533C01A830803F078
:10CF3000333300F03330184400EB101000F00F30A2
:10CF400000EB002000EB0040000E704707EE900A57
:10CF5000F5EEC07AF1EE10FA01D400F00BB8F1EE64
:10CF6000677A08B517EE900A00F004F8404261EBCA
:10CF7000410108BDD0B5FFF7BFFA0C4B00220646B1
:10CF80000F46FFF711FBFFF7E7FD0446FFF792FAA4
:10CF9000074B0022FFF708FB02460B463046394696
:10CFA000FFF74AF9FFF7D8FD2146D0BD0000F03D5C
:10CFB0000000F0412DE9F047089D04468E46002B05
:10CFC0004DD18A42944669D9B2FA82F252B101FA3D
:10CFD00002F3C2F1200120FA01F10CFA02FC41EA4D
:10CFE000030E94404FEA1C48210CBEFBF8F61FFAD2
:10CFF0008CF708FB16E341EA034306FB07F199426D
:10D000000AD91CEB030306F1FF3080F01F8199421F
:10D0100040F21C81023E63445B1AA4B2B3FBF8F0F9
:10D0200008FB103344EA034400FB07F7A7420AD980
:10D030001CEB040400F1FF3380F00A81A74240F2A8
:10D0400007816444023840EA0640E41B00261DB113
:10D05000D4400023C5E900433146BDE8F0878B4248
:10D0600009D9002D00F0EF800026C5E90001304607
:10D070003146BDE8F087B3FA83F6002E4AD18B42E1
:10D0800002D3824200F2F980841A61EB030301208B
:10D090009E46002DE0D0C5E9004EDDE702B9FFDE77
:10D0A000B2FA82F2002A40F09280A1EB0C014FEA22
:10D0B0001C471FFA8CFE0126200CB1FBF7F307FB7F
:10D0C000131140EA01410EFB03F0884208D91CEB22
:10D0D000010103F1FF3802D2884200F2CB804346BF
:10D0E000091AA4B2B1FBF7F007FB101144EA01449E
:10D0F0000EFB00FEA64508D91CEB040400F1FF312D
:10D1000002D2A64500F2BB800846A4EB0E0440EA1A
:10D1100003409CE7C6F12007B34022FA07FC4CEA23
:10D12000030C20FA07F401FA06F31C43F9404FEA16
:10D130001C4900FA06F3B1FBF9F8200C1FFA8CFE2B
:10D1400009FB181140EA014108FB0EF0884202FA7F
:10D1500006F20BD91CEB010108F1FF3A80F0888040
:10D16000884240F28580A8F102086144091AA4B2FD
:10D17000B1FBF9F009FB101144EA014100FB0EFE7E
:10D180008E4508D91CEB010100F1FF346CD28E45AD
:10D190006AD90238614440EA0840A0FB0294A1EB3E
:10D1A0000E01A142C846A64656D353D05DB1B3EB9B
:10D1B000080261EB0E0101FA07F722FA06F3F140CB
:10D1C0001F43C5E9007100263146BDE8F087C2F172
:10D1D0002003D8400CFA02FC21FA03F391400143EA
:10D1E0004FEA1C471FFA8CFEB3FBF7F007FB103623
:10D1F0000B0C43EA064300FB0EF69E4204FA02F4CF
:10D2000008D91CEB030300F1FF382FD29E422DD921
:10D21000023863449B1B89B2B3FBF7F607FB163356
:10D2200041EA034106FB0EF38B4208D91CEB0101D6
:10D2300006F1FF3816D28B4214D9023E6144C91A56
:10D2400046EA004638E72E46284605E70646E3E666
:10D250001846F8E64B45A9D2B9EB020864EB0C0E70
:10D260000138A3E74646EAE7204694E74046D1E77F
:10D27000D0467BE7023B614432E7304609E764442D
:10D28000023842E7704700BF02E000F000F8FEE716
:10D2900072B6374880F30888364880F309883648E4
:10D2A0003649086040F20000CCF200004EF63471BE
:10D2B000CEF200010860BFF34F8FBFF36F8F40F2D3
:10D2C0000000C0F2F0004EF68851CEF20001086076
:10D2D000BFF34F8FBFF36F8F4FF00000E1EE100AE6
:10D2E0004EF63C71CEF200010860062080F31488EF
:10D2F000BFF36F8F98F0D2FC99F01CFC4FF05530C3
:10D300001F491B4A91423CBF41F8040BFAE71D49F3
:10D31000184A91423CBF41F8040BFAE71A491B4AEC
:10D320001B4B9A423EBF51F8040B42F8040BF8E73E
:10D3300000201849184A91423CBF41F8040BFAE713
:10D3400098F0B0FC99F04AFC144C154DAC4203DA4D
:10D3500054F8041B8847F9E702F052FF114C124DB4
:10D36000AC4203DA54F8041B8847F9E798F098BCFC
:10D37000000600200022002000C0000808ED00E0A8
:10D38000000000200006002090D40C08002200209D
:10D390004C2600205026002030530120E0C1000818
:10D3A00030C2000830C2000830C200082DE9F04F3A
:10D3B0002DED108AC1F80CD0C3689D46BDEC108AD3
:10D3C000BDE8F08F002383F311882846A047002092
:10D3D00097F05CFCFEE797F0C9FA00DFFEE700007B
:10D3E00001F0FF01102A2BDB10F0070F08D010F816
:10D3F000013B013A8B422DD010F0070F42B3F6D11A
:10D40000F0B441EA012141EA014122F007047FF032
:10D4100000070023F0E80256083C85EA010586EA89
:10D42000010685FA47F5A3FA87F586FA47F6A5FAC5
:10D4300087F68EB9EED1F0BC01F0FF0102F00702D1
:10D4400032B110F8013B013A83EA010313B1F8D17C
:10D450000020704701387047002D06BF354603385D
:10D46000073815F0010F07D1013015F4807F02BF96
:10D47000013015F4C03F0130F0BC0138704700BFE7
:10D4800010F8012B11F8013B012A28BF9A42F7D06E
:10D49000D01A7047034613F8012B002AFBD1181A43
:10D4A0000138704738B50022002304460D46FFF7C7
:10D4B000EDFA28B920462946BDE8384000F00AB800
:10D4C000204605F1004100F005F8404261EB4101C2
:10D4D00038BD00BFD0B50C4B002206460F46FFF703
:10D4E00063F8FFF739FB0446FEF7E4FF074B002221
:10D4F000FFF75AF802460B4630463946FEF79CFEC7
:10D50000FFF72AFB2146D0BD0000F03D0000F041AE
:10D51000036800221B68184770B50D4B1C68E56A4C
:10D520002B681E6870F0FCFA014630B1E06A0368AF
:10D53000DB699847411E18BF01212846B0474BF0D0
:10D540003FF9E36ABDE8704093F89C104AF0A0BA36
:10D550005826002013B501912021044670F0ECFA02
:10D5600090B10A4BDFED0A7A93ED007A019AB4EE9E
:10D57000E77AF1EE10FA05DA2046064B202170F02A
:10D58000E3FA002002B010BD0120FBE7305B002071
:10D590000000003490E00A0837B5094B01910546B8
:10D5A000D3F8000803689B6998470199044618B9A5
:10D5B000044A284670F0D0FC204603B030BD00BFBE
:10D5C00060760020A4E00A0830B585B004460391D7
:10D5D000402170F0B1FA90B31A49039AD1F8B83FDC
:10D5E000D1F8BC1FB3F90A5040F21450854214DC44
:10D5F000B3F90E5040F2A3639D421ADDB1F90A500F
:10D60000854214DCB1F90E10994216DD1146204610
:10D6100005B0BDE8304070F0F1BA0B4B00930B4BF6
:10D620002046402170F090FA002005B030BD084B34
:10D63000F4E7054B0093074BF2E7054BFAE70120AF
:10D64000F3E700BF6056002088E00A08B8E00A0847
:10D65000E42D0B08CEE00A082DE9F041DFF8A480A4
:10D660000546D8F8000803688EB05B6A0E469847F6
:10D67000F0B13146284670F093FB044600B30AF03F
:10D6800057FD002704462E22394602A801979CF038
:10D69000BBFA2046322301AA01210AF0B1F8044660
:10D6A00090B9144A01AB3146284670F055FC07E0AA
:10D6B000D8F8000803689B6A98470028D9D101244C
:10D6C00020460EB0BDE8F08198F8183833B10A4A08
:10D6D0003146284670F040FC3C46F1E7074803F02D
:10D6E000A9F804460028EAD1054A3146284670F0D8
:10D6F00033FCE5E7E4E00A08EDE00A0860260020D4
:10D70000FAE00A0860760020A7B5C57F01910746B8
:10D7100065B91F4B1B68986A03685B6B9847019952
:10D72000054630B91B4A384670F016FC284603B04F
:10D73000A0BDBB6833B93B685B6B384603B0BDE83E
:10D74000A0401847144890F9F83C002B09DD00F57B
:10D750007E70019174F012FF0199054608B90F4AD5
:10D76000E1E73846019171F047FA019905460C4806
:10D7700075F092FF019905403846FFF7EBFEEDB2D8
:10D78000054001993846FFF707FF0540CEE700BF87
:10D790005826002014E10A08605600202BE10A08F0
:10D7A000E053002083680BB170F04ABF012070473E
:10D7B00038B5054671F0DAFA044630B90C4A1378E8
:10D7C00043F001031370204638BD0121094874F06D
:10D7D000D5F9094806F004FB084874F061FF2846B3
:10D7E000FFF79AFE0649284671F0DAF9EBE700BF29
:10D7F00064890020A858002020880020585A002062
:10D800004CE10A0838B5054671F05CFB044688B166
:10D810000948D0F8002800F6F8639A4203D000F5D2
:10D82000736026F0DBFE2846FFF776FE03492846A4
:10D8300071F0B6F9204638BD607600205CE10A0838
:10D8400010B5074CD4F8000803681B69984728B145
:10D85000A4F6C470BDE8104070F062B910BD00BFFE
:10D860006076002030B52DED028B85B00D46B0EE10
:10D87000408AFFF7E5FF0446C8B10AF059FC294683
:10D8800009F0D2F9B4EE488AF1EE10FAF0EE400A4F
:10D8900074BF9FED090A9FED090A09487EBF28EE73
:10D8A000008A9FED080A28EE000A05F061FD204677
:10D8B00005B0BDEC028B30BDE02E654200000000DB
:10D8C000E08400200000C842014802F05FB800BFB9
:10D8D0006026002001485EF077BA00BFB048002003
:10D8E000704700007047000000207047002070471C
:10D8F000012070477047000000207047C820704723
:10D9000001207047012070470820704790F8903040
:10D910008B4286BF00EB8100D0F894000020704756
:10D9200090F890308B4286BF00EB8100D0F89400D5
:10D930000020704708B5034BD3F8000803681B6844
:10D94000984708BD60760020044BD3ED007AFDEEC9
:10D95000E77A17EE903A18B2704700BF08540020DB
:10D96000014B93F85C03704760460020034B93F92A
:10D970009003003818BF0120704700BF60460020A8
:10D98000014B93F95E03704760460020044BD3F8C7
:10D99000000803F55A63C01A18BF0120704700BF82
:10D9A00060760020704700007047000008B504480A
:10D9B00007F050FE00280CBF0A200B2008BD00BF56
:10D9C0006026002038B5154DD5F800080368DB69DE
:10D9D00098470028D5F800080368DB680CBF0124CD
:10D9E0004124984708B144F008040D4BD5F80028AD
:10D9F00093F9C834002B0B4B0ADD9A420AD044F04D
:10DA00004004094870F08CF820B144F0800401E033
:10DA10009A42F6D144F0010038BD00BF6076002084
:10DA200060560020008400209C66002000B513EEA4
:10DA3000103A8DB06222CDF8253013EE903ACDF831
:10DA400029302123CDE900328DF82410192303AAAF
:10DA5000C2218DED030ACDED040A8DED051ACDED41
:10DA6000061A8DED072ACDED082A4DF0C9FD0DB03F
:10DA70005DF804FB2DE9F0412DED028B1D4F9FED6C
:10DA80001E8A002484B005462646F0EE488AA7F593
:10DA9000807897F88031E1B28B4216D9404642F047
:10DAA0000DFD80B1436836B1D3ED007AF4EEE78A1C
:10DAB000F1EE10FA07DDD3ED008ADB8808EE103AAC
:10DAC000B8EE488A01260134E3E76EB108235322F9
:10DAD000CDE90032287CCDED028A0DEB0302AD21A9
:10DAE0008DED038A4DF08CFD04B0BDEC028BBDE8DA
:10DAF000F08100BF6036002000000000F8B5A64DA0
:10DB0000B5F86C33DA07044639D505F6AC6CDCEDB4
:10DB1000000ADFEDA27A05F6A86C9CED000A05F577
:10DB20006C6305F6B46205F6CC6605F6BC6005F6D6
:10DB3000B86105F6C86796ED003AD0ED002A91ED80
:10DB4000002A93ED001AD7ED003AD2ED001A207C9E
:10DB500060EEA70A20EE270A0521FFF767FF207C69
:10DB60004DF0E4FC0646207C4EF0E4FB00F121037E
:10DB70009E4204D2207CBDE8F8404CF02DBFB5F8A1
:10DB80006C339B071FD5864B207CD3ED4E3A93ED2B
:10DB90004F3AD3ED4B2A93ED4A2AD3ED491A93ED30
:10DBA0004C1AD3ED470A93ED460A0421FFF73EFFD6
:10DBB000207C4DF0BBFC0646207C4EF0BBFB00F108
:10DBC00021039E42D6D3B5F86C335F0725D5744B3D
:10DBD000DFED727AD3ED1F0A93ED1E0AD3ED263ADC
:10DBE00093ED273AD3ED232A93ED222AD3ED211A80
:10DBF00093ED241A207C60EEA70A20EE270A02216A
:10DC0000FFF714FF207C4DF091FC0646207C4EF07F
:10DC100091FB00F121039E42ACD3B5F86C331E0793
:10DC200022D500215F486EF09FFA0721D0ED2D3AF2
:10DC300090ED2E3AD0ED2A2A90ED292AD0ED281A1F
:10DC400090ED2B1AD0ED260A90ED250A207CFFF7E7
:10DC5000EDFE207C4DF06AFC0646207C4EF06AFB0F
:10DC600000F121039E4285D3B5F86C33D80623D545
:10DC700001214C486EF078FA0821D0ED2D3A90ED54
:10DC80002E3AD0ED2A2A90ED292AD0ED281A90EDCF
:10DC90002B1AD0ED260A90ED250A207CFFF7C6FE50
:10DCA000207C4DF043FC0646207C4EF043FB00F107
:10DCB00021039E42FFF45EAFB5F86C33990620D580
:10DCC000374B207CD3ED823A93ED833AD3ED7F2A14
:10DCD00093ED7E2AD3ED7D1A93ED801AD3ED7B0A66
:10DCE00093ED7A0A0921FFF7A1FE207C4DF01EFC7E
:10DCF0000646207C4EF01EFB00F121039E42FFF4FD
:10DD000039AFB5F86C335A0620D5274B207CD3EDBC
:10DD1000003A93ED013A53ED032A13ED042A53ED33
:10DD2000051A13ED021A53ED070A13ED080A0A212A
:10DD3000FFF77CFE207C4DF0F9FB0646207C4EF080
:10DD4000F9FA00F121039E42FFF414AFB5F86C33E9
:10DD50001B0620D5154B207CD3ED003A93ED013AFC
:10DD600053ED032A13ED042A53ED051A13ED021A9D
:10DD700053ED070A13ED080A0B21FFF757FE207C2D
:10DD80004DF0D4FB0546207C4EF0D4FA00F121037F
:10DD90009D42FFF4EFAEF8BD60460020E02E6542E4
:10DDA00060560020D05100202464002050640020E0
:10DDB00038B5C5780B46352D044628BF35253522A4
:10DDC000002118469BF020FF2A4604F10C01BDE813
:10DDD00038409BF0CFBE000037B504460D460648DC
:10DDE0000192114674F04EFB019A2946204603B079
:10DDF000BDE8304052F03CBAA85900202DE9FF415F
:10DE00004FF00008CDE900289FED0F0A0F4F8DED70
:10DE1000030A0C46064615464FF47A73B1F9022000
:10DE2000D7F8B81F52F0FEFCCDE900589DED030A6B
:10DE3000B4F90420D7F8BC1F4FF47A73304652F07F
:10DE4000F1FC04B0BDE8F0810000FA446056002007
:10DE500008B54EF065FE40F4E67040F0010008BDE4
:10DE600013B54FF44470CDE900210FF0FFFF0446D5
:10DE700028B1DDE9002153F09BFA024B23602046D4
:10DE800002B010BD98E30A0810B504460FF0F6FF83
:10DE9000204610BD0B4B93F810287AB993F8182838
:10DEA00062B9D3F8000803F55A62904208D003F62D
:10DEB000D853984214BF04200320704705207047B0
:10DEC000022070476076002008B54B69012B07D10E
:10DED000084874F0EFFB08B1002008BD0420FCE7FF
:10DEE000022B03D1034874F0F1FBF4E7BDE80840CE
:10DEF0004EF0FCBE585A002010B594B0044603A85A
:10DF00000FF084FC1A4BD3F80008036803A91B6CBC
:10DF1000984750B3247C77F01DFB059BDDED047A18
:10DF20000893069B09930023F8EEE77A9FED117A98
:10DF30000B930C930D930E930F93109311931293D5
:10DF40004FF6F853ADF84C300023962267EE877AEF
:10DF50008DF84E303323CDE90032079007AA5721C0
:10DF60002046CDED0A7A4DF04BFB14B010BD00BF3A
:10DF7000607600200AD7233CF0B52DED028B2C4CA7
:10DF80000546D4F8000803688BB0DB689847002882
:10DF900049D0D4F8004827482F7CDFED278A71F05C
:10DFA000C5F9236820461B6B60EE288A9847BDEEB2
:10DFB000C00A204610EE103A1EB22368DB6A98476A
:10DFC000BDEEC00A204610EE103A1DB22368DB6B8E
:10DFD0009847DFED1A7A2368B4EEE70AB0EE408A7C
:10DFE000F1EE10FA5B6B58BFB0EE678A2046984797
:10DFF000BCEEC88A002303930593069318EE103AEB
:10E00000B722ADF824301A23CDE900323E2103AA0D
:10E010003846CDED048A8DED070AADF82060ADF8E5
:10E0200022504DF0EDFA0BB0BDEC028BF0BD00BFFD
:10E03000607600206C540020E02E654200FF7F4790
:10E0400070B52DED048B044688B02948DFED298A90
:10E0500075F05EFAD8B3492055F0E4FD9FED269A9D
:10E0600020EE090A4A2020EE288A55F0DBFD20EE3A
:10E07000090A60EE288A267C77F06CFA054620466D
:10E0800052F008FEBDEEC88AFDEEE88A18EE103A9E
:10E0900018EE902AADF80C300023CDE90533ADF829
:10E0A0000E30ADF81020ADF812308DF81C30ED2296
:10E0B0001623CDE900328DF81D0002AA2221304638
:10E0C00002954DF09DFA08B0BDEC048B70BD1A208E
:10E0D00055F0A8FDDFED097A80EE278A462055F03D
:10E0E000A1FDDFED077A28EE288A20EE270AC0E797
:10E0F000E053002000401C466F12833A00A08C457C
:10E100000AD7233C2DE9F047044692B0007C4DF03D
:10E110000DFA0546207C4EF00DF900F126039D42D4
:10E1200005D2207C12B0BDE8F0474CF055BC424807
:10E1300007F090FA002878D0404B1F68002F74D069
:10E140001921384642F03EFA00286ED009F0F0FF5F
:10E15000064604A80FF05AFB04A9304609F0AAFDB0
:10E160004FF0000A97F88082D1465FFA8AF398450B
:10E170005BD994F80F330133DBB2434534BF84F8E5
:10E180000F3384F80F9394F80F13384642F096F942
:10E19000054600284CD0836893F92130192B47D1CC
:10E1A00043F08AF8002843D02B6803A91B6A28464D
:10E1B000984708B900230393284643F073F894F86E
:10E1C0001080074677F0C6F96A68DDED057A94F8A5
:10E1D0000F3312689FED1A7A8DF84430F8EEE77A23
:10E1E0003B1F5F4208900F920698039AD6F80C12D4
:10E1F00009905F410798109267EE877A2F222623B5
:10E20000D6F804C2D6F808420A90CDE900320E9141
:10E2100008AA42F61E314046CDED0B7ACDF830C04B
:10E220000D948DF845704DF0EBF912B0BDE8F08714
:10E230000AF1010A99E700BF60260020EC8900205E
:10E240000AD7233C2DE9F04700F50057C6B097F8F0
:10E25000605B04460E46002D36D004F5A04A04F556
:10E26000BB447022002106A89BF0CEFC2068FEF77C
:10E2700043F9012D8046894629D00AF6845ADAF8F6
:10E280000000FEF739F904460D4677F063F94FF4C4
:10E290007A725043002297F8603B2290239202A9A1
:10E2A000802224A88DF81031CDE90289CDE90445FA
:10E2B0009BF060FC71228923CDE9003242F22831C3
:10E2C00022AA30464DF09CF946B0BDE8F087002404
:10E2D0000025DAE73C2938B5054620D008D81B29A7
:10E2E00011D0242926D02846BDE8384052F0CCBDB4
:10E2F0004D29F8D126214CF081FB044640B1284637
:10E30000FFF700FF05E016214CF078FB044610B93A
:10E310000024204638BD2846FFF792FEF9E7892100
:10E320004CF06CFB04460028F2D0297C0748FFF72C
:10E3300089FFEEE70C214CF061FB04460028E7D092
:10E34000297C034874F0CEF9E3E700BF6026002083
:10E35000585A002030B52DED028BCD7891B0272D85
:10E360000C464FF027024FF0000106A828BF2725D2
:10E370009BF04AFC04F10C012E4C2A4606A89BF0A7
:10E38000F9FBD4F8000803681B69984700284CD0B3
:10E390009DF83E5015F04001019146D1FFEE000A74
:10E3A00040F28F30B7EE001A9DED0E0ADFED228AA3
:10E3B00020F0E6FA0199D4F800088DED0E0AB0EECF
:10E3C000408A02F0C1FF15F0040F68EE000A9FEDCD
:10E3D0001B8A1BD0079B0293089B0393099B049302
:10E3E00002A80A9BCDED010A059322F017FC20EE4E
:10E3F000280ADDED010A20EE080A04F5686011B074
:10E40000BDEC028BBDE8304004F086BF9DED0D0AE7
:10E4100020EE280A04F5686020EE080A11B0BDEC71
:10E42000028BBDE8304004F0A3BF11B0BDEC028BFD
:10E4300030BD00BF60760020E02E65420000C8427B
:10E4400070B50E4ED6F80008036886B01B690C46FE
:10E45000984780B102AD28460FF0D8F906AB13E912
:10E4600003008DE8030004F1080195E80C0006F5AF
:10E47000686005F063F906B070BD00BF60760020EB
:10E4800070B5304D2DED028B0646D5F8000891EDA4
:10E49000018A03688AB01B690C46984750B9BDEEE3
:10E4A000C88A18EE103ADB0704D402200AB0BDEC8B
:10E4B000028B70BDD4E9040121F07EF80028F4D06D
:10E4C000236913B96369002BEFD002A80FF09EF9FE
:10E4D00002AA2146304652F015F90028E5D0D5F8B9
:10E4E000000803681B699847D0B194ED000ADFED7E
:10E4F000167AB4EEE70AF1EE10FA1ADA06AC204604
:10E500000FF084F90AAB13E903008DE803000F480C
:10E5100094E80C0002A905F011F940B10020C5E70C
:10E520000B4802220F2106F06DFF0028DDD10420E8
:10E53000BCE7D5F800080368DB6C98470028DDD1FC
:10E54000F5E700BF6076002000000034E084002082
:10E550006026002030B58C8BC22C85B005460B465A
:10E560003AD00CD8B22C26D0C02C30D0142C42D0AB
:10E570001946284605B0BDE8304053F01DBBD12CEC
:10E580003FD0B4F5967FF3D1D1ED007A9FED2D7A8F
:10E59000F0EEE77AF4EEC77AF1EE10FA50D5D1ED4D
:10E5A000017AF0EEE77AF4EEC77AF1EE10FA47D589
:10E5B0002549022221E0254A91ED010AD2F80008FE
:10E5C0000268D26C9047A0B9042005B030BD05B0F8
:10E5D000BDE83040FFF754BF1C4A91ED000AD2F865
:10E5E0000048F7EE000A20F0C7F80146204602F086
:10E5F000BFFE0020E9E716490222164806F08AFE0F
:10E60000E1E7D1ED017AFCEEE77ACDED027AD1EDCA
:10E61000007A9DF80830FCEEE77ACDED037AD1ED73
:10E62000027AFDEEE77A17EE902A12B2009291ED8F
:10E63000030A9DF80C200146064805F0B5FEC4E724
:10E640000220C2E7000000345885002060760020D8
:10E65000A8870020602600202DE9F04F2DED028BC9
:10E66000DFF870A29FB0084610A9FFF7A1FBDAF807
:10E67000000803681B699847002800F0128104AE67
:10E6800030460FF0C3F88B48314609F057FB00289D
:10E6900000F007819DF874C0BCF1010F04D0ACF10B
:10E6A0000703022B00F2FD800AF26C730FCBBDF85A
:10E6B000705008AC84E80F0015F0030305F018094A
:10E6C00005F0C00B05F4806805F4006702931ED1C5
:10E6D000BCF1070F9DED110ADDED120A14D0ACF16B
:10E6E000080CBCF1010F00F2A480734B93ED037A88
:10E6F000D3ED007A60EEC76A67EEA00AE0EE276A03
:10E70000E0EE070AB0EE660A20460FF07FFBB9F193
:10E71000000F40F093804946DAF8000802F014FE3A
:10E72000DDED157A9DED147A8DED030A27EEA70A2B
:10E73000A7EE070A20F054F89DED031A40F2E330EB
:10E74000F1EE410A20F01CF9DDED140AB0EE408A2A
:10E750009DED150A99F05EF8DFED587A9DF874305A
:10E7600060EE277A083B9FED560A012B67EE807A10
:10E770000CD8544B03F5CB6393ED000AB8EEC00AF6
:10E7800030EE270A20F0A6F8F0EE407AB8F1000F3C
:10E790001BD19FED4A0ADDED1A7A9DF8743067EEC1
:10E7A000807A083B9FED460A012B67EE807A0CD8F1
:10E7B000444B03F5CB6393ED000AB8EEC00A30EE8C
:10E7C000270A20F087F8F0EE407A002F3BD19FED2A
:10E7D0003B0A9DED1B7A27EE007A9FED390A27EE62
:10E7E000000AB9F1000F4BD105F44065B5F5406F53
:10E7F0005CD09FED357ADDED146AF4EEC76AF1EE78
:10E8000010FAFFEE000AB7EE007A88BFF0EE470A72
:10E81000029B002B37D0BBF1000F42D0B5F5406F03
:10E8200014D168EE200A2948B0EE670A04F074FD9E
:10E8300037E096E80F0084E80F0065E7DFED247A03
:10E84000B0EE678AA2E79FED220ACAE7B8F1000F8F
:10E8500006D037BB68EE200A1C4804F089FD20E092
:10E86000FFB1DEE7BBF1000F1BD0B8F1000F03D101
:10E87000BFB1DFED170AD6E79FB9DFED150AEBE769
:10E88000029B002BEED10CAD28460EF0BFFFDDE958
:10E890000E018DE803000D4895E80C00214604F0B8
:10E8A0004DFF1FB0BDEC028BBDE8F08FF7EE000A04
:10E8B000AEE700BFB83A0020083D0020E02E6542D8
:10E8C0000000C84260360020000000B4E084002050
:10E8D00000000000607600202DE9F04F2DED028B46
:10E8E000DFF8D0B19BB008460CA9FFF761FADBF85E
:10E8F000000803681B699847002800F095809DF880
:10E9000064300B2B00F29080DFE803F0068E8E0659
:10E910008E06068E8E8E06060BF26C730FCBBDF83C
:10E92000604004AD14F0030985E80F0004F01808F6
:10E9300004F0C00A04F4806704F4006609D1DDE93C
:10E940000D0120F039FE00286ED00D9B06930E9B22
:10E950000793B8F1000F6CD14146DBF8000802F0D4
:10E96000F3FCDDED117A9DED107A8DED030A27EEB3
:10E97000A70AA7EE070A1FF033FF9DED031A4FF415
:10E980008A60F1EE410A1FF0FBFFDDED100AB0EEE8
:10E99000408A9DED110A98F03DFFDFED417A60EE6F
:10E9A000277A9FED400A67EE807A4FB99FED3C0AC7
:10E9B000DDED167A67EE807A9FED3A0A67EE807A8F
:10E9C000002E3BD19FED360A9DED177A27EE007A97
:10E9D0009FED340A27EE000AB8F1000F53D104F47A
:10E9E0004064B4F5406F4BD09FED2F7ADDED106A97
:10E9F000F4EEC76AF1EE10FAFFEE000AB7EE007A05
:10EA000088BFF0EE470AB9F1000F1AD108AC2046D2
:10EA10000EF0FCFEDDE90A018DE80300234894E8CE
:10EA20000C00294604F08AFE1BB0BDEC028BBDE849
:10EA3000F08FDFED1F7AB0EE678AB6E79FED1C0A14
:10EA4000CAE7BAF1000FEFD0B4F5406F07D168EE16
:10EA5000200A1648B0EE670A04F05EFCE4E73FB116
:10EA6000002EE1D168EE200A104804F081FCDBE7BB
:10EA7000002ED9D0EBE7002ED6D1DFED0D0AF3E75B
:10EA8000F7EE000ABFE7B9F1000FBFD0BAF1000FEF
:10EA9000CAD0002FEFD1002EC6D0DFED050AD8E78F
:10EAA000E02E65420000C842000000B4E08400206F
:10EAB000000000006076002010B44B7A8C7ACA7A8D
:10EAC00043EA042343EA0243542B07D0562B09D0D0
:10EAD000522B0BD15DF8044BFFF73CBC5DF8044BA7
:10EAE000FFF7BABD5DF8044BFFF7F6BE5DF8044BC7
:10EAF00051F0FABE014B93F85A037047604600206C
:10EB0000084BD3F8001803F58E52914201BFA3F5CC
:10EB1000005393F9F403B0FA80F0400918BF0020C5
:10EB2000704700BF60760020084BD3F8001803F54B
:10EB30008E52914207D1A3F5005393F9F403431E7B
:10EB40005842584170470020704700BF607600204F
:10EB500038B5036A1D4D43F4B84303620446D5F843
:10EB6000000803681B6A984738B1D4E9092342F4C6
:10EB7000406243F440636262A362D5F80008036810
:10EB8000DB68984738B1D4E9092342F4A04243F442
:10EB9000A0436262A3620E4B1868A8B190F880325D
:10EBA00093B1236A43F480732362636A43F48073EE
:10EBB0006362002141F082FC30B142F07DFB18B16C
:10EBC000A36A43F48073A36238BD00BF607600205F
:10EBD000EC8900207FB500F538560C3604463046E7
:10EBE00070F0A4FBDFED1E7A04F5A25020EE270A98
:10EBF000002301A9183001938DED020A039304F557
:10EC00008D5507F0B9FC09F093FA09F03DF810357D
:10EC100004F53A5228326D21284648F001FE284674
:10EC200006F543726C2148F0FBFD204601F06CFBB9
:10EC300030B104F5415238326A21284648F0F0FDDF
:10EC400004F5405393F9F83C002B06DD04F54752D8
:10EC500028326921284648F0E3FD04B070BD00BFAA
:10EC6000E02E65422DE9F04F054693B0354806F099
:10EC7000F1FC002862D005F570691921484641F081
:10EC8000A1FC00285AD00EA80EF0C0FD05F5A25038
:10EC90000EA9183009F00EF805F58D58002708F177
:10ECA000100805F58053FEB293F88031B34245D980
:10ECB0003146484641F002FC044600283CD08368B7
:10ECC00093F92130192B37D142F0F6FA002833D0CE
:10ECD00063681A6905EB860303F5A043D3F820188F
:10ECE000914229D0C3F8202823680DA91B6A204629
:10ECF000984708B900230D9376F034FC82460D98AE
:10ED00008B46FDF7F9FBCDE90A0162681068FDF753
:10ED1000F3FB119A0C4B0692109A01930B4B009344
:10ED2000CDE90801CDE90462CDE902AB084B094AFF
:10ED30000949404649F0C0FA0137B2E713B0BDE8CF
:10ED4000F08F00BF60260020CFE40A08D6E40A084E
:10ED5000A4E40A08ABE40A08CAE40A08F0B58BB0D8
:10ED6000154606460F462422002101A81C469AF0AB
:10ED70004BFFA3238DF8043095238DF80530032332
:10ED80008DF8063076F0EEFB2B6804936B680593E4
:10ED9000AB6806932368CDF80700079306F58D50FE
:10EDA0006368CDF80B1008932422A3688DF80F70C8
:10EDB00001A91030099348F083FE0BB0F0BD0000AC
:10EDC00030B589B01D220446002168469AF01CFF28
:10EDD000A3238DF8003095238DF8013001238DF8A1
:10EDE000023076F0BFFB04F5A045CDF80300D5F85E
:10EDF0000008CDF807100368DB6B984710EE103A57
:10EE0000D5F80008CDF80B300368DB6A984710EEA0
:10EE1000103AD5F80008CDF80F3003681B6B9847FF
:10EE200010EE103ACDF8133004F58053D5F80008F1
:10EE3000D3F85836ADF8173003685B6B984704F584
:10EE40008D5010EE103A1D2269461030CDF8193061
:10EE500048F036FE09B030BD2DE9F04F2DED068BA0
:10EE600000F5405791B097F9F83C002B054650DD6E
:10EE700000F58D5600F54F50383073F07FFB10369B
:10EE8000044600284AD007F2444393ED008ADFEDA0
:10EE9000257A97F8B84428EE278A76F063FB05F5C3
:10EEA00036598046D9F844000F46FDF725FB8246C7
:10EEB000D9F848008B46FDF71FFB41EC190BD9F838
:10EEC0004C00FDF719FB41EC1A0B05F57350383077
:10EED00005F096FD10EE100AFDF70EFBCDE90E01D0
:10EEE00018EE100A8DED0CAB8DED0A9BCDE908AB49
:10EEF000FDF702FB0C4B01930C4B0093CDE906018F
:10EF0000CDE902870A4B0B4A0B490494304649F07D
:10EF1000D3F911B0BDEC068BBDE8F08F9FED078AE9
:10EF2000BBE700BFE02E654220E50A0828E50A0895
:10EF3000E0E40A08E8E40A081BE50A085241C07F39
:10EF400030B52DED028B00F538558BB00C350446ED
:10EF50002C4B00936946284670F0D8FA21220021F4
:10EF600001A89AF051FEA3238DF8043095238DF863
:10EF7000053002238DF8063076F0F4FA04F540539C
:10EF8000CDF80B10D3F8B83FCDF80700B3F908302F
:10EF9000ADF80F3004F536539FED1B8A5B6ACDF850
:10EFA000113004F5A043D3F8000803689B6B984721
:10EFB00010EE103A2846CDF81530009BCDF81930E8
:10EFC00070F0A4F820EE080A04F5BC5110EE103AD7
:10EFD00004F5BB5010310C30CDF81D3022F076FC1A
:10EFE00020EE080A04F58D5010EE103A212201A9F6
:10EFF0001030CDF8213048F063FD0BB0BDEC028B32
:10F0000030BD00BF5241C07FE02E654270B590F820
:10F01000842D0C2100F6980301FB023300F53855CE
:10F020008AB00D440446D3F800621C4B019301A939
:10F03000284670F0FDF91D22002102A89AF0E4FD97
:10F04000A3238DF8083095238DF8093076F08AFADD
:10F0500004F54053CDF80B00D3F8BC3FCDF80F10AA
:10F06000B3F90830ADF8133004F5365328469B6ADF
:10F07000CDF8153070F0C4FB10EE103A04F58D5049
:10F08000CDF819301D22019BCDF81D3002A910309A
:10F09000CDF8216048F014FD0AB070BD5241C07F28
:10F0A00013B5044600F58D50103004F580540190DE
:10F0B00048F024F8019848F0BBF894F968320198B8
:10F0C00023B102B0BDE8104048F05AB902B010BDFB
:10F0D00010B500F5A0430446D3F8000803681B6888
:10F0E000984704F50053014604F58D5093F80C231E
:10F0F000103048F08DFE04F5A250183009F00EFAD9
:10F1000004F59070BDE8104017F062B89920704780
:10F110002DE9F3410446043053F06AFA3E4E3F4B6A
:10F1200063605425601953F019FC66513035B5F50C
:10F13000557FF7D104F5557055F038F804F25C713D
:10F1400004F5FC65084601916CF0E4FD0199284640
:10F150006CF04EFF04F67C27294604F51F6074F01E
:10F16000D1F838466FF0E8FE002104F6B86072F07E
:10F1700039FA04F577605EF059FC04F6B87072F065
:10F180007DFF04F5825004F58058103040F07CFE7D
:10F1900004F5CD56224BC8F8503004F5835004F5E1
:10F1A00089551C351836083073F09EF932463946B9
:10F1B000284671F0FBF81B4BC8F83C3104F5C850E9
:10F1C0000EF024FB05F2D4700EF020FB04F5C950BC
:10F1D0000EF01CFB05F2F4700EF018FB04F5CA509B
:10F1E0000EF014FB05F614000EF010FB04F5CB50E6
:10F1F000083005F093FA3946304670F0C1FC04F54A
:10F20000DC50083003F092FC204607493FF0E8FE4E
:10F21000204602B0BDE8F081C4270B08D8270B08B0
:10F22000C8E10A08C8990C082C1F0B08F0B5102279
:10F2300000F50D51B5B01144044647F09BF857480E
:10F2400000222B213FF046FA40F0D0F8544A1388B0
:10F250001A2143F002030020138054F031FF0220F2
:10F26000462154F02DFF204601F04EF838B11E2300
:10F2700014A904F54D508DF8503040F0CFFC494DA5
:10F2800054F028FD95E80F0004AE86E80F0002A9AF
:10F2900030463FF027F9F0B105F1100314AA1835F4
:10F2A00018685968164603C60833AB423246F7D190
:10F2B00018681B79306033719DF808300C2B0AD820
:10F2C00034AA1344079813F8803C00EE103AB8EEC5
:10F2D000400A40F02DFA344D95E80F0008AE103585
:10F2E00086E80F0095E80F000CAF87E80F0003A930
:10F2F00030463FF0F7F8014600284AD00021B7EE2B
:10F30000000A30463FF03AF904F50E5527498022AD
:10F3100014A89AF02FFC1035082114A800223FF001
:10F32000D9F910A928463EF05DFF00282FD02049CA
:10F330000B68D8070ED41F4B04F5025218321A601E
:10F3400004F509521032DA6004F5075238329A6136
:10F3500001230B602846174903223FF011FA0125CB
:10F3600004F58D51144A009500231031FD203FF023
:10F37000B5F9124B1A68D20705D4114A1D6004F57D
:10F380009B541C3414600E4801213FF015FA35B02F
:10F39000F0BDB7EE000A3846B4E700BF7C1C0B088E
:10F3A000D08900201CDE0A083CDE0A085CDE0A0860
:10F3B000502600200022002098C60B08542600206A
:10F3C000242200200069C0F3401070470F299DBF20
:10F3D000302303FB0100503000207047014B93F9AC
:10F3E0008403704760460020024B93F8080800F041
:10F3F000010070476076002008B503689B68984755
:10F4000080F00100C0B208BD014BD3F8B80F7047BF
:10F410006056002000290DDB074890F8D42FCBB2AE
:10F420009A4207D3D0F8D03F0122595CA0F5405052
:10F4300005F0E8BF704700BF6056002008B53AB13C
:10F44000022A10D1BDE808400748352205F062BF06
:10F45000064AD2F800288A4205D153F049FABDE89D
:10F46000084053F0CFB908BD602600206076002028
:10F4700030B589B01C220021104D03AC01A89AF0D0
:10F48000C3FB20460EF0C2F905F26C730FCB84E883
:10F490000F00102301A905F57360ADF8063023F0C5
:10F4A00039F940B1064BB5F8642F1B6805499869D6
:10F4B00003681B68984709B030BD00BF6076002024
:10F4C00058260020DC250B0801290A4603D0022912
:10F4D00000D019B90122024805F0FEBA704700BFFA
:10F4E000586300204A2910B40B4604462FD026DC6E
:10F4F0003F2921DC292913DC04390C2918D920469D
:10F5000019465DF8044B53F0DFBFA3F1C900012198
:10F51000814040F243400142F1D05DF8044B704716
:10F520002A39012088400C4901400029E7D0F4E73E
:10F5300001200A499840F7E74829E0D1EDE7D329AF
:10F54000DDDCC829E1DC6129E7D09B29F5E75DF81E
:10F55000044B1146FFF7B8BF01FF220090000100E5
:10F560000B464A2BF7B5064611465FDC292B0FDC0C
:10F57000072B70D056DC002B5DD0042B00F0AD8043
:10F580000A463046194603B0BDE8F04053F060BD6E
:10F59000A3F12A02202AF3D801A050F822F000BFDC
:10F5A000DFF6000881F5000881F5000881F5000804
:10F5B00081F5000881F5000881F5000881F5000853
:10F5C000B1F60008BDF60008C9F60008CFF600083D
:10F5D000D5F60008E5F60008EBF6000881F500080E
:10F5E00081F50008F1F6000881F5000881F50008B2
:10F5F00081F50008FDF6000881F5000881F5000896
:10F6000081F5000881F5000881F5000881F5000802
:10F6100081F5000881F50008F7F6000881F500087B
:10F620000BF70008102BABD14D494AE09B2B70D053
:10F6300003DC612BA4D101240AE0A3F1C9050A2D42
:10F640009ED8012404FA05F540F24342154297D0B2
:10F65000204603B0F0BD022AEDD1424DD5F8003866
:10F6600005F6F867BB42E6D0A5F6C4706EF058FA0E
:10F67000044678B905F5736022F00AFE51F07AFE6F
:10F68000394A05214AF09EFF2146A5F5A04000F029
:10F6900043FED0E7D5F80038BB42CCD0B5F9643F83
:10F6A00013B93046FFF7E4FE3046FFF7E1FECFE73F
:10F6B0000229C0D12D4800F0CDFFBCE70A462C49F5
:10F6C0003046FFF7BBFEB6E70A462A49F8E70A4686
:10F6D0002949F5E70A462949F2E72949F1E70A46A7
:10F6E0002849EDE70A462849EAE70A462749E7E7B5
:10F6F0000A462749E4E70A462649E1E7194BD3F8C9
:10F70000000803685B6D984795E73046FFF7DCFE1D
:10F7100091E72148019273F0FBFE00288BD11F482E
:10F720006EF0FEF90446002885D00E4BD3F8002871
:10F7300003F5865082423FF47EAF03F6D8539A42D7
:10F740003FF479AF019902297FF475AF1A2054F084
:10F750003BFC51F00FFE124A01994AF033FF77E764
:10F760005885002060760020F0250B0860260020D8
:10F7700070840020A88400206C870020388400203A
:10F78000A8870020E4870020E08400202087002054
:10F790002088002078650020E05300209C6600202F
:10F7A00009260B0800207047002070470020704792
:10F7B00000207047002070470020704700207047ED
:10F7C0000020704708B50368DB68984780F00100A7
:10F7D000C0B208BD01207047012070479FED010AAB
:10F7E000704700BF000000000020704701207047F4
:10F7F0000020704770470000102070470048704795
:10F80000F4270B0870470000002070470120704764
:10F81000002070470020704700F50D5014307047ED
:10F8200000487047EC080B0800F5A040D0F800082D
:10F8300003681B681847000000F5A04300F5BD40B1
:10F84000D3F8003878301B1A5842584170470000EE
:10F85000034808602021117008221A60704700BF19
:10F86000882A0B0803685B681847000000F0A0BFF7
:10F8700000F000BE55F0EABC46F0A2B91CF028BD6D
:10F8800048F06CBA05F0B0BB04F01EBB01F0A8B89C
:10F8900001F03EBA0CF086B955F07EB857F084BA44
:10F8A0000BF006BD52F072BF52F078BC50F032BE81
:10F8B00005F096BB05F0B2BB72F0EEBF0AF016BEC3
:10F8C00017F0DEBB00F0C4BC05F050BC04F002BF72
:10F8D00001F0ECB910B50368DB680446984728B11D
:10F8E00020460021BDE8104001F042BD10BD0000DF
:10F8F00003F030B802F06ABD02F0AEBA70B50A4B40
:10F900000446D3F800080368DB680E4698470546AE
:10F9100040B104F5A044D4F800080368DB6B9847B5
:10F9200086ED000A284670BD6076002070B50A4B4F
:10F930000446D3F800080368DB680E46984705467E
:10F9400040B104F5A044D4F800080368DB6A984786
:10F9500086ED000A284670BD6076002070B50A4B1F
:10F960000446D3F800080368DB680E46984705464E
:10F9700040B104F5A044D4F8000803685B6B9847D5
:10F9800086ED000A284670BD6076002070B500F54F
:10F99000A0430446D3F80008036886B01B690D46EF
:10F9A000984778B102AE30460DF030FF06AB13E950
:10F9B00003008DE80300294696E80C0004F5BD40DD
:10F9C00003F0BCFE06B070BD70B5224B036000F5BD
:10F9D000A0430446D3F800071F4AC3F8502508B1D6
:10F9E0000EF050FA1D4B236004F5005393F83420B9
:10F9F0003AB91D6B2DB128461BF0E8FA28460EF0E7
:10FA00003DFA04F59B506DF0CFFB04F593500830A0
:10FA100055F0F6F904F6B46504F65466B54204D020
:10FA2000183D28461AF028FFF8E70D4BC4F898381F
:10FA300004F6F81049F0B2FF04F6CC1049F0AEFF1E
:10FA400004F62C1049F0AAFF04F5106049F0A6FF57
:10FA5000204670BD182D0B0898DE0B080CC00B0853
:10FA600044880B0838B5474B044640F8043B55F032
:10FA70000DFD04F110000BF041FD04F1680045F0AC
:10FA80002DFE04F5907015F085FF04F586600AF0F0
:10FA90009DFB04F254500EF0F7F904F698001CF0A8
:10FAA0005DFA04F5636055F0CFFA04F5706040F03C
:10FAB000AFFC04F58D50103047F04AFF04F5935029
:10FAC000083055F085F904F5955004300DF008F82C
:10FAD00004F59B506DF054FB04F59B501C3046F030
:10FAE000BFF904F59E50103056F07EFE04F58053A9
:10FAF0000025254A83F8F45304F5A05004F59F53DC
:10FB00001433043013603CF02DF904F5A25029465B
:10FB1000183006F085FE04F5D65065F0CFFE04F5EA
:10FB2000F65004306AF014F804F5FE501C306CF006
:10FB300081FC04F501506DF0B7F804F5025018305F
:10FB400005F090FD04F50750383066F015FB04F51C
:10FB5000095010305BF066FE04F5005304F50C50BC
:10FB600083F80C53094D24306DF0DEFE2B6813B181
:10FB7000074875F0BDFC204606493FF031FA2C607D
:10FB8000204638BD0CC00B08BC920020208A002003
:10FB9000FC270B0834BF0B08F8B50446254601F0D6
:10FBA00047FA214B45F8383B204B6465C4E91634CD
:10FBB0001F4BC4E918341F4BA36604F17C000DF001
:10FBC00025FE04F198000DF021FE04F1B4000DF0C3
:10FBD0001DFE4FF6FF76184BC4F8C830A4F8CC6071
:10FBE00004F1D0000DF012FE4FF0FF37134B144913
:10FBF000C4F82C7128461D603FF0F2F9A4F8747027
:10FC0000A4F8906004F5A2700DF000FE04F5BE703B
:10FC10000DF0FCFD04F5CC700DF0F8FD04F5DA7084
:10FC20000DF0F4FD2046F8BD28310B08F1F800086E
:10FC3000F5F80008F9F800080000FFFF148900201B
:10FC40008C950B082DE9F041044686B0FFF70AFFBA
:10FC5000864B2360864B8748186004F50D520C32A2
:10FC6000002314269DB206FB05010133097C0029FF
:10FC7000F8D1814B1D80814B196811B1804875F016
:10FC800037FC04F50E5010301A60FFF741FA04F506
:10FC90007E5030306FF036F904F5405304F50E52C3
:10FCA0000532C3F8D02F04F57F50062283F8D42FF5
:10FCB000183054F09FFC04F5804004F580453C303A
:10FCC0006DF0EEFE6F4BEB63284674306DF0D2FEA4
:10FCD0006D4B6B672846783004F5A04504F5AA47BC
:10FCE0005FF01EFA5037694BC5F8503507F1080030
:10FCF00074F0FAFD04F5AA4604F5AB487C3608F129
:10FD00006008304614364EF0DDFDB045F9D10723CA
:10FD1000C5F804370023A5F808374FF4CB700EF070
:10FD2000ABF8C5F8000704F5AE400C3074F0DCFD0C
:10FD300004F5AE40503074F0D7FD554B1A6802B947
:10FD40001F60544BC5F8503504F5AE406C300DF0D3
:10FD50005DFD04F5AE404FF480517C300BF0A8FC03
:10FD600004F5BB464C4B059320364C4BC5F8006858
:10FD70000494009304F5B04006AB13E90C004FF473
:10FD800000714C300AF012FF304601F051F9444B3B
:10FD9000C5F8A03D04F5BB40583001F049F9414B8E
:10FDA000C5F8D83D04F5BC40103001F041F93E4B98
:10FDB000C5F8103E04F5BC40483001F039F93B4B22
:10FDC000C5F8483E04F5BD4001F032F9384BC5F89E
:10FDD000803E04F5BD4068300DF018FD04F5C146C5
:10FDE00004F5BD404036783004F5C045FFF7D4FE39
:10FDF000304601F01DF92F4BC5F8C03006F1380030
:10FE00000DF004FD04F5C2400C3001F011F92A4B4D
:10FE1000C5F80C3104F5C240483001F009F9274B10
:10FE2000C5F8483104F5C340043001F001F9244B12
:10FE3000C5F8843104F5C340403001F0F9F8214B96
:10FE4000C5F8C03104F5C4454FF0804603A92846E3
:10FE500003964AF04BF802A905F10C0002964AF00D
:10FE600045F8204606B0BDE8F08100BF182D0B080C
:10FE7000E08900207C210B08DE8900209C8900207D
:10FE800010280B0878E10A08B8E10A0898DE0B0888
:10FE90003C8D00206CE40A08D1F80008082D0B08FE
:10FEA00034280B0874330B085C340B08482F0B08FC
:10FEB00008330B08E8330B084C360B08DC340B080E
:10FEC000E0350B0850350B08F0B5044600F58040CE
:10FED00085B03C3004F5A256FDF71EFB18362046CF
:10FEE00005F058F90021304608F0A8F804F5AE41B5
:10FEF0006C31304607F0DEFE04F5A04504F580576E
:10FF000085F81C0897F8D41611F0010103D1236875
:10FF100020469B6C9847002301A930460193029329
:10FF2000039307F017FF28B301A821F063F905F642
:10FF3000480585ED000A0121204605F085FB28B122
:10FF40002046FEF747FE2046FEF786FF802120462A
:10FF500005F07AFB18B11DF0C3FF1BF0C3FE4FF490
:10FF60008011204605F070FB10B1304606F0DEFB34
:10FF700005B0F0BD94F8E433B02202FB034394F8DB
:10FF8000282493F8C131002AD5D1022B81BF07F66E
:10FF90005C0705F648053B682B60CCE7FFF794BF8C
:10FFA00070B500F50053044693F97C3333B300F584
:10FFB000A043D3F8FC560DB375F0CCFA04F57C538E
:10FFC00093ED050ADFED0E7A9FED0E1ADFED0E0AB6
:10FFD000451B20EE270A40F269101EF0D1FCFCEE12
:10FFE000C07A204617EE903A9D42084ABDE870401C
:10FFF00034BF00230123022100F09CBD70BD00BF6F
:020000040801F1
:1000000000007A440000804F00000000121B0B0823
:10001000FFF7C6BF38B50221044605F015FB50B105
:100020000121204605F010FB28B92046FEF7D2FD3D
:100030002046FEF711FF1021204605F005FB10B108
:100040002046FEF7E3FF2021204605F0FDFA00B32D
:1000500004F5755520460835FEF7B2FE28466FF0C8
:10006000D3FDB0B1284604F58D5504F5755410350F
:1000700024346FF0C1FE04F1400228466E2147F09F
:10008000CFFB04F16C0228466F21BDE8384047F0F1
:10009000C7BB38BDFFF7BEBF10B54FF400510446D3
:1000A00005F0D2FA10B12046FEF74AFF4FF4804126
:1000B000204605F0C9FA38B12046FEF7F1FF04F5F5
:1000C0002B502C306BF022FF8021204605F0BCFA2B
:1000D00028B11DF005FFBDE810401BF027BE10BD84
:1000E000FFF7DABF73B50368354D9B6D044604F521
:1000F000804698473C3654F079F953F061FE002170
:100100003046FDF701FBA87130462E4E0123EB71FE
:100110006DF006FD33682871DB6A2B4A93F89C303A
:100120006B7104F50055B5F85A13117013B92046D8
:1001300000F072F93368DB6A93F89C6036B195F889
:100140000E331BB975F006FAC5F8100385F80E6377
:1001500004F5405604F5365596ED900A28468DED87
:10016000010A73F0D5F9014604F553509DED010ADB
:100170000C3070F05DFA96ED900A28468DED010A7C
:1001800073F0C6F9014604F575509DED010A08307B
:100190006FF07AFD45F0CAFD45F032FA04F52D50B6
:1001A00030306BF0E7FF66F0EBF80446284674F059
:1001B000D3FA0146204602B0BDE8704066F0BCB8F4
:1001C000458900205826002089230020FFF78ABF98
:1001D00010B5094B1B78044623B100F538500C309C
:1001E0006FF0BEFC04F5A044D4F800080368BDE835
:1001F00010409B68184700BF708D0020FFF7E8BFD4
:1002000038B5054B1C6823680A461D68034B014638
:100210002046A847002038BD582600206026002030
:1002200010B574F0C7FD064C064B18602046FFF76A
:1002300009FD2046044A0549BDE8104096F0A2BFDA
:1002400060260020582600203CEA0020C9F900085A
:1002500013B500F5A043044693F89D3D23B102B0C9
:10026000BDE8104003F0D8BF00F53850002301A9C5
:100270000C3001936FF0DCF804F580403C306DF0F9
:100280004FFCD4ED460A9DED010A014604F53650B7
:1002900074F00EFA02B010BD10B500F54053D3ED66
:1002A000CF0AD1ED007A9FED157A90ED461A03F250
:1002B000C44393ED000A00F5005367EEC77A9FED43
:1002C000107A93F8803D67EEA07A20EE070A13F0CB
:1002D0000C0F00F538500C46A7EE870A14BF012119
:1002E000002160EE870A0C306EF03EFFDFED057AEC
:1002F00020EE270A84ED000A10BD00BF0AD7233C78
:1003000035FA8E3C0000C84200F5405090F9FC02DE
:10031000C31E5842584170477FB5044604F5A255A4
:10032000684618350E460DF071FA284606F00EFEA6
:1003300018B90025284604B070BD6946284607F064
:10034000B9FC0028F5D023683246DB6C69462046AC
:10035000984705460028ECD004F5495001210830A3
:1003600071F00CFCE6E70000F0B52DED028B0446C1
:1003700000F5A25087B018300D46174607F088FBED
:10038000064600283DD03FB104F5805292F8D4369D
:1003900043F0020382F8D43604F5BE40303022F038
:1003A000D9F9D5ED017A9FED197A9FED198AF8EE0A
:1003B000E77A04F5AA4467EE877A503417EE900A7C
:1003C000FCF79AF8D5ED037AF8EEE77ACDE9040167
:1003D00067EE887A17EE900AFCF78EF8D5ED027A70
:1003E000F8EEE77ACDE9020167EE887A17EE900A17
:1003F000FCF782F8074ACDE90001062120464AF0C1
:10040000E1F8304607B0BDEC028BF0BD0AD7233CC3
:1004100095BFD633842D0B087FB500F58056054671
:1004200096F8D4369A0716D405F5A25468461834BF
:100430000DF0ECF96946204607F03CFC58B105F593
:10044000866009F097FF96F8D436DB0705D4694635
:10045000204607F01DFB04B070BD04F51B71684613
:100460000DF064FCF6EE007AB4EEE70AF1EE10FA55
:10047000EDD5F0E7F8B500F580463C360446304649
:100480006DF04EFB054618B94F4B00221A80F8BD9F
:1004900004F5005797F97D33002BF5D004F5A04300
:1004A000D3F800080368DB68984720B92046FFF7B7
:1004B0002BFF0028E8D004F5405393F94033002B7C
:1004C00040D007EE903A9FED417AF8EEE77A04F5D6
:1004D000A25367EE877A93ED887AB0EEC77AB4EECE
:1004E000E77AF1EE10FA03F118030ADC93ED817A52
:1004F000B0EEC77AB4EEE77AF1EE10FACCBF012580
:1005000000252046FFF700FFF0B1002DBFD048F0D6
:1005100057F90C21012248F0AFF82046FFF7F4FE0E
:1005200004F5AA435033014600283CD0284A002154
:1005300018464AF047F830460122BDE8F8400C2141
:10054000FDF760B91D46DCE72DBB04F5805303F6CB
:100550005C029FED207AD2ED007AF4EEC77AF1EEDC
:1005600010FA91DA03F26C73D3ED027AF0EEE77AC7
:10057000F4EEC77AF1EE10FA86DA04F53653D3EDCD
:100580000A7AB1EE047AF0EEE77AF4EEC77AF1EE89
:1005900010FA3FF579AF0C4A138801339BB2132B45
:1005A0001380B2D9B3E718460B4A4AF00BF804F5AA
:1005B000BB4113225831204604F0ACFE97F97D333D
:1005C000022B7FF464AFB6E78888002035FA8E3CB2
:1005D000A42D0B080AD7A33DB52D0B082DE9F04D2E
:1005E00088B0044648F0ECF8054674F0BBFF04F50B
:1005F000C0430746D3F8183204F5C440B3F10008ED
:1006000018BF4FF001080E4649F00EFC0068FBF7DA
:1006100073FF824604F5C4400C308B4649F004FC5D
:100620000068FBF769FFCDE904ABCDE90601CDE930
:100630000076054B054A0649CDF80880284647F064
:100640004BFE08B0BDE8F08DCC2D0B08D12D0B086A
:10065000ED2D0B0873B5044600F580403C306DF07D
:100660005FFA04F5AA45503504F5C04648B90023A1
:10067000154AC6F818320221284649F0A3FF02B0F5
:1006800070BD04F5385069460C306EF0D1FE00287C
:10069000EDD0694604F5C44049F0C8FB04F5365373
:1006A00004F5C4409B6A019301A90C3049F0BEFBDC
:1006B00074F050FF0023C6F81802C6F81C3220461A
:1006C000FFF78CFF014AD6E7F42D0B08102E0B081C
:1006D00070B52DED028B00F5C04686B0D6F8183205
:1006E0000446002B51D000F5C4400C3049F09CFB6F
:1006F00090ED008A04F5C44049F096FBB2EE047A0E
:10070000D0ED007AB4EEC78A04F5AA45F1EE10FAEE
:10071000CDED057A05F150053BDB9FED217AB4EE76
:10072000C78AF1EE10FA34D89FED1E7AF4EEC77A3C
:10073000F1EE10FA2DDBFDEEC87A04F50D5017EE40
:10074000903A0DF113012E308DF813303FF094FAEA
:1007500004F50D5005A920303FF024FA04F50052AD
:1007600092F96E33D2F860030393FBF7C5FE039B47
:100770000D4ACDE900010221284649F023FF00235C
:10078000C6F818322046FFF729FF06B0BDEC028BF1
:1007900070BD064A0221284649F014FFEFE700BF6A
:1007A0000000C84200000034282E0B084B2E0B0816
:1007B0007FB500F5C0450446D5F81832A3B300F55F
:1007C000385001A90C306EF033FE68B3174E039613
:1007D00003AA01A904F5C44049F096FB04F5365379
:1007E00004F5C4409B6A029303AA02A90C30039645
:1007F00049F08AFBD5F81C320D4A5343B3F1333F1D
:1008000002D82046FFF7EAFED5F81C320133C5F8BE
:100810001C3274F09FFED5F81832C01AB0F5FA6F8A
:1008200002D32046FFF754FF04B070BD0AD7A33CA3
:10083000CDCCCCCC13B5044600F5A250183006F050
:1008400085FBD8B101A9134806F03EFE04F58040AF
:100850003C306DF065F99DF8043088B9DC06C3F3CF
:1008600000100BD49DF805209107C2F3400005D479
:100870001C07C3F3C00001D402F0010002B010BD98
:10088000D90603D41A07C3F3C000F7D583F080005C
:10089000C009F3E7B83A002070B500F50055D5ED72
:1008A000E07AF5EEC07AF1EE10FA8AB004464FF025
:1008B000000346D907930893099307AE06AB00F5EA
:1008C000A250019303AA05AB04A90096183007F0C3
:1008D00065F9304621F07CFBD5EDE07A9DED047A98
:1008E000DDED036AB4EEE70AF1EE10FAF4EEC77A32
:1008F000ACBF01230023F1EE10FAF4EEE67A77EEB6
:10090000A76A98BF0133F1EE10FA98BF0133B4EE35
:10091000E67A98BFDBB2F1EE10FA10DAF4EEC77A9D
:10092000F1EE10FA9CBF0133DBB2012B07D8204651
:10093000FFF780FF80F00100C0B20AB070BD012057
:10094000FBE70020F9E7000070B500F5A04504467C
:1009500095F818382BBB012685F8186847F030FF4A
:100960003246112147F088FED5F8000803685B6A1B
:100970009847B0B104F5005393F97E338BB1022B45
:1009800006D004F5BB4106225831204604F0C2FCD3
:1009900004F5AA40034ABDE870400221503049F0F6
:1009A00011BE70BDEDE00A0838B500F5A04304465D
:1009B00093F818288AB1002583F8185847F000FFEB
:1009C0002A46112147F058FE04F5AA40034ABDE823
:1009D00038400221503049F0F5BD38BD642E0B0877
:1009E000F0B585B0054668460CF010FF05F5A2503D
:1009F0006946183007F0A2F9D8B105F580403C30BF
:100A00006DF08EF8344C354E40B105F50053D3ED02
:100A1000E07AF5EEC07AF1EE10FA0CD8238823F4D0
:100A2000FF7323F00103238028460023F373FFF7AD
:100A3000BBFF05B0F0BD2846FFF72EFF074688B381
:100A40006378DB0705D423780133DBB2092B05D8A3
:100A50002370637803F00103F373EAE7238823F438
:100A6000FF7323F0010343F48573238047F0A8FE4E
:100A70000222102147F000FE74F06CFD6368C01A7A
:100A800047F23053984209D905F5AA40144A022189
:100A9000503049F097FD74F05DFD60602846FFF727
:100AA00053FFD6E72378002BD3D0013B2370238854
:100AB000C3F30803B3F5807FCBD1637860F3000301
:100AC000637047F07DFE3A46102147F0D5FD284679
:100AD000FFF76AFFBDE700BF8C8800204589002032
:100AE0007C2E0B0810B5044674F028FD0E4AB4F8AD
:100AF000BE1013888B420D4B02D01180186010BDC0
:100B00001B68C01A0A4B9842F9D904F580443C345A
:100B100020466DF005F80028F1D020460122BDE8FE
:100B200010400621FCF76EBE9488002098880020B3
:100B3000400D03002DE9F84F00F5A045914604460D
:100B400095F808280E46002B71D042EA010385F87B
:100B5000083822B91BB174F0FDFCC5F80C0895F8F3
:100B6000103853B195F808383BB904F5AA404B4A00
:100B70004B460621503049F025FD95F8103895F880
:100B80000828134085F81038002B40F08580002A93
:100B900000F0828074F0DEFCD5F80C38DFED406A9E
:100BA000C01A04F5005A07EE900A9AEDDD7AF8EEC5
:100BB000677A27EE267AF4EEC77AF1EE10FA6BDD4B
:100BC000D5F8003804F5C24808F14808434563D019
:100BD00004F5BB475837BB4205D104F54053D3F861
:100BE000443DDB0758D504F5AA4B95F808382D4A43
:100BF00085F810380BF1500B4B460421584649F04C
:100C0000E1FC51F075FDD5F8002804F5BD437833BB
:100C10009A4214D1012E0DD19AF97833022B0ED1BC
:100C20005846214ABDE8F84F042149F0CBBC22EADE
:100C300001038CE7022E02D19AF97C33EEE79AF990
:100C40007033013B042B27D8DFE803F00B110318A6
:100C50001D0004F5C34119220431204604F05AFB5B
:100C6000D0B919224146204604F054FBA0B93946B8
:100C700020461922BDE8F84F04F04CBB04F5C341EF
:100C800019220431EFE704F580400122BDE8F84F56
:100C900014213C30FCF7B6BDBDE8F88F8C2E0B0854
:100CA00000007A44A02E0B08AC2E0B08013A10B5B8
:100CB0000446042A2AD8DFE802F00A12031B2000A7
:100CC000042200F5C341114404F024FBF0B904F5FB
:100CD000C24104224831204604F01CFBB0B904F59F
:100CE000BB4120460422BDE81040583104F012BB3D
:100CF000042200F5C3411144EDE700F58040BDE852
:100D00001040012207213C30FCF77CBD10BD0000E3
:100D10002DE9F84300F5095700F50058103704464F
:100D20000021384698F88C925BF0F0F904F5804683
:100D30003C36054630466CF0F3FE002846D0002DC8
:100D400041D098F956325BB3294638465BF044FAF5
:100D5000DFED1F7AB4EEE70AF1EE10FA19D898F930
:100D60005632013B042B1BD8DFE803F00B130322A0
:100D7000270004F5C3410A220431204604F0CAFAD0
:100D800070B904F5C2410A224831204604F0C2FA83
:100D900030B904F5BB410A225831204604F0BAFAB2
:100DA00047F00EFD2A460921BDE8F84347F064BC30
:100DB00004F5C3410A220431E7E701220F2130463E
:100DC000FCF720FDECE7B9F1000FE9D1BDE8F883AD
:100DD0000000C84201207047002070470120704782
:100DE0000120704710B50368DB680446984748B196
:100DF000E368DFED067A03F5C75393ED040A20EEAE
:100E0000270A10BD9FED020AFBE700BF0AD7233C6B
:100E10000000000010B50368DB680446984748B13D
:100E2000E368DFED067A03F5C75393ED030A20EE7E
:100E3000270A10BD9FED020AFBE700BF0AD7233C3B
:100E40000000000010B50368DB680446984728B12D
:100E5000E36803F5C75393ED050A10BD9FED010A42
:100E6000FBE700BF0000000010B50368DB68044624
:100E7000984728B1E36803F5C75393ED020A10BD04
:100E80009FED010AFBE700BF0000000010B50368FA
:100E9000DB680446984738B1E06800F5CB50BDE800
:100EA0001040083003F0D2BE10BD000070B52DED2B
:100EB000028B5A4D84B0D5ED460A8DED010A0446E9
:100EC000806A0E466EF0AAFC8DED010A7EB3E068E2
:100ED00000F57766A06A6EF075FC6368D5ED461A7A
:100EE00093ED831AF6EE000A60EE200A30469FED7D
:100EF0004C0A01A95EF08EF8E06800F5CB5008308E
:100F000003F038FE98B1E66874F024FBD6F8983FF9
:100F1000C01AB0F5FA7F0AD205F5A043D3F800084D
:100F200003F64863984202D003685B6D9847E06817
:100F30009DED010A0023039300F5805393F968396E
:100F4000002B10DD00F5CB5003A9083003F0F0FFB3
:100F5000E0689DED030A00F51F6072F037FA04B0F7
:100F6000BDEC028B70BDDFED2F7ADFED2F8A9FED98
:100F70002F8AB0EEC00AB4EEE70AF1EE10FA1FD4E1
:100F8000E368A06A93F8F0395A0745D490F84413FF
:100F9000D5ED461A9DED010A1B07A36858BF90F8CE
:100FA000442393F91E60D3ED040A01EE106AB8EEF3
:100FB000C11A48BF012221EE281A6EF08BFC1DE0F9
:100FC0001648FFF7A1F90028DAD1A268E36892ED8C
:100FD000040A93F8F01992F91E3095ED461AA06AAA
:100FE00007EE903AF8EEE77AC1F3C00267EEA80A7E
:100FF0000DF10B03C1F380016EF01AFD20EE080A1B
:1010000006488DED030AFFF77FF90028A0D00348BA
:1010100003A9FFF741F99BE70121B9E7602600200A
:1010200000000000000000340AD7233C0000C84242
:101030000C4A02600C4A426002F6F86102F638720D
:10104000C2600A4A0261043242610432826104329F
:10105000C2610432026204324262A2F58E528160A1
:1010600082627047D42E0B08B83A00201866002020
:101070000368DB6D1847000037B51D4B1B68DB6A42
:1010800093F89C3004460BB301A91A4806F01CFAE9
:101090001948FFF7CFFB054620B1184B93F81858B5
:1010A00085F00105236820465B6A984700B14DB181
:1010B000236820469B6A984740B13DB99DF80430AB
:1010C0009B0703D40025284603B030BD2368204683
:1010D0009B6D984705460028F5D0236820461B6D78
:1010E0009847E06800F5CB50083003F0C1FCEAE710
:1010F00058260020B83A00206026002060760020A4
:1011000070B52DED028B2F4C94F80838DB070D4697
:10111000164605D500230B601360BDEC028B70BD35
:10112000836893F91F30012BA4F5005420D0032BC2
:10113000D4F8BC3FB3F9083007EE903AF8EEE77AFE
:10114000C2ED007A35D0002BD4F8B83FB3F908309F
:10115000FFEE007AB7EE007AB8BFB0EE677A07EE1E
:10116000903AF8EEE77A67EE877AC5ED007AD4E731
:10117000D4F8B80F51F0BEFCD4F8BC0FB0EE408AE2
:1011800051F0B8FC78EE007AB6EE007A67EE877A16
:10119000DFED0D6A38EE408A67EEA67A28EE078A00
:1011A000C6ED007ADFED097A28EE278A85ED008A00
:1011B000B3E7D4F8B83FB3F9083007EE903AF8EE49
:1011C000E77AD2E7607600200000C84200A08C4594
:1011D00070B506462DED028B0D461446FFF790FFC5
:1011E000F06800F51F6072F093F9A0B3DFED317A7B
:1011F00095ED000A722080EE270AB7EE001AFFEE86
:10120000000A1DF0BDFBDFED2C7AB0EE408A94EDB4
:10121000000A732020EE270AB7EE001AFFEE000A3C
:101220001DF0AEFBB0EEC88AB0EEC00A38EE000A80
:10123000F7EE007AB4EEE70AF1EE10FA0BDD95ED69
:10124000007AC7EE007AC5ED007A94ED007AC7EE19
:10125000007AC4ED007A194BF068D3ED460A94ED9C
:10126000000A00F51F6072F03BF9DFED157A94ED8E
:10127000007AB4EEE77AF1EE10FAB4EEE70A94BF22
:1012800001220022F1EE10FA94BF012300239A42BA
:101290000BD0B36893F91F3033F0020302BFD5EDD2
:1012A000007AF1EE677AC5ED007ABDEC028B84ED31
:1012B000000A70BD00A08C450AD7233C60260020A0
:1012C000000000B40A4B93F80828D2070DD4A3F508
:1012D0000053D3F8C03F43B1B3F9083007EE903A5A
:1012E000F8EEE77AC1ED007A7047DFED027AF9E7B0
:1012F000607600200000000070B5C36905461868DC
:101300000E46144658B151F0B5FB86ED000A2B6A23
:10131000186838B151F0AEFB84ED000A70BD0023AF
:101320000B60F4E700232360F8E7000010B5436A80
:1013300018680C4620B151F09DFB84ED000A10BDE9
:1013400000230B60FBE70000C36851B103F668722D
:1013500092ED000ADFED057AB4EEE70AF1EE10FA3D
:1013600003DA03F5805393ED500A70470000003410
:10137000C36803F5805383F8CD18704730B52DED61
:10138000028B3C4D9FED3C8A83B0002304462846E7
:101390008DF80330FEF7B8FFD4E90223DFED370AFA
:1013A00093F8F01992F91E30002848D001EE103A57
:1013B000B8EEC11AA06AD5ED461A9FED310A21EEAA
:1013C000201AD2ED040AC1F3C002C1F380016EF00D
:1013D00081FA20EE080A01A928468DED010AFEF7E0
:1013E0005BFFE06800F5CB50083003F09FFAE0683F
:1013F0009DED010A00F51F6071F0E8FF9DF80330D4
:10140000ABBBE368D5ED460A93F8F0199FED1C0AD3
:10141000A06AC1F3400201F001016EF08FF8E068AC
:10142000DFED187A012120EE270A00F51F6071F028
:10143000C7FF9DF8030003B0BDEC028B30BD07EE83
:10144000903AF8EEE77A92ED040A95ED461AA06A12
:10145000C1F3C00267EEA00A0DF10303C1F38001DE
:101460006EF0E6FA20EE080A8DED010AB9E79FED6D
:10147000040AD4E7602600200000C8420AD7233CB3
:101480000000000000A08C45B7EE007AF4EEC70A19
:10149000F1EE10FA18DCDFED107AF4EEE70AF1EE67
:1014A00010FA11D4C368DFED0D6A03F5CD53D3ED07
:1014B000037AF4EEE67AF1EE10FAB6BFC7EE207AC0
:1014C000B0EE670A20EE270ADFED050A40F27D1034
:1014D000B3EE0E1A1DF054BACDCC4C3D00000034D2
:1014E0000000000070B52DED028B044682B0154659
:1014F00001AA0E46FFF704FEA3689DED010A93F9C9
:101500001E20DFED200A07EE902AF8EEE77A20EEA3
:10151000208A204667EEA00A93ED040AFFF7B4FF85
:1015200028EE000A184B85ED000AE068D3ED460A64
:1015300000F67C206EF072F9DFED147A95ED007AFA
:10154000B4EEE77AF1EE10FAB4EEE70A94BF0122A6
:101550000022F1EE10FA94BF012300239A420BD02F
:10156000A36893F91F3033F0020302BFD6ED007A6F
:10157000F1EE677AC6ED007A85ED000A02B0BDECA7
:10158000028B70BD0AD7233C60260020000000B407
:10159000F8B5324F2DED028B0446D7F8B80F0E4642
:1015A000154651F0A7FAB7EE001AFFEE000AA62082
:1015B0001DF0E6F9D7F8BC0FB0EE408A51F09AFA68
:1015C000A720B7EE001AFFEE000A1DF0D9F9A368B4
:1015D00093F91F30012BF0EE408A09D178EE008A92
:1015E00038EE407AF6EE007A68EEA78A27EE278A70
:1015F000F0EE680AB0EE480A96F00CF9DFED187AC2
:1016000020EE270A1DF050F986ED000A28EE080AA0
:10161000A8EEA80A1DF0E4F8A368DFED120A93F91A
:101620001E20F7EE007AB4EEE70AB0EE408AF1EE43
:1016300010FA58BFB0EE678A07EE902AF8EEE77A04
:1016400093ED040A67EEA00A2046FFF71DFF20EE87
:10165000080ABDEC028B85ED000AF8BD605600203B
:10166000A00CB3450AD7233C30B52DED028B83681F
:101670009B7F053B5F2B83B00546F0EE408A0C460E
:1016800021D801AA6946FFF73BFDAB68DFED200AD0
:1016900093F91E209DED018A93ED040A07EE902A2E
:1016A000F8EEE77A28EE208A284667EEA00AFFF7D0
:1016B000EBFEDFED187A28EE000AB4EEE70AF1EE51
:1016C00010FA03DBE4B1B0EE680A0DE0DFED127A48
:1016D000B4EEE70AF1EE10FA0AD8002CF3D0B4EE1B
:1016E000E80AF1EE10FAEEDC03B0BDEC028B30BD7F
:1016F000002CF4D1B4EEE80AF1EE10FAE3D4F3E7EB
:10170000DFED057AB4EEE70AF1EE10FAF2D8DAE787
:101710000AD7233C00000034000000B410B52DEDC2
:10172000028B0368DB680446B0EE408A9847A8B194
:10173000E36803F5805393F93831002B0EDDBDEEDD
:10174000C80A10EE103A1BB200EE103A2369B8EE48
:10175000C00A186851F002FBB0EE408AB0EE480AA9
:10176000BDEC028BE0680121BDE8104000F51F6070
:1017700071F026BE10B5C36893F8F019094B044602
:10178000C1F34002806AD3ED460A01F001016DF019
:10179000D5FEDFED057A204620EE270ABDE8104091
:1017A000FFF7BCBF6026002000A08C4510B59FED60
:1017B000107AC368DFED0F7A93F8F0190E4B20EE24
:1017C000070A044660EEA70A20EE270A806A93ED16
:1017D000461AC1F3400201F001016DF0AFFFDFEDE9
:1017E000077A204620EE270ABDE81040FFF796BF93
:1017F0000AD7233C35FA8E3C6026002000A08C4599
:1018000010B5836ADFED157A93EDB91AB4EEE71AD5
:10181000F1EE10FAD8BFB0EE671ADFED117A21EEC3
:10182000271A0446F1EE410A4FF4F2701DF0A8F8B1
:10183000E368A06A93F8F0190A4BC1F34002D3EDB4
:10184000460A01F001016DF091FFDFED077A2046B5
:1018500020EE270ABDE81040FFF760BFCDCCCC3D9D
:101860000AE81C416026002000A08C45102937D8CA
:10187000DFE801F0090D36111519361D3620242830
:101880002B36362F320000F5BC401030704700F583
:10189000BC404830704700F5C2400C30704700F53E
:1018A000BB405830704700F5C1404030704700F5EC
:1018B000C340FAE700F57C501830704700F5BD4092
:1018C0007830704700F5C240E3E700F5C3400430CC
:1018D000704700F5BD40704700F5BB4020307047B1
:1018E0000020704782B073B50E4606A981E80C004F
:1018F000C5680446DDE908018DE8030006AB05F57F
:1019000089500CCB31461C306FF01AFC40B1E368B3
:1019100003F5C75318331B68E362002384F83030A3
:1019200002B0BDE8704002B07047000070B52DED08
:10193000028BC368554D03F5805303F6D40293F828
:10194000CD1892ED000A0029B7EE007AFFEE007A7A
:1019500008BFF0EE477A044682B027EE800AFFF710
:1019600083FEE06841F23C16B0EEC00A30446EF0EF
:101970005BFDE06895ED460A30446FF0DFFBE06800
:1019800000F5C753183300F5CB501B68E3620830ED
:1019900003F0F0F878B1E66873F0DCFDD6F8983F14
:1019A000C01AB0F5FA7F06D205F5A045D5F80008B3
:1019B00003685B6D9847E368226803F5C753126EAE
:1019C00093ED000A002120469047E06800F5895019
:1019D0001C306FF0A7FBE06841F668163044B0EEAB
:1019E000408A03F047F9E56808B3A819B0EE480A41
:1019F00003F074F9E0688DED010A304403F032F928
:101A00009DED010A80B1E36803F58053B3F94A31D3
:101A100000EE903AF8EEE00A204602B0BDEC028BF0
:101A2000BDE87040FFF7C2BEDFED190AF4E705F527
:101A3000C75393ED018A73F08DFDD5F8983FC01A16
:101A4000B0F5FA7F17D2A06A6DF0DAFEA36AD3ED83
:101A5000B67AF5EEC07AF1EE10FAD8BFDFED0C7A67
:101A6000B0EEC00AB4EE670ADFED097AF1EE10FAC3
:101A700098BFB0EE678AB0EE480A204602B0BDECCF
:101A8000028BBDE87040FFF775BE00BF60260020E6
:101A9000000000000120704700487047382F0B08F5
:101AA0000120704700207047F0B52DED028B85B006
:101AB00001A90446806A3D4D6DF0BAFC03AA02A953
:101AC00000284DD12046FFF783FB2846FEF71CFC7B
:101AD00018B103A92846FEF7DFFBE0689DED030A75
:101AE00000F51F6071F072FCDDED027A9FED307A37
:101AF000F0EEE77AF4EEC77AF1EE10FA05D4E0687A
:101B000000F5CB50083002F0B3FFE0689FED298A62
:101B100041F66816304403F0A5F8E36858B3981905
:101B2000A76A02F0B1FFE36895ED461A93F8F01941
:101B300003F58053C1F34002B3F94A3100EE903A05
:101B400001F00101F8EEE00A38466DF0F7FD20EEF5
:101B5000080A2046FFF7E2FD05B0BDEC028BF0BDA0
:101B60002046FFF7BFFC23689DED030A1B6E012191
:101B700020469847B8E7DDED027A93F8F0199FED1B
:101B80000E7AD5ED460AA06A87EE880A03F6B4639A
:101B9000C1F3400201F00101D3ED007A67EE877ACC
:101BA00020EE270A6DF0CAFCD1E700BF60260020B6
:101BB0000000003400A08C4535FA8E3C08B5C068A2
:101BC00000F51F6071F0A4FC80F00100C0B208BDF8
:101BD000C06800F5CB50083003F00CB80A207047FD
:101BE00000487047AC2F0B080120704790F8300177
:101BF00000F0FD00031F58425841704790F83C30F8
:101C0000012B02D1383020F02BBB704790F97020A7
:101C100022B190F8711009B9FFF7AABB7047000014
:101C200010B504460348FFF727FA10B1022384F8E1
:101C3000303110BDA887002030B52DED028B90F813
:101C4000324183B00546002C39D1AB6893F91510A9
:101C50004A1C52D1D3ED067A9FED307AF0EEE77A46
:101C6000F4EEC77AF1EE10FA53D4AB689FED2B7AFD
:101C7000D3ED067AF0EEE76AF4EEC76AF1EE10FAF9
:101C800049D4274B93F8842D0C2103F6980301FBCC
:101C9000023393ED808AF4EEC87AF1EE10FA3AD866
:101CA0004FF068FB044618EE100AFAF725FC1D4AAF
:101CB000CDE900010421204648F084FC29E0836836
:101CC00093F915104B1C13D01548C9B203F0A4FCAE
:101CD000012809D14FF04EFB134A042148F072FC51
:101CE000002485F8324103E095F83231002BACD066
:101CF000204603B0BDEC028B30BD0948C9B203F0E9
:101D00008BFC0028B1D14FF035FB084A042148F084
:101D100059FC0124E5E70024EAE700BF0000003495
:101D200060260020DF2F0B08B42F0B08C72F0B08ED
:101D300010B504460348FFF79FF910B1032384F858
:101D4000303110BD2087002010B5B0F86C30012B69
:101D5000044607D84FF00EFB114A052148F032FC2B
:101D6000002010BDC0689FED0F0A00F589501C309F
:101D70006FF068F800230C4884F8323101F052FB10
:101D80000A4803F067FC18B12046FFF7D1FF10B9ED
:101D9000052384F83031012084F83101E1E700BFE8
:101DA000FC2F0B0800000000E084002060260020CB
:101DB00070B505460E480C46FFF75EF9B0B1042336
:101DC00085F830310A4801F033FBA3680BB9E368AA
:101DD00053B194E80F0005F5A27686E80F00054997
:101DE00030460BF0F5FD012385F8543170BD00BF7E
:101DF000E0840020CC7D00201FB590F854310446CB
:101E00002BB373F0A7FBD4F858311BB1C31AB3F549
:101E10007A7F1CD90DF10F03C4F8580100930D48C7
:101E20000DF10E030DF10D0212214AF005FB70B108
:101E30004FF0A0FA03689DF80F101B6998479DF8B2
:101E40000E209DF80D1004F5A2734EF015F904B0A4
:101E500010BD00BFF98B002010B5144A137804465A
:101E600043F0800313704FF085FA114A052148F0C2
:101E7000A9FBE36803F5805393F93031022B0BD0B3
:101E8000032B0FD0012B03D12046FFF751FF10B9D0
:101E9000052384F8303110BD06490822064803F0B6
:101EA00039FAF4E705490822F8E700BF6489002001
:101EB00018300B08A88400206026002070840020C1
:101EC0002DE9F04701F108030446884691460FCBFF
:101ED00092B003AE86E80F00274930460BF078FD3C
:101EE000B8F9043023EAE372A4F83A2100229342BD
:101EF0000DAFC4F83C21C8BF4FF0010938460BF0C4
:101F000085FC07AD0DF1240AB9F1000F15D0236847
:101F100028465F6C0BF07AFC9AE803008DE803001A
:101F2000314695E80C002046B84718B1002384F8E4
:101F30004031012012B0BDE8F087B8F8001001313F
:101F40000BAA89B204F1380022F0AAF90028DED0E9
:101F500097E80F0085E80F00314628460BF038FD62
:101F60009AE803008DE80300276895E80C003146E5
:101F70007D6C2046A847D8E7CC7D002037B50446C5
:101F80000D4673F0E7FAC4F868011C4803F062FBE1
:101F900018B12046FFF7CCFE10B9052384F8303184
:101FA000D5ED027AF5EEC07AF1EE10FA16DD9FED6E
:101FB000147A67EE877AFCEEE77AC4ED597A4FF02F
:101FC000D9F9D4F864214FF47A73B2FBF3F30D4AD4
:101FD000062103B0BDE8304048F0F4BA59F0BAFB2E
:101FE0000023009395F90D2095F90E3095F90C100A
:101FF00059F04CFBC4F86401E1E700BF6026002003
:1020000000007A442C300B088B8813B10831FFF79D
:10201000CFBE704738B59FED180A0B7C2DED028BB3
:1020200091ED028A044628EE008A0D4653B14368BA
:1020300093ED800AB8EEC00A30EE080A1CF04AFCA4
:10204000B0EE408AE36895ED030A03F5805393ED03
:10205000501A40F22F30F1EE410A1CF091FC84ED51
:102060000D8ABDEC028B002384F83831012384ED06
:102070004D0A84F8303138BD0000C84273B503689A
:102080009B6C05460E469847044640B395F8403190
:102090009BB9B5F83A31012285F8402113B34FF0CE
:1020A00069F9B5F83A31134A00930621338848F0AC
:1020B00089FA73F04FFAC5F83C01B5F83A3173B1BB
:1020C00073F048FAD5F83C41041B4FF47A70B4FB26
:1020D000F0F4B5F83A01844234BF002401242046CC
:1020E00002B070BD4FF046F93388034A062148F02C
:1020F00069FAE2E73C300B0868300B0810B504467B
:1021000073F028FAD4F86831C01AD4F864319842D0
:102110004FF0000084BFC4F86401012010BD00002E
:1021200003689B6C1847000010B5FFF7A7FF044633
:1021300028B14FF01FF9034A042148F043FA204622
:1021400010BD00BF80300B0810B590F83031042B63
:10215000044618D18B88B3B190F8543123B9BDE847
:1021600010400A4801F072B900F5A27108480BF05E
:10217000DDFDE36803F58053D3ED517AB4EEE70A51
:10218000F1EE10FAEBD8012010BD00BFE084002072
:10219000CC7D00207FB501F108030C4606460FCB2D
:1021A0006D4685E80F00124928460BF011FC628845
:1021B000A388122A4FEA132305D1227ED20744BFF7
:1021C00003EB83035B00F068227A07EE903A00F598
:1021D000DC50B8EE670AC2F340022946083000F02E
:1021E0002DFF10B1072386F8303104B070BD00BF59
:1021F000CC7D00200B799FED0F6A07EE903A0B7EA5
:102200009B07C36848BF9FED0C7AF8EE677A03F529
:10221000DC5348BF67EE877A93ED247AB0EEC77A35
:10222000C7EE066AF4EEE76AF1EE10FAACBF0120E1
:1022300000207047DB0FC9400000803B38B50446E2
:102240000D4673F087F9C4F86001D5ED027A9FED71
:10225000047A67EE877AFDEEE77AC4ED577A38BDE7
:1022600000007A4410B5044673F074F9D4F8603174
:10227000C01AD4F85C3198424FF0000084BFC4F813
:102280005C01012010BD000010B503680446DB6B43
:102290009847D4ED577AF8EEE77A0020B4EEE70AD3
:1022A000F1EE10FA44BFC4F85C01012010BD00003B
:1022B00010B54B885C2B02460C4671D041D8103BC0
:1022C00099B2042936D94FF055F863883E4A042163
:1022D00048F078F947E0C23B132BF4D801A151F83C
:1022E00023F000BF6723010867230108C722010804
:1022F00067230108C7220108C7220108C722010875
:1023000067230108C7220108C7220108C722010864
:10231000C72201086723010867230108C7220108B3
:10232000C7220108C7220108C7220108C7220108E5
:10233000B9230108042BC6D8DFE803F01A23282D9F
:102340001F00722B34D007D85D2B2DD0702BBAD143
:10235000BDE81040FFF786BFD52B06D8C12BBAD8F1
:10236000B23B012BAFD801200FE0DE2BFBD0AAE758
:102370002146BDE81040FFF781BEBDE81040FFF7E1
:10238000CFBE2146FFF77AFE002010BD2146BDE8F2
:102390001040FFF72FBF2146BDE81040FFF7C4BE35
:1023A000BDE81040FFF7D0BEBDE81040FFF7A6BE65
:1023B000BDE81040FFF768BF92F83031012BD2D151
:1023C00092F83801E1E700BF98300B0838B50D46A8
:1023D000FFF76EFF044620B14EF0CCFF29884CF089
:1023E00053FA204638BD000037B50368D1F80920FC
:1023F000DB6C00EE102A0C46984768B14EF0BAFF2D
:102400000546D4F80900FAF777F8044ACDE9000147
:102410000621284648F0D6F803B030BDB4300B088A
:1024200089884B1E59425941FEF7A2BF8B8891ED16
:10243000040A03484FF47A71594300F0EFBF00BF1C
:10244000E084002030B5684B1B68DB6A93F89C3051
:1024500085B0044633B9B0F86C30012B9CBF05231E
:1024600080F8303194F83131E3B168460BF0CEF9A1
:102470006068694605F062FC50B104F1380022F052
:1024800003FB002384F8313104F5B6701FF080FEA1
:1024900094F83031072B43D8DFE803F02444878DCC
:1024A0009381969C04F5B6701FF072FE04F1380516
:1024B00080B194F83C30012B0CD194F830314BB9F9
:1024C000284622F04FF948B14EF054FF474A022106
:1024D00048F078F8284622F073F9D9E74EF04AFF21
:1024E000434AF4E7434803F0B5F828B9204605B05D
:1024F000BDE83040FFF71ABAE06800F589501C309B
:102500006EF0F4FD0028F1D0E36803F5805393F8F2
:102510008C38002BEAD12046FFF70AFC0028E5D0D2
:1025200005B030BD94F8383183BBDFED330A94ED4C
:102530000D0A2046FFF73AF9DFED307A94ED4D0AA7
:102540002368B4EEE70AF1EE10FA94BF01210021EE
:1025500020461D6EFFF788F801212046A8476368D2
:10256000D4ED0D7A93ED807AB8EEC77A77EEC77A1C
:102570009FED237AF0EEE77AF4EEC77AF1EE10FAE7
:102580004CBF0123002384F83831C9E7194803F010
:1025900061F820B12046FFF7CBFB0028C0D12046D0
:1025A00005B0BDE83040FEF7E9BE164805B0BDE80D
:1025B000304001F083BB144805B0BDE8304001F065
:1025C00069B92046FFF718FC104805B0BDE8304057
:1025D00000F07CBFE06800F5DC50083005B0BDE8D5
:1025E000304000F0E7BB00BF58260020C4300B0885
:1025F000EC300B086026002000000000000000B452
:102600000000FA43A887002020870020E0840020F3
:1026100013B504468DED010A0091FFF70DFB0099FB
:102620009DED010A28B9204602B0BDE81040FEF732
:10263000A5BE204602B0BDE81040FEF737BC000042
:1026400090F83031072B1FD8DFE803F0041E0E117D
:10265000151E1518C36803F5C75393ED040ADFED83
:102660000C7A20EE270A70470A48FEF7BBBB0A4BDC
:1026700093ED3D0AF3E7094800F0E8BDC06800F5B6
:10268000DC50083000F018BA9FED050A704700BF13
:102690000AD7233CA887002060860020E084002021
:1026A0000000000090F83031072B1FD8DFE803F05E
:1026B000041E0E11151E1518C36803F5C75393EDBC
:1026C000030ADFED0C7A20EE270A70470A48FEF76E
:1026D000A1BB0A4B93ED3D0AF3E7094800F0D2BDD8
:1026E000C06800F5DC50083000F0B8B99FED050A6D
:1026F000704700BF0AD7233CA887002060860020CF
:10270000E08400200000000090F83031072B17D83B
:10271000DFE803F004160A160D160D10C36803F562
:10272000C75393ED050A70470748FEF78BBB074870
:1027300000F0C4BDC36803F5DC5393ED260A70476F
:102740009FED030A704700BFA8870020E0840020A7
:102750000000000090F83031072B19D8DFE803F0B3
:1027600004180A0D0F180F12C36803F5C75393ED31
:10277000020A70470848FEF777BB0848FBE708489D
:1027800000F0A4BFC06800F5DC50083000F048B984
:102790009FED040A704700BFA88700202087002013
:1027A000E08400200000000090F83031072B19D899
:1027B000DFE803F00418070B0F180F1290ED0B0A57
:1027C00070470A4B93ED5D0A7047084B93ED3B0A47
:1027D0007047074800F080BDC36803F5DC5393EDF4
:1027E0000D0A70479FED030A704700BF6086002006
:1027F000E08400200000000038B590F830310C462D
:10280000072B2CD8DFE803F0042B14191E2B1E23F2
:10281000C06800F5805393F8CC583DB100F589505D
:102820001C306EF075FC0FC884E80F00284638BDD8
:10283000BDE838400B4801F083BABDE838400A488B
:1028400001F020B8BDE83840084800F055BFC06826
:1028500000F5DC50BDE83840083000F0E7B800254E
:10286000E4E700BFA887002020870020E084002044
:1028700082B037B50D4606A981E80C000446DDE9B3
:1028800008018DE8030006AB0CCB29462046FFF774
:1028900029F810B1002384F8303103B0BDE830408E
:1028A00002B0704790F83031062B11D8DFE803F002
:1028B00004100A100D100D00C06800F589501C307E
:1028C0006EF014BC034801F0F3B9034800F0F2BD08
:1028D00001207047A8870020E084002090F8303164
:1028E000072B1BD8DFE803F0040A0E1A1104111499
:1028F000C06800F589501C306DF086BD80ED4D0A32
:1029000001207047064801F089B9064800F0F8BC7C
:10291000C06800F5DC50083000F042BB0020704772
:10292000A8870020E08400208B88012B08D107486D
:1029300090F81C3823B10021A0F5A040FDF7ECBCB5
:10294000034800220831FDF70FBD00BF607600206C
:102950006026002038B54B88702B04460D4642D0C7
:1029600010D8142B08D80F2B0AD9113B032B20D8D1
:10297000DFE803F02A2C2A265C2B2BD05D2B2FD0EE
:10298000002020E0C22B37D00CD8B22B2ED0B32B96
:102990002FD0722BF4D1D1ED027AFDEEE77AC0EDA3
:1029A000577A0FE0D52B18D0DE2BE9D1FFF73EFD8B
:1029B00008E0002229462046BDE83840FFF780BAEB
:1029C000FFF72EF9012038BD0122F3E7BDE83840BA
:1029D000FFF7E0BBFFF718FBF4E7FFF71BFBF1E79E
:1029E000FFF7CCFAEEE7FFF729FCEBE7FFF7FCFC7B
:1029F000E8E7FFF799FFE5E7FFF712FDE2E70000E0
:102A00000920704700487047C11A0B080120704721
:102A100090ED240A7047000090ED0B0A704700000B
:102A2000C36803F5CD5393ED740A704738B500F1D0
:102A3000440305460C460FCB84E80F00DFED067A11
:102A400095ED1B0AD5ED170A204620EE270A0BF05C
:102A5000E3F9012038BD00BFE02E654207B5C0682C
:102A600000F5CD5018306DF0A1F9DFED107A8DED45
:102A7000000AB0EEC00AB4EEE70AF1EE10FACDEDAE
:102A8000010A06D5F0EEE00AF4EEE70AF1EE10FADC
:102A900009D468461EF064FBDFED057A20EE270AB4
:102AA00003B05DF804FB9FED030AF9E70000003472
:102AB000E02E65420000000010B586B000230446F9
:102AC0000093019305F034FB694604F093FA18B9BA
:102AD0009FED130A06B010BD636F226F0492694622
:102AE00004A805931EF0CAFADFED0E7A8DED020AF6
:102AF000B0EEC00AB4EEE70AF1EE10FACDED030A2B
:102B000006D5F0EEE00AF4EEE70AF1EE10FADFD4B3
:102B100002A81EF025FBDFED047A20EE270AD9E794
:102B20000000000000000034E02E654210B50446AD
:102B3000FEF77EFA20460B4B40F8443B0AF066FE57
:102B40000023204608496365A36523676367A3677D
:102B5000E367C4F88030C4F884303CF041FA204682
:102B600010BD00BF54320B080C320B081FB50023F8
:102B700004460093019305F0DBFA694604F03AFA43
:102B800030B905F0D5FAD0F80C32E36604B010BDC8
:102B900004F1540168461EF071FA02A88DED020A94
:102BA000CDED030A1EF026FBDFED077AB0EEC00A7A
:102BB000B4EEE70AF1EE10FAE3D402A81EF0D0FA60
:102BC00084ED1B0AE2E700BF0000003413B5D0ED2E
:102BD000170AC3689FED217A90ED1B0A426DF6EE4D
:102BE000007AF4EEE70ADFED1E7AF1EE10FA03F553
:102BF0006B63B8BFF0EE477A93ED007A90F88C30B3
:102C00000267B4EE677AF1EE10FAC8BFF0EE477AC9
:102C100090ED247AB4EEE77AF1EE10FA98BF43F023
:102C20000103DFED107A80F88C3000F17001836DC4
:102C30004367044620EE270A084601911EF080FBF8
:102C4000E068094B019993ED460A00F5CD50183024
:102C500002B0BDE810406DF06BB800BFCDCCCC3DEC
:102C6000CDCC4C3EE02E65426026002030B52DEDE7
:102C7000048BC3684B4D90ED180A03F5CD5393EDCB
:102C8000611AF6EE007A21EE271AD5ED467A21EE8A
:102C9000271AD0ED1A7A044630EE670A85B0D320A1
:102CA000F1EE410A1BF06CFED4ED1A7A94F89430E0
:102CB00070EE277AF0EE408AC4ED1A7A002B6CD1C0
:102CC000DFED396A94ED177A636E95ED469A94EDCF
:102CD0001B0A27EE267A002B87EE878ABFEE007A42
:102CE00028EE268AF7EE007A18BFF0EE477A28EE33
:102CF000278AA9EE080A1BF02FFED4ED227A84ED74
:102D00001B0AE9EE087AC4ED227A94ED1B0ADFED86
:102D1000277AA36D626DD4ED170A226704F1700162
:102D2000084620EE270A636703911EF009FBA36E95
:102D300094ED1B0ADFED1E7AA36704F178020023ED
:102D4000104630EE270AE36702921EF01FFBD4ED17
:102D50001A7AD5ED466A94ED176A94ED1B0A67EE70
:102D6000E77A88EEA67A04F1800318460193C7EE4D
:102D7000866A84ED217AC4ED206A1EF007FBE068C4
:102D80000399DDE9013200F5CD50183005B0BDECF6
:102D9000048BBDE830406CF0D9BF2046FFF7E6FE5B
:102DA000B3E700BF60260020DB0FC940E02E65427C
:102DB000DB0FC93F30B52DED028B8BB000230446ED
:102DC0000293039305F0B4F902A904F013F930B9A2
:102DD0002046FEF7D3FA0BB0BDEC028B30BD04F1F8
:102DE000540102A81EF04AF9636F226F079302A9EB
:102DF00006A8CDED050A06928DED040A1EF03EF9F7
:102E000008A8CDED090A8DED080A1EF0F3F904A813
:102E100084ED0B0A1EF0EEF9D4ED177A94F88C309D
:102E200030EE670AB0EEC00A84ED240AEBB9204602
:102E3000FFF7CCFEE068344B00F5CD5093ED460A29
:102E400018306DF0E7F8E36803F5CD5393ED730A9E
:102E500093ED728A2046FEF78DFC236801211B6EDC
:102E6000B0EE480A20469847B5E7B6EE007AE36828
:102E7000F4EEC77A9FED257ADFED257AF1EE10FAB0
:102E800003F56B63B8BFF0EE477A93ED007AB4EECA
:102E9000677AF1EE10FAC8BFF0EE477A37EEA77AFC
:102EA000B4EEC70AF1EE10FA1BDD94F8943023BBA0
:102EB0009FED187AD4ED187A67EE877AC4ED187A08
:102EC0004EF058FA0546206EF9F716FB124ACDE986
:102ED00000010421284647F075FB012384F8943053
:102EE000A8E7B4EEE70AF1EE10FA02D594F89430B0
:102EF00043B92046FFF7BAFE9CE7B4EEE70AF1EECD
:102F000010FAF6D50023E9E760260020CDCCCC3DB1
:102F1000CDCC4C3ECDCC4C3F8C310B0837B5C36883
:102F2000DFED1B7A03F5566393ED000AB4EEE70A72
:102F3000F1EE10FAD8BFB0EE670ADFED167A20EE98
:102F4000270AD0ED177A20EE270A04461BF048FC2A
:102F5000B5EEC00AF1EE10FAD8BF9FED0F0AD4ED1E
:102F6000187AF4EEC07AF1EE10FA0EDD84ED180A4C
:102F70004EF000FA0546206EF9F7BEFA074ACDE991
:102F800000010421284647F01DFB03B030BD00BFFF
:102F9000CDCCCC3D0AE81C4100000000B8310B0844
:102FA000DFED137AB4EEE70AF1EE10FA10B504463D
:102FB0001CDB80ED180AFFF7B1FFE06894ED180AFA
:102FC00000F5CD53D3ED607AB4EEE70AF1EE10FAD6
:102FD00003F1180308DDD3ED5D1A93ED5C1AD3ED10
:102FE0005B0A18466CF01CFE012000E0002010BDBA
:102FF0000000003437B5C36890ED177A03F56B63B2
:10300000D3ED007AB4EEE77AF1EE10FA044611D56A
:10301000C0ED177A4EF0AEF9E36803F56B63054631
:103020001868F9F769FA044ACDE900010421284635
:1030300047F0C8FA03B030BDD4310B08F0B52DED20
:10304000028B0D4683B00023044669462846B0EE45
:10305000408A1746009301930AF02EFD28B90026F6
:10306000304603B0BDEC028BF0BD236820469B6D5B
:10307000984706460028F2D09FED110A68461EF0D8
:103080000DF8DFED107A84ED150AB0EEC80AB4EE43
:10309000E70AF1EE10FAD8BFB0EE670AC4ED160ADF
:1030A00084ED170A2046FFF7A5FF67662046FFF765
:1030B0005DFD95E80F00443484E80F00D0E700BFC1
:1030C0000AD7233CCDCCCC3D70B504462DED048B06
:1030D00005F02EF804F1540103F08CFF0646002899
:1030E00000F09C80D4ED0E7ADFED4E9A9FED4E9A63
:1030F000DFED4E8AF0EEE77AF4EEE97AF1EE10FABF
:10310000D8BFF0EE697AC4ED177A2046FFF772FF58
:1031100094F94030D4ED0F7A5A1EF4EEC97A534236
:103120005341F1EE10FA6366BEBFE36803F58053C6
:10313000D3ED507AC4ED187A04F0FAFFD0F80C32CF
:10314000E3663B4BC4ED1A8A0FCB04F1440585E8D6
:103150000F002046FFF7E2FE002384F89430E36876
:1031600003F67C2003F6485393ED008AB4EEE88A18
:10317000F1EE10FAD8BFB0EE688A6CF023FBB4EE23
:10318000480AF1EE10FAF0EE400AC8BFF0EE480A25
:10319000E068F4EEC90AF1EE10FAF7EE007A00F5F5
:1031A0008053B8BFF0EE670AD3ED577AF4EEC97AD0
:1031B000F1EE10FA06DBF4EE670AF1EE10FAC8BF82
:1031C000F0EE670AD3ED581A9FED167A9FED191AA3
:1031D00094ED180A00F55663D3ED007AF4EEC91A9F
:1031E000F1EE10FAF4EEE97AB8BFF0EE601AF1EE03
:1031F00010FAD8BFF0EE477A41F6B81527EE811ADB
:1032000028446CF00DFDE06828446CF08BFE002330
:10321000C4ED228A84F88C30C4ED248ABDEC048B82
:10322000304670BDCDCCCC3D000000340000000025
:10323000CC7D00200AE81C410F20704700487047F1
:10324000B8320B08012070470120704790F83830E1
:1032500023B1032B0CD09FED080A7047C36803F518
:10326000C75393ED040ADFED057A20EE270A704775
:10327000034B93ED3D0AF6E7000000000AD7233C1C
:103280006086002090F8383023B1032B0CD09FEDDE
:10329000080A7047C36803F5C75393ED030ADFEDCF
:1032A000057A20EE270A7047034B93ED3D0AF6E7B7
:1032B000000000000AD7233C6086002090F83830D8
:1032C0002BB9C36803F5C75393ED050A70479FED0B
:1032D000010A70470000000090F8383023B1032B3A
:1032E00005D09FED050A704790ED0B0A7047034B20
:1032F00093ED3B0A704700BF00000000608600208D
:1033000090F838302BB9C06800F589501C306DF04A
:103310007BB800207047000030B52DED028B0125F1
:1033200087B080F838500446F0EE408AB0EE608AEC
:1033300072F010F90023E063019302930493059364
:1033400094F838100948C4ED0D8A84ED128A84F887
:10335000395003AB6A46CDED008A8DED038AFBF749
:10336000FDFC07B0BDEC028B30BD00BF6026002025
:1033700010B52DED028B022386B080F8383004465C
:10338000F0EE408AB0EE608A72F0E4F8012384F82F
:1033900039300023E063019302930493059394F87A
:1033A00038100848C4ED108A84ED128A03AB6A46CF
:1033B000CDED008A8DED038AFBF7D0FC06B0BDECA5
:1033C000028B10BD6026002010B504460348FDF7AF
:1033D00053FE10B1032384F8383010BD208700203D
:1033E00010B504460B4802F035F918B12046FFF736
:1033F000EBFF10B9052384F83830E0689FED060A2A
:1034000000F589501C306DF01DFD002384F8443018
:10341000012010BD6026002000000000C16580ED85
:10342000180A70470023C365002303667047000035
:1034300010B5044672F08EF8034B60660FCB68340B
:1034400084E80F0010BD00BFCC7D002010B5C36D17
:10345000044653B994ED187ADFED107AB4EEE77AAA
:10346000F1EE10FA0ADA002010BD72F073F8636E04
:10347000C01AE36D9842EDD30120F5E7084804F146
:1034800068010AF053FCD4ED187AB4EEE70AF1EEC5
:1034900010FACCBF01200020E6E700BF0000003496
:1034A000CC7D0020C36803F58053D3F8780BC0F3BC
:1034B0008010704790F838302BB9C06800F58950FB
:1034C0001C306DF013BE01207047000070B590F8FD
:1034D00038300446052B00F2D880DFE803F0032DD6
:1034E000709FA44AC06800F589501C306DF0FEFD45
:1034F00020B92046BDE87040FEF718BA94F8443071
:103500002BB10021654884F844104BF0BDF96448A4
:1035100002F0A0F818B12046FFF756FF10B9204678
:10352000FDF72CFFE1685F4801F5C5510C310AF049
:10353000FDFB84ED0B0A70BD90F8393083B172F059
:1035400009F8E36BC01A40F6B833984216D94DF02B
:1035500011FF554A042147F035F8002384F839302B
:103560004F4802F077F820B12046FFF72DFF0028E2
:10357000E1D12046BDE87040FDF700BF94F8393036
:10358000002BEDD0DFED490A94ED0D0A2046FEF741
:103590000DF994ED120ADFED467A2368B4EEE70ADE
:1035A0001D6EF1EE10FA204694BF01210021FEF7B6
:1035B0005BF820462B460121BDE87040184790F883
:1035C0003930002BCCD071F0C5FFE36BC01A40F648
:1035D000B8339842BBD894F83930002BC0D0E36898
:1035E000D4ED107A9FED330A93F8F0192C4BA06AB2
:1035F000D3ED460A67EE807A9FED2F0AC1F34002B1
:1036000027EE800A01F001016BF098FFDFED2B7AC5
:10361000204620EE270AFEF781F8BAE7BDE87040A1
:10362000274800F037B990F84C30002B98D071F053
:1036300091FF236DC01A40F6B833984208D9002391
:1036400084F84C304DF096FE174A042146F0BAFF3C
:1036500094F84C30002B83D094ED150AE068DFED30
:10366000177A00F51F6020EE270A00216FF0A8FEF0
:1036700094ED160AE068DFED137ABDE8704020EEA5
:10368000270A00F51F606FF0A1BE4DF073FEBDE884
:1036900070400D4A042146F095BF00BFB07B00206A
:1036A00060260020CC7D0020C0320B080000000006
:1036B000000000B40AD7233C35FA8E3C00A08C45AC
:1036C000208700200000C842E9320B0890F838300B
:1036D00023B1032B08D09FED060A7047C36803F59A
:1036E000C75393ED020A70470248FDF7BDBB00BF08
:1036F000000000002087002038B590F838300C46D4
:1037000023B1032B12D00025284638BDC06800F530
:10371000805393F8CC58002DF6D000F589501C301A
:103720006DF0F6FC0FC884E80F00EDE7BDE8384007
:10373000014800F0A7B800BF2087002082B070B514
:10374000054688B00CAC84E80C00FFF7ABFEEC68D3
:1037500004F589540E461C34002833D0DDE90E01EF
:103760008DE803000CAB0CCB314620466DF0E8FC35
:1037700030B30021012485F8381085F84440EB6807
:10378000D6ED027A114803F5C653B8EEE77A143342
:10379000D6ED037A1B6805930022F8EEE77A0492CF
:1037A0000692079205AB02AA8DED027ACDED037A5F
:1037B000FBF7D4FA204608B0BDE8704002B070476D
:1037C0000020F8E720466DF0F5FAD1E760260020EA
:1037D0000420704700487047C52D0B080020704733
:1037E000002070470020704713B50023044610489E
:1037F0000193FCF789FD18B10D4801A9FCF74CFDB8
:10380000E06800F5CB50083001F090F8E0689DEDDD
:10381000010A00F51F606FF0D9FDE0689FED050A11
:10382000012100F51F606FF0CBFD02B010BD00BF9D
:103830006026002000000000052070470048704707
:10384000D8330B080120704790ED0D0ADFED027AA6
:1038500020EE270A704700BF0AD7233C90ED0D0ADF
:10386000DFED027A20EE270A704700BF0AD7233C1B
:103870009FED010A704700BF0000000090ED0B0AA9
:103880007047000010B538300C460FC884E80F00B0
:10389000012010BD30B52DED028B044683B000F140
:1038A00038017C4801910AF041FAE06884ED0B0A86
:1038B00000F5CB50083001F05DF9E368019900286C
:1038C00055D003F5CC5292ED027AD4ED0B7AF4EE9A
:1038D000C77AF1EE10FA4FD841F66815581901F081
:1038E00049F96D4BDFED6D7A9FED6D0AD3ED460A18
:1038F000002808BFB0EE670AA06A6BF08FFFE0688F
:1039000084ED120A284401F035F990B9E36803F513
:10391000805393F96829002A0BDDD3ED2C7A9FEDB3
:10392000617A67EE877A9FED607A67EE877AC4EDF9
:103930000D7AE06894ED0D0A41F66815284401F00F
:1039400099F9002840F08D80DFED540A94ED0D0ABE
:103950002046FDF72BFF236894ED120A1B6E012110
:10396000204603B0BDEC028BBDE83040184703F59C
:10397000805292ED137AA8E703F5805303F51B629A
:1039800077EEC77A92ED007A4248DFED488A67EE1B
:10399000877A93ED507AF4EE477AF1EE10FA48BF49
:1039A000B0EE677A84ED127A0AF0DAF8B6EE008AA1
:1039B0009FED3F7A6368F0EE487AE0EE077AFDEE1D
:1039C000E77AF8EEE77AC4ED0D7A93ED800AB8EE67
:1039D000C00A37EEC00A1AF07DFFF0EEC07AF4EEAE
:1039E000E87AF1EE10FAE36804DD03F5805292F90B
:1039F00049202AB103F5805393F94930022B18D19D
:103A0000DFED2C7A94ED0D0A30EE270A1AF062FFF2
:103A1000636884ED0D0AD3ED807AF8EEE77A30EE34
:103A2000670A1AF057FFD4ED127AF1EE677AC4ED07
:103A3000127AC0EE287A3620DFED180AB0EEE70AD7
:103A4000B7EE001A1AF09CFFF7EE007AE0EE487A23
:103A5000B0EE677AD4ED127A67EE877AC4ED127A07
:103A600067E7E06894ED0D0A284401F037F9E06853
:103A700084ED0D0A284401F0F5F800283FF464AF06
:103A8000E36803F58053B3F94A3100EE903AF8EE5B
:103A9000E00A5BE7CC7D00206026002000000000EB
:103AA000CDCCCC3DE02E65420000C84200A00C46C3
:103AB000A00CB34500A08C4638B50446C06800F59C
:103AC000895004F138011C306CF010FD054670B1CE
:103AD000A06A04F148016BF0ABFC08B90023A364B1
:103AE0006368D3ED807AF8EEE77AC4ED0D7A284664
:103AF00038BD000000207047004870474C340B0868
:103B00000120704700207047002070470020704758
:103B1000C0689FED030A00F51F606FF073BC00BF23
:103B20000000000010B52DED028B86B0044601AAFE
:103B30006946FDF74DFB204602A9FDF7C3FBE3688C
:103B40009FED2D8A9DED000A03F5DC5380EE080AF7
:103B5000D3ED000A1BF0C2FB20EE080A27488DEDCA
:103B6000000AFCF7D1FB18B1244801A9FCF794FB2B
:103B700004AA03A92046FDF7BFFB05A92046FDF7CF
:103B8000D5FBE0689DED030A00F51F606FF04AFC6D
:103B9000E0689DED040A00F51F606FF04FFCE068DF
:103BA0009DED050A00F51F606FF056FCE06800F51A
:103BB000CB50083000F0D6FEE0689DED010A00F51C
:103BC0001F606FF003FCE0689DED000A00F5805374
:103BD00000F51F60D3F87C1B01F001016FF0F0FBD2
:103BE000E0689DED020A00F51F606FF00BFC06B067
:103BF000BDEC028B10BD00BF00A08C4560260020EC
:103C00000B207047004870474CF00A0801207047AD
:103C10000020704790ED0B0A70470000C06800F567
:103C200089501C306CF0F0BB70B58AB0044604F0CB
:103C30007FFA90F87C32DB0702D400200AB070BD16
:103C4000E36803F5895003F6687393ED000AB5EE57
:103C5000C00AF1EE10FA48BF9FED130A1C306DF058
:103C6000F1F86368E66893ED9C0A104A06F5825104
:103C70001031B8EEC00A02A806AD3CF00DFA284695
:103C800009F0C4FD0AAB13E903008DE8030006F553
:103C9000895095E80C0002A91C306DF051FA0028FB
:103CA000CBD001232387C9E700000000CC7D002092
:103CB000C06800F589501C306DF018BA10B5044684
:103CC000C06800F589501C306DF010FA20B920460C
:103CD000BDE81040FDF72ABE94F8383043B1002308
:103CE00084F838304DF046FB114A062146F06AFC54
:103CF000104801F0AFFC60B92046FDF73FFBE168DA
:103D00000D4801F5C5510C310AF010F884ED0B0A8D
:103D100010BD94F839301BB10848FFF7BBFDEEE742
:103D20000648FDF7A9F984F839000028E4D0F3E744
:103D3000C0340B0860260020CC7D002020870020A6
:103D400038B5C06800F580530C4693F8CC583DB1A7
:103D500000F589501C306DF0DBF90FC884E80F00C6
:103D6000284638BD072070470048704740350B088B
:103D700013B5044601AA6946FDF70AFCE36803F59A
:103D8000805393F964304BB994ED0E0ADDED007A5F
:103D900030EE270A1AF088FD8DED000ADFED0E7A6D
:103DA0009DED017ADFED0D0AB4EEE77AF1EE10FA3F
:103DB000B5BFE36B009B0093E3639DED000A2046D3
:103DC000FDF7F4FC23689DED010A1B6E01212046DE
:103DD000984702B010BD00BF000000340000000092
:103DE0004368D3ED807AF8EEE77AC0ED0E7AD3ED32
:103DF000807AF8EEE77AC0ED0F7A70470C207047B2
:103E0000004870474BF00A080120704700207047B7
:103E100090ED0B0A7047000090F83800831E58425E
:103E200058417047C06800F589501C306CF0ECBAFE
:103E300030B590F83830012B0C460CD1C36803F52F
:103E4000805393F8CC5825B103F6AC030FCB84E82C
:103E50000F00284630BD0025FBE700001FB50446D3
:103E6000684609F0D3FC6068694603F067FF10B943
:103E7000002004B010BDE36893F8C42E002AF7D0E8
:103E800003F5895003F6687393ED000AB5EEC00A96
:103E9000F1EE10FA54BFBDEEC00A9FED0A0A1C30C5
:103EA000B8EEC00A6CF0CEFFE06800F589501C3017
:103EB0006CF068FB0028DBD0002384F8383084F8ED
:103EC0003A30D6E700000000064BC068D3F800285F
:103ED000054BD21A18BF0122012100F6B8606DF01F
:103EE00095BE00BF60760020E487002030B590F8D2
:103EF0003830012B87B0044615D004D9023B012B82
:103F000072D907B030BDC068002100F6B8606DF00E
:103F100031F910B140F201132387204607B0BDE804
:103F20003040FDF72BBA90F83930002B3AD0C068FA
:103F30000025694600F6B8600095019502956DF080
:103F400057FD48B94DF016FA344A062146F03AFBBF
:103F5000022384F83830D4E7E068039503A900F61B
:103F6000B860049505956DF075FDE56841F23C1368
:103F700038B303AA6946E8186CF082FA78B94DF0B4
:103F8000F9F9274A062146F01DFB032384F838304F
:103F900042F068FF3D224FF4801142F01BFF0023E6
:103FA00084F839302046FDF7C1FCE06800F58950FF
:103FB0001C306DF09BF80028A3D0012384F8393021
:103FC0009FE76946E8186CF035FA0028E7D14DF014
:103FD000D1F9134A062146F0F5FA032384F8383064
:103FE00042F040FF4522D6E7012380F830300D48EB
:103FF00001F030FB002890D094F83A302BB10A48F9
:1040000007B0BDE83040FFF745BC0748FDF734F87E
:1040100084F83A00002880D0F1E700BFC0340B08D4
:10402000B4350B086026002020870020032070474D
:10403000004870475B080B0801207047002070475C
:104040000120704790ED0E0A7047000070B52DED0D
:10405000048B84B0044601A9806A6BF0E9F9B0B919
:104060009FED4E8AE068B0EE480A00F51F606FF0E1
:10407000ADF9E0680121B0EE480A00F51F606FF06D
:104080009FF984ED0E8A04B0BDEC048B70BD03AAC9
:1040900002A92046FDF726FADFED418A9DED039A3D
:1040A000E0689FED408AB4EEE89AF1EE10FA00F570
:1040B0001F6094BF012600266FF02AFAE368A56A04
:1040C00098B3DDED037A9FED387AF0EEE77AF4EEFF
:1040D000C77AF1EE10FA28D5DDED027A9FED337A3A
:1040E00087EE880A03F6B4622846D2ED007A0022F1
:1040F000A26393F8F0192E4B67EE877AC1F3400262
:10410000D3ED460A20EE270A01F001016BF016FA02
:10411000204620EE080AFDF701FB23689DED030A07
:104120001B6E012120469847ADE703F56B63DFED79
:10413000210AD3ED007A95EDB97A9DED010A9FED44
:104140001E1AF4EEE07AF1EE10FAB4EEE07AD8BF7F
:10415000F0EE607A20EE000AF1EE10FAD8BFB0EE71
:10416000607A27EE011A80EE270A26201AF008FC52
:10417000314620469DED027AC7EE087AB4EEE89A01
:1041800027EE800AF1EE10FA98BFB1EE400A84EDF6
:104190000E0A94ED0E0AFDF733FBBEE700000000A7
:1041A000000000B400A08C450000003435FA8E3CBD
:1041B00060260020CDCCCC3D0AE81C4170B500F54E
:1041C000A046044696F89D3DF3B16AF095FE03685B
:1041D000012203219B6898470C4B00251D6004F5C4
:1041E0000D500B4B3C301D603AF0D0FF04F50D50E4
:1041F00038303AF0CBFF04F50D503D303AF0C6FFB1
:10420000044B86F89D5D5D7270BD00BFA0880020E4
:10421000A48800204589002037B500F5A043044656
:1042200093F89D3D002B32D071F094F9274B1B6819
:10423000C01A274B1B68984205D3204603B0BDE83F
:104240003040FFF7BBBF234B1B78012B10D0022B54
:104250001FD0E3B9204BB3F9003000EE103A1F4BEA
:10426000B8EEC00A197804F536506FF041FE0CE044
:10427000194BB3F9003000EE103A184BB8EEC00AF3
:10428000197804F536506FF083F90028D5D003B0C3
:1042900030BD124B1978022904F5365504F5405308
:1042A0000BD1D3F8B80F01914EF024FCDFED0C7A5E
:1042B000019920EE270A2846D7E7D3F8BC3FB3F987
:1042C000083000EE103AB8EEC00AF4E7A0880020EB
:1042D000A4880020A8880020AA8800209C880020AC
:1042E0000000C8422DE9F843984600F5A0439DF828
:1042F000206093F8FC57BDF924700C463DB9224A62
:104300000221204649F0BCFB2846BDE8F8836AB18B
:1043100000F5804001213C30F9F756F930B91B4ACD
:104320000221204649F0ACFB0025EDE7184B1B6845
:10433000D86A0368DB699847012801D1154AEFE77D
:10434000B8F1040F06D9144A43460221204649F029
:1043500097FBE9E7022E02D9104A3346F5E7012E12
:1043600006D140F698039F42CEDD0D4A3B46ECE76E
:10437000002EC9D1642FC7DD0A4A3B4602212046E0
:1043800049F07EFB3546BFE7B0360B08CF360B0849
:1043900058260020ED360B0807370B0826370B0888
:1043A0004C370B086A370B082DE9F0432DED028BD3
:1043B00000F5A04583B01E4695F89D3DBDF93080BF
:1043C00004461746B0EE408A2BBB1346721E18BF38
:1043D0000122CDE90068FFF785FF28B9042003B06A
:1043E000BDEC028BBDE8F0834FF0010985F89D9D7F
:1043F00004F580453C35284669F092FB50B304F53E
:104400000054002384F87C3384F8783384F87D33B7
:10441000144B01225A7271F09DF89FED130ADFEDE3
:10442000137A134B28EE000A1860B4EEE70AF1EE97
:1044300010FA58BFB0EE670A0E4BBCEEC00A00205F
:1044400083ED000A0C4B1F700C4B1E700C4BA3F835
:104450000080C4E74A4603212846F9F7A9F9002855
:10446000CDD1BBE74589002000007A440060EA46D0
:10447000A0880020A48800209C880020A888002014
:10448000AA88002073B500F50E561436054630464E
:104490004EF006FA05F54054C4F8B80F30464EF019
:1044A00013FAC4F8BC0F30464EF018FA41F29411DA
:1044B000C4F8C00FD4F8B80F4EF060FAD4F8BC0FAF
:1044C00064214EF05BFAD4F8C00F10B164214EF0B5
:1044D00055FAC92130464FF0A9F9CA21C4F8C40FD2
:1044E00030464FF0A3F9D321C4F8C80F30464FF03F
:1044F0009DF9C4F8CC0FD4F8C40F40B141F2941127
:104500004EF03CFAD4F8C40F1E214EF03BFAD4F81A
:10451000C80F40B141F294114EF030FAD4F8C80FF0
:104520001E214EF02FFAD4F8CC0F40B141F2941175
:104530004EF024FAD4F8CC0F1E214EF023FA05F5E4
:104540007350383000F0F4F805F580403C3069F0E5
:10455000E7FA38B905F5365001906EF005FF01987D
:104560006EF0E2FE084B1B685B6A4FF47A7205F549
:104570001B50DA8046214FF4FA6224301A8102B0CF
:10458000BDE870404FF0AABC5826002010B500F5D9
:1045900040541E21D4F8B80F4EF0F4F9D4F8BC0FF3
:1045A0001E214EF0EFF9D4F8C00F20B1BDE8104045
:1045B0001E214EF0E7B910BD70B500F50053054659
:1045C00093F978230C46DAB1B3F97A6370F0C2FF3D
:1045D00005F5A043D3F81438C01AB0F5FA7F0DD80A
:1045E000B3B29C422CBF00230123064A9372284693
:1045F000054ABDE870400121FCF79CBA0123F4E7AD
:1046000070BD00BF4589002090370B082DE9F843A5
:1046100000F58043054693F94C90B9F1000F0BD09B
:1046200000F5405805F5A044D8F8BC0F4EF014FB37
:1046300020B90023C4F87C3DBDE8F883D4F8000815
:1046400003685B6998470028F3D005F580463C363F
:10465000304669F065FA0746B8B9D8F8B83FB3F9FB
:104660000830B3F57A6FE4DD70F074FFD4F87C3D68
:104670006BB3C31AB3F5FA6FDED301223946304665
:10468000F9F796F8C4F87C7DD6E7B9F1020FD3D1DB
:1046900005F5365070F060F805460028CCD1D8F802
:1046A000B83FB3F9083013F57A6FC2DA70F052FFF1
:1046B000D4F87C3D5BB1C31AB3F5FA6FBCD30122C9
:1046C00029463046F9F79EF8C4F87C5DB4E7C4F893
:1046D0007C0DB1E738B5044600F50E5014304DF0AE
:1046E000C1FF04F5405538B9D5F8BC3F2046D988FC
:1046F000BDE83840FFF760BF70F02CFF04F5A04321
:10470000C3F81408D5F8BC3F2046D988FFF754FFFA
:104710002046BDE83840FFF779BF000010B50349D7
:1047200004463AF05DFC204610BD00BF04380B087B
:1047300010B504464EF0DCF8CF214FF077F848B1C1
:10474000606264214EF01AF9606A1E21BDE81040D3
:104750004EF018B9024BD3F8BC3F636210BD00BFE6
:104760006056002038B52DED088BDFED627A624D82
:104770009FED62BAD5ED460ADFED61BADFED618AE1
:10478000F0EE40AA90ED040A044620EE270A5E48A7
:104790006AF0E0FD05F55053D3ED0E7A9FED5B7A9C
:1047A00067EE877ABFEE008AF4EECB7AF1EE10FA6C
:1047B000B7EE001AF4EEEBAA88BFB0EE418AF1EE34
:1047C00010FA20EE28AAB0EEE79A76DB94ED030A01
:1047D00094ED021AD4ED010AD32039EE400A1AF002
:1047E000CFF8F0EE680AB0EE401A94ED022AD4ED4C
:1047F000011A9FED470A1AF003F8DFED450A3AEE79
:10480000000AD820B0EE681A1AF0BAF841486EF0E3
:1048100031FEF4EECBAAF1EE10FADFED3A7A3D4824
:10482000B4EEE8AAF7EE009ABFEE000A88BFB0EE39
:10483000690AF1EE10FA48BFF0EE4A7A78EEE78A9C
:1048400068EE888A28EE800A6EF026FEF4EEEBAA67
:10485000F1EE10FA4BDB94ED037AB4EEC97AF1EE87
:1048600010FA44DCDFED2C8A77EE287AF4EEC97A70
:10487000F1EE10FA24DDDFED296AF0EE697AEAEE56
:10488000667AF5EEC07AF1EE10FAD8BFDFED207A45
:10489000A7EE679A28EE091A94ED022ADFED190AAD
:1048A0009FED1F0AF1EE421A19F0AAFFBDEC088B2A
:1048B0001848BDE838406EF001BEB0EE680AA5E7C2
:1048C000DFED187AB4EEE79AF1EE10FA0CDD8920EC
:1048D0004FF0A8F99FED141AB4EECB0AF1EE10FADE
:1048E00088BFB0EE681AD7E728EE281AD4E79FED04
:1048F000080ADBE735FA8E3C60260020000000B491
:10490000000000340000C8426C540020E02E6542D4
:1049100000000000E05300200000B4420AD7233C0E
:104920000000C8C2000007430000B4C207B59FEDF5
:104930000A0A0A486EF09EFD9FED090A07488DEDB0
:10494000010A6EF0A9FD9DED010A044803B05DF86F
:1049500004EB6EF0B3BD00BF0000C842E05300207E
:104960000000000038B5224D95F80838DB070446F2
:1049700001D4436A23B92046BDE83840FFF7D6BFCB
:10498000B3F908309FED1B1ADFED1B0A00EE103A59
:10499000B720B8EEC00A19F0F3FFA5F50A506EF083
:1049A00069FD636A9FED131AB3F90830DFED130A4E
:1049B00000EE103AB820B8EEC00A19F0E1FFA5F5F4
:1049C0000A506EF069FD636A9FED0A1AB3F9083068
:1049D000DFED0A0A00EE103AB920B8EEC00A19F06D
:1049E000CFFFA5F50A50BDE838406EF067BD00BFA7
:1049F000607600200000C842000000000000C8C22D
:104A000013B5164801A96AF013FD18B3144CD4F875
:104A100000080368DB68984718B99DED010A02B0E9
:104A200010BDA4F59C53D3ED007A9FED0E7AA4F54A
:104A3000665467EE877A14ED070A9FED0B7A97EEBE
:104A4000870A19F089FF92F0C3FCDDED017A20EEB0
:104A5000270AE4E79FED050AE1E700BF6C54002058
:104A6000607600200AD7233C35FA8E3C0000000017
:104A700010B5002380F8283080F83C3003630446EA
:104A800070F068FDA06310BD10B5114B90ED0B0ADE
:104A9000D3ED007A30EE670A044619F05DFFDFEDD2
:104AA0000D7AB0EEC00AB4EEE70AF1EE10FA05D5C1
:104AB0002046FFF7DDFF94ED0B0A10BD70F04AFDB4
:104AC000236BC01A41F288339842F1D8F3E700BF54
:104AD000C43C0020C2B8323E70B5054616460C46AE
:104AE00009B92C6470BD0C486EF012FD0028F8D195
:104AF00046204FF027FA0028F3D1084B93F9D8331A
:104B0000002BEED1002EEDD04CF034FCBDE870400F
:104B1000034A042145F056BDE053002060560020B2
:104B200098370B0810B5036C012B044601D0002008
:104B300010BD90ED067ADFED0C7AB4EEE77AF1EE77
:104B400010FAF4DB09486DF01FFD0028EFD0084B88
:104B5000D4ED067A93ED007AB4EEE77AF1EE10FA2E
:104B60004CBF01200020E3E700000034585A002029
:104B7000FC5A002008B590F90020002A08DD036CDB
:104B8000022B05D0FFF7CEFF80F00100C0B208BDB8
:104B90000020FCE713B590F90030002B04460EDD31
:104BA000002311488DF807300DF107013BF036F86E
:104BB000236C0E4A023B18BF012382F81E3C20469C
:104BC000FFF7D8FF38B1012309488DF807300DF100
:104BD00007013BF023F800220121204602B0BDE886
:104BE0001040FFF779BF00BFA05900206056002099
:104BF000395A002010B52DED028B0446FFF7BAFF9D
:104C0000E0B194F82830CBB9012384F828300D4B5B
:104C100093ED008A0C4B93ED000A30EE480A19F030
:104C20009BFEF0EE007AA0EE278AB0EE480A19F05B
:104C30007DFE84ED0B0A70F08DFC2063BDEC028BD1
:104C400010BD00BFC43C0020A05A002010B504468F
:104C5000FFF790FF28B194F8283013B970F07AFC70
:104C6000206310BD10B50446FFF784FF08B194F827
:104C7000280010BD10B52DED028B0446B0EE408A21
:104C8000FFF778FF00B394F82800E8B9DFED107A59
:104C9000104B27EEC87A93ED000A9FED0F8AA7EE1E
:104CA000080A19F059FED4ED057AB2EE047A77EECF
:104CB000877AB0EEC00A67EE887AB4EEE70AF1EEC2
:104CC00010FA94BF01200020BDEC028B10BD00BF84
:104CD0000AD7233CA05A002035FA8E3C2DE9F84330
:104CE0002DED048B0446B0EE408AFFF743FF81466A
:104CF000002800F0D980DFF83482DFED807ADFED24
:104D0000808A98F8B87408F58863D3ED009A67EE46
:104D1000C87AB0EE699AA7EEA89AB0EE490A19F0DF
:104D20001BFED4ED057A67EEA87AB0EEC00AB4EEA9
:104D3000E70AF1EE10FA40F3A68094F82830002B31
:104D400040F0A180B0EE490A19F006FEDFED6D7A61
:104D5000B4EEE70AF1EE10FA8CBF012300239F4264
:104D600000F0A28008F58763D3ED007AB0EEC00AA8
:104D7000F0EEE77A37EE800ADFED637AB4EEE70A09
:104D8000F1EE10FA40F190804E4670F0E3FB236B99
:104D9000054653B14EB994F8282032B9C31AB3F579
:104DA000FA7F2CBF00260126226308F6844898ED7E
:104DB000007AD4ED077AF0EEC76AF4EEE76AF1EE16
:104DC00010FA1EDBDFED516AF0EEE77AF4EEE67AD8
:104DD000F1EE10FA15D4A6B994F828308BB9B4EED8
:104DE000E67AF1EE10FA02DB7B1E5E425E41DFEDF9
:104DF000457AB4EEE77AF1EE10FA02D8002F08BF38
:104E00004E46D4ED057A9FED428AB0EE690AA7EED0
:104E1000A80A19F08BFDD4ED057AB0EE409AB0EEF9
:104E2000690AA7EEE80A19F081FDDFED3A9AF0EE83
:104E3000408A86B3A36B41F28832EB1A93422AD997
:104E40004CF098FA344A062145F0BCFBEFB1012F33
:104E50001ED0012384F828306563304B94ED0B0A93
:104E6000D3ED007A30EE670A19F076FDDFED2C7A8B
:104E7000B0EEC00AB4EEE70AF1EE10FA1AD82046F6
:104E8000FFF7F6FD2CE000267FE7C4ED0B8AE0E794
:104E900084ED0B9ADDE794F82830002BDDD10FBBB1
:104EA00029EE299A29EE088AB0EE480ABDEC048B57
:104EB000BDE8F883606B41F288332D1A9D420FD90B
:104EC000236C012B13D107EE905A9FED167AF8EE62
:104ED000677AF4EEC77AF1EE10FA08D584F83C3020
:104EE000D4ED0B8A68EEA98A28EE888ADCE74CF0BC
:104EF00041FA0D4A062145F065FBC0E70AD7233C7D
:104F000035FA8E3C000000B4DB0F4940000000344D
:104F10000000C842E02E6542BC370B08C43C0020AC
:104F2000C2B8323E00606A46CE370B086056002099
:104F300038B52DED028B00230B6090F90030002B6B
:104F40000446B0EE408A0D4606DCBDEC028B2046DE
:104F5000BDE83840FFF7EABC036C022B2ED11D4A96
:104F60009FED1D1AD2ED461A02F50053D3EDD80A73
:104F700093F96E0393F8801D07EE900AF8EEE77A36
:104F8000C1F3C00227EE811AC1F38001B0EE480AD6
:104F900003F60C606AF09EFCDFED107A20EE270A23
:104FA00085ED000A236C022BCFD0B0EE480ABDEC91
:104FB000028B2046BDE83840FFF7D4BB012B03D15C
:104FC00090F83C30002BCAD12046FFF7ABFD0028FB
:104FD000C5D1E7E7602600200AD7233C0000C8427D
:104FE00000F2545009F0DABB10B5044609F0C6FCD3
:104FF00090F921308BB190F8403373B194F9783542
:105000005BB104F580403C3068F08AFD28B904F2B9
:105010005450BDE8104009F0D9B910BD2DE9F04356
:105020002DED028B00F5005783B097F8603B0646E4
:10503000002B00F0938000F52B542C34204666F0B2
:10504000B3FE4FF0000897F8602B5FFA88F5AA428C
:105050000CD92946204666F0FBFE05F5BB5506EB4C
:10506000850585ED000A08F10108ECE706F5A04585
:1050700095F8883DEBB9012285F8882D1D4697F8F3
:10508000603B5FFA85F94B4568D94946204666F092
:10509000BFFE06EB890808F5A04808F68C5383ED9F
:1050A000000A4946204666F079FF0135C8F8940D9C
:1050B000E5E795F89C3D0133DBB2934228BF00231E
:1050C00085F89C3D95F89C1D204666F0A1FE95F85C
:1050D0009C1D2046B0EE408A66F060FF074670F0E7
:1050E00039FA95F89C1D06EB810303F5A04303F6FE
:1050F0008C52D2ED008A82ED008AD3F8942DA7EB72
:10510000020808F1FF3CBCF1630F84BF0746A0EB27
:105110000208C3F8947D204666F072FE95F89C1D47
:105120000190204666F060FE07EE908ADFED0E0AE1
:10513000019AF8EE677A78EE688A06F5A25067EE73
:10514000A00AB0EE401A3946B0EE680A183003B033
:10515000BDEC028BBDE8F04321F020B903B0BDECFB
:10516000028BBDE8F08300BF6F12833A10B504468E
:1051700000F570603BF0B8FA2046BDE81040F9F742
:1051800071BD0000F9F7A4BF0148FBF7ABBC00BF3D
:105190006026002070B52DED048B00F540530446C9
:1051A00093F9FC32022B54D000F50053F6EE008A3E
:1051B00093F96E3308EE103AB8EEC88AF2EE0E7A22
:1051C00028EE288A00F53855B4EEE78A0C3500F54C
:1051D0003656F1EE10FA284658BFB0EE678A96EDC3
:1051E0000A9A6AF0FDFA48B128466AF009FBB4EE63
:1051F000E80AF1EE10FACCBF01200020B4EEC98A13
:10520000F1EE10FA04F5A04509D496ED0A7ADFED27
:10521000127AB4EEE77AF1EE10FA16DBA8B170F06C
:1052200099F9D5F8783D0BB9C5F8780DD5F8783DE2
:10523000C31AB3F5FA6F94BF0023012304F5805419
:1052400084F86137BDEC048B70BD0023C5F8783D50
:10525000F4E70023F2E700BF0000003408B5044A79
:105260000B2341F075FC80F00100C0B208BD00BF07
:1052700030390B0838B5044600F5AA40154A062116
:10528000503045F09FF9144B1B68986A036804F589
:10529000A2555B68642118359847284601F038FC10
:1052A00004F58053012283F8612783F86C26B4F952
:1052B000A43004F698001BB9B4F8A230A4F8A430C6
:1052C000B4F8A41018F0B8FE2846BDE8384001F044
:1052D00025BD00BFA4380B085826002070B50B6808
:1052E0000B4EDB68054608460C4698473074236829
:1052F00020461B689847F070236820465B689847F3
:10530000014605F5A0500430BDE8704036F000BFFE
:10531000458900202DE9F04700F5A0470646D7F85B
:1053200000388B420C46914665D000F5AA48022A07
:1053300008F1500816D10B6808461B6898470146CB
:105340003046FFF78BFF054660B9236820465B684F
:1053500098472A4A03460521404645F033F9284636
:10536000BDE8F0872046D7F800A8FBF785FE054684
:1053700088B943F025FA236806461B6820469847FB
:105380000A210246304643F077F91D4A042140467F
:1053900045F018F9E3E706F50950C7F80048103062
:1053A00056F03EFFD7F8000803681B689847A0F145
:1053B0000A035842584106F5005487F8EC07504656
:1053C000FBF756FE84F80C93D7F8000803681B68B7
:1053D0009847014606F58D5094F80C23103042F0A2
:1053E00017FD404600214CF0BFFBD7F800183046AF
:1053F000FFF774FFB3E70125B1E700BFD4380B080E
:1054000014390B0873B505460A4801920E46FCF79D
:105410002DFA019A044630B10146064802B0BDE8B3
:105420007040FFF777BF2846314641F0D7FA204653
:1054300002B070BD602600200148FFF7E3BF00BF47
:10544000602600202DE9F043044604F5A04600F54F
:10545000A05087B0043036F00FFED6F80018204672
:10546000FFF73CFF04F5B0404C3005F04BFC04F571
:105470007F5018304FF054F904F5935008304FF036
:10548000CDFC04F59B5104F54F501C3104F58665A5
:1054900038306DF07FF8284605F0A8FA04F5AA40E8
:1054A000503049F059FA04F5804078305AF03EFA0D
:1054B00009F064FA4FF40063036309F05FFA0AF03D
:1054C000D5FA04F5005904F580534FF48062802723
:1054D000C9F8E8710021C3F8AC2104F570603BF015
:1054E000FDFC01212846C4F8447405F00FF904239B
:1054F000C4F8743104F5907010F0C8FA04F54058FF
:105500004FF40023C4F8883D2046FFF73FF898F891
:10551000D8133C4F04F536506EF002FB4EF066FF98
:105520004EF04EFC04F52B502C3066F00BFC04F5CD
:105530009E50103051F068FB04F5AE407C3006F010
:10554000E5FD314B31491B68986A03684FF47A7264
:10555000DB6A984704F5BB4504F54950083020350F
:105560006BF06EFF1A2229462046FFF7D3FE204635
:10557000FFF780FE04F5BE4030301EF0A5FA04F5BA
:10558000C0434FF480725A62214B0593049706ABD7
:1055900004F58D5013E90600103042F06DFA99F8C9
:1055A00059132046FCF762F91A22002814BF01465D
:1055B00029462046FFF7AEFE04F50E50143099221E
:1055C000292101904EF074F99B22052101984EF09B
:1055D0006FF901984DF034F90E48FFF7DBFA98F9AE
:1055E000FC32022B08D101230DF10F0107F55350B6
:1055F0008DF80F303AF012FB012386F8FC3707B024
:10560000BDE8F0836026002058260020895101085B
:10561000855101085863002070B50A4B1D68E86980
:10562000036800225B680C469847E86903682146D6
:105630001B6901229847E86903682146DB68BDE8D9
:10564000704018475826002000F58D50103043F068
:1056500081B8000000F5405090F9FC02831E5842CA
:105660005841704713B50446143000F0F1FE04F1C0
:105670002C0000F0EDFE04F1740071F05FFB04F10A
:10568000F40071F05BFB4FF0FF331549C4F8503163
:10569000204639F0A5FC00230DF1070104F1280094
:1056A0008DF807303AF0BAFA01230DF1070104F141
:1056B00029008DF807303AF0B1FA0F230DF10701F8
:1056C00004F125008DF807303AF0A8FA054B1A6866
:1056D00012B105486FF00CFF20461C6002B010BDEF
:1056E000EC3A0B08AC8800203C390B082DE9F04758
:1056F0008CB003A938F03EFD60B300210D2208A84C
:1057000007AF1C4CDFF87080DFF8709007910B2614
:1057100094F07AFA0697237ADFF864A08DF81430B3
:10572000002554F825300493D8F80000E368B5B993
:105730000093C06A53461122394615F0E1FB00215F
:10574000B7EE000A03A838F019FF35B1013E04F1A5
:105750001004E0D10CB0BDE8F0870125E1E701932A
:105760000223009311224B463946C06A15F0C8FB4C
:10577000E5E700BF8C3B0B085826002099390B0841
:1057800090390B082DE9F74FD0F85431044683BB0C
:10579000DFF88CA1074600F1740800F5AA75012610
:1057A000721ED2B297ED070A0192404671F0E6FAF6
:1057B000FB69C8F83C304FF07E53C8F8483097F981
:1057C0002830019A013B5FFA86FB0E2B20D8DFE8D8
:1057D00003F0133E4A5760691F1F1F1F1F1F891FB9
:1057E0007A00D4F8543103B96361D4F8583103B95D
:1057F000E36203B0BDE8F08F4820019208F036FB69
:10580000814618B1019A214670F05CFAC5F8009003
:10581000286890B103689B689847002874D14BF0C2
:10582000A9FD3C4A3346032144F0CCFE286810B160
:1058300003685B68984700232B60022E07F1180766
:1058400008F1800805F10405CBD00226A8E728203E
:10585000019208F00BFB81460028D7D0019A21461F
:1058600071F054FAD2E76820019208F0FFFA8146FD
:105870000028CBD0FF23019A214670F0C5FCC5E774
:105880006820019208F0F2FA81460028BED0002379
:10589000F1E76820019208F0E9FA81460028B5D0C6
:1058A0000123E8E74420019208F0E0FA814600284D
:1058B000ACD0019A21466FF0C7FFC9F800A00023C1
:1058C000C9F84030A2E74420019208F0CFFA81469F
:1058D00000289BD0019A21466FF0B6FF0E4BC9F805
:1058E0000030ECE76020019208F0C0FA8146002801
:1058F0008CD0019A21466FF0A7FF084BC9F8003001
:105900000023C9F8243081E72B68002B95D084F858
:105910004FB192E776390B08F0A20C084C3C0B080B
:1059200024A50C0813B50446FFF7E0FE204638F026
:1059300077FD68B994F9283013B994F940303BB138
:1059400001230DF1070120468DF807303AF094F954
:1059500094F90030002B08DD94F928302BB1204653
:1059600002B0BDE81040FFF70DBF02B010BD00004F
:105970000346406C012807D0032805D0986C012805
:1059800002D0032818BF02207047000090F90030B1
:10599000002B0ADD012908D8182303FB010090F928
:1059A0002800003818BF0120704700207047000011
:1059B00037B50446FFF7EAFF9FED0B0A0D4680B1AD
:1059C00004EB81038DED010AD3F8540138B103686B
:1059D00001A9DB68984704EBC51484F865009DEDC8
:1059E000010A03B030BD00BF0000000070B50446DE
:1059F000FFF7CCFF50B104EB8104D4F8540128B177
:105A00000368BDE870401B6911461847002070BD4F
:105A10002DE9F04F2DED028B90F90030002B83B073
:105A20000646894653DD2C4B1B68D86A03685B68C1
:105A30009847044650B14BF09DFC284A062103B01C
:105A4000BDEC028BBDE8F04F44F0BCBD9FED248A55
:105A5000DFF890A0DFF890B0354606F14407B04675
:105A600021463046FFF792FF20B195F8643043B1EC
:105A700088ED068A8035043708F118083CBB0124FC
:105A8000EEE7B9F1000F03D098F92630002BF1D1E1
:105A9000D7F81021631C01933AB94BF06BFC019BC2
:105AA0005A46032144F08EFDE4E76FF053FD0022D7
:105AB000A5F87020A5F872200122A86685ED1B8A42
:105AC0003A604BF057FC019B52460621EAE703B0CF
:105AD000BDEC028BBDE8F08F58260020A4390B08DE
:105AE00000000000E2390B08BB390B082DE9F04338
:105AF0002DED028B85B004460D46B0EE408AFFF7CF
:105B000045FF98B304EBC119CF01D9F868306BB3E6
:105B10006FF020FDD9F86830C01AB0F57A7F03D352
:105B2000B9F872300F2B0CD8E31993F86520002ACE
:105B300040F08C803C44B4F872300133A4F87230E9
:105B400014E0B9F8703005F1010805F1100693B9B9
:105B50004BF010FC04EB86064346454A042144F012
:105B600031FD032373603C440023A36605B0BDEC04
:105B7000028BBDE8F08307EE903AD9ED1B6AD4F8AA
:105B80005C21F8EEE77A86EEA77A8DED037ACAB348
:105B900094F90230002B35DD07EE903AB2F90C2073
:105BA0009FED345AF8EEE75AF7EE007AE5EE857A83
:105BB000182101FB054506EE902AF8EEE66A95ED00
:105BC000066A67EEA67A37EE467A67EEA77AB0EEF7
:105BD000C77AE6EEE67AF6EE006A67EEA67AF4EEAB
:105BE000C77AF1EE10FA0DD5B0EEC66AB5EEC06A0E
:105BF000F1EE10FA06DD4BF0BDFB1F4A43460421CF
:105C000044F0E0FC182003A900FB084004EB8606E2
:105C100039F0C8FF022373606368DB060ED54BF0D2
:105C2000A9FB05460398F6F767FC144ACDE9000185
:105C300043460621284644F0C5FC94E74BF09AFB06
:105C40000F4A4346062144F0BDFC8CE7B3F87220AE
:105C5000052A7FF66FAFD3ED1B7AB3F8702037EECD
:105C6000880A013283ED1B0AA3F8702062E700BFA7
:105C7000043A0B080AD7233C1A3A0B08473A0B0898
:105C80006E3A0B0810B590F90030002B02460C4616
:105C90001CDD90F84D31CBB9FFF778FEA8B1182183
:105CA00001FB042292F9243093B1022B0DD146203E
:105CB0004DF0B8FFDFED077AB0EEC00AB4EEE70AA8
:105CC000F1EE10FA4CBF0120002010BD0020FCE7CF
:105CD0001846FAE7000000342DE9F8432DED028B59
:105CE00004460E46FFF752FEE8B104EB81090DB2FF
:105CF000D9F85431BBB16FF02DFC04EBC6174FEA55
:105D0000C6183866D9F8540103685B69984770B1C2
:105D1000D9F85401036839469B69503198473B6D67
:105D200087F86500FB64BDEC028BBDE8F883314663
:105D3000204697F86590FFF73BFE182303FB0643C8
:105D400093ED068ABB6E30EE488A87ED178A1BB149
:105D500031462046FFF7CAFEB9F1000F43D0DFED10
:105D6000447A9FED447A04EB080368EE277AD3ED7A
:105D7000166AE6EE877A182104EB080701FB06464F
:105D8000C7ED167A96F9273083B3012B53D1DFED97
:105D90003A8AF1EE487A05EB4505B4EEE88AC7ED9C
:105DA000157A04EBC505F1EE10FA95ED070A58BF18
:105DB000F0EE687A27EE800A91F076FE87ED130AFE
:105DC00097ED160AB4EEE80AF1EE10FA48BFF1EECC
:105DD000408A95ED070A28EE800A91F065FE44445A
:105DE00084ED140A9FE7F0EE487AC4E7B5EEC08A66
:105DF00005EB4505F1EE10FA87ED158A04EBC505B4
:105E0000D8BF9FED1D8A95ED070A28EE000A91F094
:105E10004BFE04EB0803D3ED167A83ED130AF5EE7F
:105E2000C07AF1EE10FAD8BFDFED137A95ED070ACC
:105E300027EE800AD1E7B0EEC88A05EB450587ED6D
:105E4000158A04EBC50494ED070A28EE000A91F0C8
:105E50002BFED7ED167A87ED130A94ED070AF0EEC4
:105E6000E77A27EE800A91F01FFE87ED140A5AE7C1
:105E70009A99993E3333333F0000000038B50A4603
:105E80000446FFF783FD10B304EBC113CD0193F873
:105E9000653033B104EB8103D3F85431003B18BFB4
:105EA0000123182101FB0242D2ED067AF0EEE77AD7
:105EB000F5EEC07AF1EE10FA08DC2C4494F8640098
:105EC00020B992F92600003818BF0120184038BDCB
:105ED00010B500210446FFF759FD18B12046FFF721
:105EE000CDFF50B101212046FFF750FD30B12046D3
:105EF000FFF7C4FF003818BF012010BD0846FCE7BB
:105F000010B50246FFF742FD20B102EBC11292ED3F
:105F1000140A10BDBFEE000AFBE7000010B50246F0
:105F2000FFF734FD20B102EBC11292ED130A10BD50
:105F3000BFEE000AFBE7000010B50246FFF726FDA2
:105F400020B102EBC11292ED150A10BD9FED010ABE
:105F5000FBE700BF0000000010B50246FFF716FD8A
:105F600020B102EBC11292ED170A10BD9FED010A9C
:105F7000FBE700BF000000002DE9F04F2DED028B84
:105F80008DB004466FF0EEFA9FED3C8ADFED3C8A5F
:105F900080468946274625464FF0000B04F5AA7A2D
:105FA0005FFA8BF631462046FFF7F0FC002858D008
:105FB0005AF82B30002B54D06A462046FFF716FDC6
:105FC00008B9CDED008A1D22002104A893F01CFE23
:105FD000A3238DF80430952331468DF805302046F3
:105FE00072238DF80630CDF80780CDF80B908DF830
:105FF0000F60FFF793FF20468DED040AFFF79CFF2B
:10600000DDED007A8DED050A67EE887A2046FDEE1B
:10601000E77A17EE903AADF81830FFF79DFF10EED3
:10602000103A2046CDF81A30BB69CDF81E30FFF784
:1060300029FE31468DF822002046FFF71FFFD5F8D4
:10604000BC300993D5F8C0300A9394F84E318DF8DE
:1060500023008DF82C3042F0B3FB292201A941F036
:106060002FFD18378035BBF1000F04D00DB0BDEC0B
:10607000028BBDE8F08F4FF0010B91E70000C842A2
:1060800000000000F8B590F90030002B04464DDD0B
:106090000021FFF721FE01212046FFF71DFE94F9A4
:1060A0000030002B0DDD94F9403053B14BF062F914
:1060B000012105462046FFF723FF1D49284644F0ED
:1060C000F7FC667894F84E7131462046FFF7D6FE0D
:1060D000054668B901462046FFF7D0FE28B90121E0
:1060E0002046FFF7CBFE28B1012584F84E5101E090
:1060F00084F84E6120466FF085FD94F84E31BB4226
:1061000004D042F05DFB5A2142F096FAD4F85031A7
:1061100001330BD042F054FBD4F8501142F01AFB7B
:1061200020B12046BDE8F840FFF726BFF8BD00BF0C
:10613000883A0B08014B1868704700BFAC880020F4
:10614000002070477047000001207047436AC3B1C8
:10615000B0F850301BB9436D0B600120704707EE5B
:10616000903AD0ED136AF8EEE77A002386EEA77A2C
:1061700081ED007AA0F85030002380ED157AC364D9
:10618000EBE718467047000070B5044640F0ECF8A5
:106190000022222105463FF043FF606220B3002326
:1061A0001A461946062014F027FB014620466FF0D8
:1061B00085FB002222212846666A3FF051FF0146F6
:1061C000304614F077FD94F82020E369182101FB94
:1061D0000233002283F82420E36994F8202003EBA3
:1061E000C213012083F8640070BD000010B5034B9A
:1061F000036004466FF038FB204610BD4C3C0B0892
:1062000010B50446FFF7F2FF204607F037FE2046A0
:1062100010BD000073B590F8455004463DB301230E
:1062200080F846300DF10601002390F828008DF823
:1062300006308DF8073007F09BFA18B9002528467C
:1062400002B070BD94F829000DF1070107F090FA33
:106250000028F3D09DF806509DF8073043EA051357
:1062600094F84450DBB2EB1A5D425D41E7E790F8E9
:106270003830FBB990F82830413B192BDFD890F823
:106280002930413B192BDAD800F12A06174930464C
:10629000F7F7F6F810B984F84850D0E714493046BB
:1062A000F7F7EEF818B9012384F84830C7E784F807
:1062B0004750C4E790F8482042B9012BBFD1294686
:1062C000283094F0C7FF84ED100AB8E7012AB6D150
:1062D000072BB4D12946283094F0BCFFDFED057AB6
:1062E00020EE270A84ED0F0AA9E700BF3C3C0B080B
:1062F000403C0B08E4388E3E242970B504460D4618
:1063000040D016DC0A291ED00D291CD094F8373055
:106310000D2B9FBF5A1C1B1984F8372083F8285077
:1063200094F8450090B994F844104D4084F84450D6
:106330000DE02A2907D02C29E8D190F8443083F0C9
:106340002C0380F8443094F846600EB1002070BDF4
:1063500094F84730002BF9D094F837302344204686
:1063600083F82860FFF756FF94F8383084F83760D8
:10637000013384F83830A5F12A035D425D4184F889
:106380004550E4E700204FF0807384F8380084F82B
:1063900037006364DBE700002DE9F0412DED028B4F
:1063A000436A0446884623B90020BDEC028BBDE851
:1063B000F0816FF0CFF80546606A9FED248A03688C
:1063C0005B699847002687B23BB2002B26DD606AE6
:1063D00003689B699847431CE6D041B22046FFF70B
:1063E0008BFF50B194F84830E565012B08D1D4ED0E
:1063F0000F7A013638EE278AB6B2013FBFB2E3E723
:10640000D4ED137A94ED107AB4F8503077EE877AA1
:106410000133C4ED137AA4F85030EEE756B9A36DFA
:10642000C8F80030E06D281AB0F5FA6F2CBF0020D4
:106430000120BAE707EE906AF8EEE77A88EE277A4D
:1064400088ED007A84ED167AECE700BF00000000CA
:1064500010B50349044638F0C3FD204610BD00BF07
:106460006C3C0B08F0B52DED048B91B004466D46E5
:10647000284607F0CBF994F8BC33002B72D004F512
:106480007A730FCB85E80F0094F8F833D4EDEC8ADB
:1064900094EDED8A94EDEE9A002B63D094F8D0330E
:1064A000002B5FD02D22002104A8D4F8C073D4F8AB
:1064B000C463D4F8C853D4F8CC4393F0A5FBA3230A
:1064C0008DF8103095238DF8113046238DF8123059
:1064D0006FF048F89FED250A9FED257ACDF817104B
:1064E00068EE807ACDF8130067EE877AFDEEE77AE2
:1064F00017EE903A68EE007A29EE000A67EE877A86
:10650000ADF81B30FDEEE77A20EE070A17EE903A61
:10651000ADF81D3018F0C8F9DDED017A9FED157A60
:10652000CDF82D70BCEEC00AF8EEE77A10EE103A06
:1065300067EE877AADF81F3017EE903ACDF821302C
:10654000029BCDF82530039BCDF82930CDF8316082
:10655000CDF83550CDF8394042F032F92D2204A95A
:1065600041F0AEFA11B0BDEC048BF0BDE02E6542F7
:106570000000C8420AD7233C30B52DED028B8BB00A
:10658000044624220D4601A8002193F03DFBA323DD
:106590008DF8043095238DF8053048239FED1F8A30
:1065A0008DF806306EF0DEFFD4ED817A2B68CDF8E1
:1065B0000F3067EE887A95ED020ACDF80B1017EED2
:1065C000903AD4ED827ACDF8133067EE887A6B6812
:1065D000CDF8173017EE903ACDF80700CDF81B3004
:1065E00018F038F910EE103A94ED830ACDF81F3008
:1065F00020EE080A18F02EF910EE103ACDF82330EC
:1066000094F80C338DF8273042F0DAF8242201A9EF
:1066100041F056FA0BB0BDEC028B30BDE02E654266
:1066200030B587B014460D4618220021684693F015
:10663000EBFAA3238DF8003095238DF80130492320
:106640008DF802306EF08EFFA3680393E368049325
:106650006368CDF807100593CDF803008DF80B5053
:1066600042F0AEF81822694641F02AFA07B030BD70
:1066700010B58EB0044602A807F0C8F802A920465B
:1066800001F018FB002845D001F052FD694601F0E9
:10669000A9F91F22002106A893F0B6FAA3238DF8CA
:1066A000183095238DF819304A238DF81A306EF082
:1066B00059FFDDED037A9FED1B7A049BCDF8233063
:1066C000F8EEE77A059BCDF8273067EE877ACDF8AC
:1066D0001B0017EE903ADDED007ACDF82B30F1EE8D
:1066E000677A17EE903ACDF81F10204601A9CDF831
:1066F0002F3000F08DFC78B1DDED017AF1EE677A94
:1067000017EE903ACDF8333042F05AF81F2206A91E
:1067100041F0D6F90EB010BD42F052F8DFED027A2A
:10672000EEE700BF0AD7233C5241C07F10B594B0BA
:106730004FF07E5303A90393002304460693059369
:10674000049300F06BFA17F0CBFB90F8EC340C22BA
:1067500002FB030004F5577100F500701BF024F8EC
:106760003322002107A88DED000ACDED010A8DED41
:10677000021A93F049FAA3238DF81C3095238DF863
:106780001D30CC238DF81E306EF0ECFED4F814339F
:10679000CDF82730D4F81833CDF82B30D4F81C338B
:1067A000CDF82F30009BCDF83330019BCDF837303A
:1067B000029BCDF83B30039BCDF83F30049BCDF8D6
:1067C0004330059BCDF84730069BCDF82310CDF81C
:1067D0004B30CDF81F0041F0F3FF332207A941F001
:1067E0006FF914B010BD00000023036043608360A4
:1067F000C360036143618361C3610362704700004A
:1068000090F8C432B02202FB030390F8082393F8F7
:10681000A13012B1012B28BF012318467047000098
:106820002DE9F04F04468BB04FF0000A0D461FF0E3
:1068300037FA84F814A204F506704FF07E576EF014
:1068400053F84FF47A73A4F8623284F86852C4F8AB
:106850004872C4F84C72C4F8507204F51B700025DD
:1068600006F0D4FF04F52B790323C4F8803204F535
:106870003476C4F89452C4F89852C4F89C52C4F8C0
:10688000A052C4F8A452C4F8A8524846FFF7ACFF7F
:1068900004F5487B3046FFF7A7FFC4F81453C4F84B
:1068A0001853C4F81C535846FFF79EFFC4F84453CE
:1068B000C4F84853C4F84C53C4F85053C4F8545364
:1068C000C4F85853C4F85C53C4F86053C4F8645314
:1068D000C4F86853C4F86C53C4F87053C4F88C53AC
:1068E000C4F89053C4F89453C4F8A853C4F8A453FC
:1068F000C4F8A053C4F8B053C4F8B453C4F8B853A0
:10690000C4F8CC53C4F8C853C4F8C453C4F89C7337
:10691000C4F8C07304F5757006F078FF04F57A705A
:1069200006F074FF04F58063C4F8FC531D6004F5A1
:10693000816304F583601D605D609D6006F066FF05
:1069400004F22C4304F264481D605D609D606D4B51
:10695000C4F83C3404F50D73C4F8403404F50E73E8
:10696000C4F8443404F50F73C4F8483404F51073C4
:10697000C4F84C3404F24523C4F8503404F51173C0
:10698000C4F8543404F58B6340461D605D609D601F
:10699000FFF72AFF04F59160FFF726FF04F59763E0
:1069A00004F23C421D605D609D6004F2C44304F249
:1069B000BC501D605D609D6004F59A631D605D6064
:1069C0009D6004F2DC431D605D609D6004F2EC4359
:1069D0001D605D609D6004F2FC431D605D609D6014
:1069E00004F5A1631D605D609D6004F22C53C2F844
:1069F000E070C2F8E4701D605D609D6004F5A763FF
:106A00001D605D609D6004F244531D605D609D608B
:106A100004F5AC631F605D6004F284531D605D602B
:106A20009D6004F5B2631D605D609D6004F5B56313
:106A30001D605D609D6006F0E9FE04F2CC532422E7
:106A40001D605D6004F2D45351461D605D6004F228
:106A5000DC5340461D605D6093F0D6F804F2FC50B4
:106A6000C8F82070C8F81070C8F80070FFF7BCFEB6
:106A700004F5C46304F5CA601D605D609D6004F2A6
:106A80002C631D605D609D6004F5C7631D605D60E3
:106A90009D6004F244631D605D609D6006F0B6FE7B
:106AA000194B1A491C60204638F09AFA51462422A4
:106AB000584693F0A9F8C4F84073C4F83073C4F88A
:106AC000207304F5257207CA04F5287383E80700CC
:106AD000484694EDAA1AD4EDA90A94EDA80A18F034
:106AE0005DFF3546494668466E4618F079FE0FCE82
:106AF0000FC50FCE0FC533682B6020460BB0BDE825
:106B0000F08F00BF843F0B08B0880020403E0B0888
:106B100010B5044688B001F095FB94F93232012B90
:106B200002D1274804F0B8FD022B0AD1032384F8D0
:106B3000323204A9012304F111008DF8103039F02C
:106B40005DF894F8323284F8903204F23C4001F05F
:106B50002FFB94F93132642B30D1652304A904F260
:106B600031208DF8103039F087F804A9204637F02D
:106B700039FB18B304238DF818300023CDE9013315
:106B800003930F230593694604A837F0ABFC059BDC
:106B900028B108AA02EB8302009942F8581C01337D
:106BA000112B0593EFD966F051FF9DED031ADDED32
:106BB000020A9DED010A652166F006FF08B010BDCE
:106BC0002C3D0B0870B500F5257600F528758CB0C6
:106BD0000446314628461AF087FDE0B996E80700DA
:106BE00085E8070004F52B7194EDAA1AD4EDA90AE3
:106BF00094EDA80A0191084618F0D0FE02AD019963
:106C000002A818F0EDFD0FCD04F534740FC40FCDBC
:106C10000FC42B6823600CB070BD00000B4600F55C
:106C20004871184619F084BD84B000F5487004B06E
:106C300018F016BD13B540F2411200F50671044676
:106C400001A813F07FFF04F23C4001F0C1FC204694
:106C50001FF07EFA01A813F097FF02B010BD0000EC
:106C6000F8B50B68C0F804324B68C0F808328B687E
:106C7000C0F80C3201F10C0607460C4600F54875C9
:106C80000FCE0FC50FCE0FC533682B6004F1300255
:106C900007CA07F5457383E8070004F13C0207CAF9
:106CA00007F5517383E8070004F1480207CA07F5A6
:106CB000547383E80700543494E8070007F55773CA
:106CC00083E80700384601F0D1FB3846BDE8F840BC
:106CD00001F0B4BB13B5044600F23C40019003F050
:106CE000B5F804F5BE610198009102F0C5FB00996A
:106CF000204602B0BDE81040FFF7B2BF4A78064B0D
:106D0000C2F340121A754A78C2F380125A750A7893
:106D1000C2F300129A7570474589002013B540F2FE
:106D2000F522044600F5067101A813F00BFF0021BF
:106D300004F23C4001F0BEFE94F8603223B12046DC
:106D40001FF00EFC84F8600201A813F01DFF02B0D2
:106D500010BD000038B590F80C3305460C462BB139
:106D6000032B0BD095F86832DB070CD405F5CA630A
:106D70000FCB84E80F0095F8600603E01FF03EFAA1
:106D80000028EFD038BD0020FCE7000000F23C40B6
:106D900090ED380A7047000000F23C4090ED390A4F
:106DA0007047000010B490F80C230C462AB1032A57
:106DB0000AD000205DF8044B704700F5B56007C8A5
:106DC00084E807000120F5E75DF8044B1FF0FEB9E9
:106DD00090F88403431E58425841704738B590F8E4
:106DE0000C330D468BB900F23C4001F063FC0446C5
:106DF00010B90024204638BD01F0B0FBD5ED007A73
:106E000027EE800A85ED000AF4E7D0EDE07AC1EDC7
:106E1000007A90F87C43002CEBD090EDDE7ADFED29
:106E2000086AB4EEE67AF1EE10FAF7EE006AB8BF3F
:106E3000B0EE667A67EE877AC1ED007ADAE700BFD6
:106E40000000003490F80C33032B01D11FF02EB951
:106E50000020704710B490F80C43032C03D15DF868
:106E6000044B1FF02FB900205DF8044B7047000061
:106E700090F80C23032A01D11FF06ABA00F23C40BB
:106E800002F07AB830B590F80C3385B004460D4660
:106E90008BB1032B18D004F525701AF05FFC28463F
:106EA00001A98DED010ACDED020A8DED031A19F04D
:106EB000F5FF012006E000F23C4001F0A5FB0028B0
:106EC000E9D1002005B030BD90F86032002BF8D039
:106ED0001FF026FADFE700007FB590F80C2332B1EF
:106EE000032A4FF0000309D0039304930CE000F24F
:106EF0003C4007B05DF804EB01F060BC03A90393CC
:106F0000049305931FF0C8F89DED030ADDED040A14
:106F100007B05DF804FB000007B590F80C3333B1FF
:106F200000F57F7003B05DF804EB1AF063B900F26E
:106F30003C4001F043FC68468DED000ACDED010AAE
:106F40001AF058F903B05DF804FB000090F80C0348
:106F5000003818BF0120704708B590F80C23032AA9
:106F600005D0BDE8084000F23C4001F011BC1FF024
:106F700093F8012008BD000010B590F80C230C46D2
:106F80001AB1032A07D0002010BDBDE8104000F25E
:106F90003C4001F0A1BB1FF0A5F8012084ED000AE0
:106FA000F2E7000030B590F80C3385B005460C468A
:106FB00023B1032B09D0002005B030BD00F23C40C6
:106FC00005B0BDE8304002F087BA002302A9029361
:106FD00003931FF049F80028EDD001A928461FF0BF
:106FE0004FF80028E7D0029B2360039B6360019B5E
:106FF000A360E1E790F80C231AB1032A05D0002022
:10700000704700F23C4002F09BBA1FF02DB8000020
:1070100090F80C231AB1032A05D00020704700F223
:107020003C4002F07FBA1FF02BB8000090F93232DA
:107030003BB990F8683213F0010F14BF0320002011
:107040007047032070470000F7B50446FFF7EEFFD6
:107050000546002862D0032839D194F860326BB31A
:1070600094F86832D8072BD501A920461FF0AAFB57
:10707000BDF80430002B18BF002594F8146206F008
:10708000FD06012E4AD10023032D019307D101A94A
:1070900020461FF0A3FB20461FF072F9064604F2BB
:1070A0003C4002F0CBFA08B994F809039DF804308B
:1070B000D90703D55A0701D59F0632D400252DE004
:1070C00020461EF041FF002808BF0025D5E7002517
:1070D000D3E713F0020F2EE094F9443223B99DF860
:1070E0000430DB092FD0E9E7002EF8D010F006F8C5
:1070F000FFF786FB022807D99DF805309806DDD5F5
:107100009DF80430D906D9D5FB6A93F89C30002B42
:10711000E5D118E0DA0601D41B0718D5284603B0DC
:10712000F0BD0028FAD094F80923B4F96436002A97
:10713000CFD013F0010FF1D1154B1F68FB6A93F804
:107140009C30002BC8D19DF804309C07E2D407F096
:1071500015FC07F011FB0028B0D10FF0CFFFFFF7AF
:107160004FFB0228AAD90FF0C9FF90F8C432B02211
:1071700002FB030090ED2F7AF0EE007AB4EEE77A8E
:10718000F1EE10FA9AD59DF80530DB09C6D195E7E6
:10719000582600202DE9F04790F8603292B004465E
:1071A000002B00F0948020461FF05CFC2046FFF787
:1071B0004BFF03287BD104F5487800274146204641
:1071C0000097019702971FF081F8694620461FF04B
:1071D00073F8009BC4F80432019BC4F80832029B88
:1071E000C4F80C32204601F041F9204601F026F99E
:1071F00016F076FE054620461EF028FF0028A8BFA0
:10720000C6B203AA4FF0FF312046BCBF95F8EB94FD
:1072100095F8EC640397A8BFB146049705971EF054
:107220006FFF03A81AF09AFA4FF00C0A0AFB0950F4
:1072300084EDD10AC4EDD20A84EDD31A04F551715C
:1072400000F55C701AF09AFA04F557770AFB0655B8
:1072500084EDC50AC4EDC60A84EDC71A3A464FF05C
:10726000FF31204605F500751EF05EFF95E807002A
:1072700006AE86E80700394630461AF0E5FA04F50E
:107280002B72414609A818F03BFA314609A818F0BC
:10729000B9F909A9204684EDD40AC4EDD50A84EDD4
:1072A000D61A1FF09BFA09A92046FFF727FD94F88C
:1072B0006636002B3AD109A806F0A8FA09A920469B
:1072C0001EF0A8FF90B3012384F866362EE0D0F8B4
:1072D00064321BB96EF03EF9C4F86402154B1B68AA
:1072E000D86A03685B68984788B16EF033F9D4F8C0
:1072F0006432C01AB4F86232984204D920461FF0B2
:107300002FF984F8600294F860327BB14BE76EF09D
:1073100021F9D4F86432C01A41F287339842E4D894
:1073200041F04EFA41F032FA0028DED112B0BDE849
:10733000F08700BF5826002090F80C3323B1032BB0
:107340004FF0000007D0704790F93222032A04D191
:107350000A70012070470870FBE71846704700006C
:1073600073B50D460DF107010446FFF7E5FF06462C
:1073700028B19DF807302BB1032B09D000263046E9
:1073800002B070BD04F5CA630FCB85E80F00F6E7C5
:10739000294620461EF032FF94F86062EFE70000B5
:1073A0007FB50E460DF103010446FFF7C5FF054604
:1073B00018B90025284604B070BD9DF8033083B18C
:1073C000032B16D004F525701AF0C8F901A9304630
:1073D0008DED010ACDED020A8DED031A19F05EFD67
:1073E000E8E7314604F23C4001F00EF90028E9D10B
:1073F000DFE794F86032002BDBD0314620461EF0E8
:107400008FFFDFE737B50D460DF107010446FFF7A3
:1074100093FF28B19DF8073023B1032B0FD0002034
:1074200003B030BD04F5BE631B682B6004F2F45357
:1074300004F5BF641B686B602368AB60F0E720460F
:1074400029461EF039FF94F86002E9E710B50446BA
:10745000FFF7ECFD18B1032807D0002010BD04F29F
:107460003C40BDE8104001F0F9B894F86032002BC0
:10747000F3D020461EF068FD0028EED094F81432B8
:1074800003F0FD03012BE9D194F80C03C31E58420D
:107490005841E3E710B50446FFF7C8FD80B1032863
:1074A00010D194F8600250B16EF054F8D4F8643200
:1074B000C01A44F62063984294BF0020012010BDFA
:1074C0000120FCE70020FAE708B50246FFF7AEFD11
:1074D000032804D110461FF081F9012008BD0020C7
:1074E000FCE7000030B585B004460191FEF722FEAE
:1074F0000199054610B9002005B030BD0191FEF795
:10750000C1FB01990028F6D02846FEF7B7FC0028F9
:10751000F1D0B4F864365907EED494F80933002B4F
:10752000EAD00B4A1268D26A92F89C506DB103A956
:107530002046FFF7C9FF30B19DF80E309A07DBD522
:10754000C3F38000D8E72846D6E71846D4E700BF43
:10755000582600202DE9F04190F80C338CB000271C
:10756000032B06460C46154600970197029719D142
:107570001EF06CFD6A4680464FF0FF3130461EF02B
:10758000D3FDB8F1FF3FA760676027600DD116F00B
:10759000A7FC2B4690F8EC14224615F0B7FB0CB074
:1075A000BDE8F0814FF0FF38EBE716F099FC2B4671
:1075B00022465FFA88F115F0A9FB95ED000A6846AE
:1075C0001AF008F903A920468DED051A8DED030A7E
:1075D000CDED040A1AF038F906F52B7206F548715C
:1075E00003A818F08DF8214603A818F00BF884EDD5
:1075F000021A84ED000AC4ED010A95ED007ADFED70
:10760000037AA7EE271A84ED021AC8E70AE81C419C
:107610001FB5DFED0B7A20EE270A0C461946094B01
:10762000CDE90042BDEEC00A18688DED020A064B96
:107630009DF81820C06A13F063FC04B010BD00BFB1
:10764000E02E654258260020403D0B082DE9F0470A
:107650002DED028B92B0002504460F464FF07E5A66
:1076600000F5487106A89046CDF818A00995089530
:10767000079519F05DF807F081F907F07DF881466C
:107680002046FFF7D3FC032803D094F80C33032BD8
:107690004FD19FED558ADFED558A00262379F2B24E
:1076A000934247D90AAA71B22046CDF828A00D9579
:1076B0000C950B951EF014FE0AA906A819F060FCA3
:1076C000B4EEC80AF1EE10FA0DDD494ACDF800809B
:1076D0003B4648492046FFF79BFF002012B0BDEC17
:1076E000028BBDE8F0870AA906A8039504950595C5
:1076F00019F030FC03A90EA88DED0E0ACDED0F0A8E
:107700008DED101ACDED111A19F098F9B9F1000F9D
:107710000DD09DED050AB0EEC00AB4EEE80AF1EE18
:1077200010FA04DD344ACDF800803B46D1E701363B
:10773000B4E7002394F8686216F0010001D0012B31
:10774000CCD104F2FC510AA8CDF828A00D950C95D7
:107750000B9518F0EDFF0AA906A819F011FCDFED52
:10776000227AB4EEE70AF1EE10FA05DD204ACDF8F0
:1077700000803B462149ADE72046FFF757FC032830
:107780002DD120461EF0F0FD94F86832DB0728D496
:1077900038BB0AA906A803950495059519F0DAFBEC
:1077A00003A90EA88DED0E0ACDED0F0A8DED101A6E
:1077B000CDED111A19F042F9B9F1000F11D09DED7C
:1077C000050ADFED0A7AB0EEC00AB4EEE70AF1EE80
:1077D00010FA06DD084ACDF800803B46CAE70020D3
:1077E000D2E701207AE700BFC2B8323EC2B8B23E4B
:1077F0006C3D0B08773D0B08EE920B087C3D0B08A7
:107800002DE9F7431446054688460193FFF71EFE0F
:10781000019A074638B92448244B00682146C06ABB
:1078200013F06EFB019A019221462846FFF70EFFE6
:10783000064630B32846FFF7F9FB95F80C33019A5A
:1078400083420DD007F09AF806F096FF019A38B1FE
:10785000174B154800682146C06A13F051FB10E031
:107860002846FFF7E3FB18B103280FD0114BF0E7D0
:1078700013464146224605F23C4000F003FF00B1AA
:1078800007B90026304603B0BDE8F08395F8609252
:10789000B9F1000F01D1084BDBE713464146224600
:1078A00028461EF061FBEAE758260020803D0B08C1
:1078B0008C3D0B08BC3D0B08AB3D0B0890F80C331E
:1078C000032B01D11EF0A0BF0020704737B505463D
:1078D00000F5067140F6033201A813F033F928468B
:1078E000FFF7A4FB044640B103280AD0002401A8F6
:1078F00013F04AF9204603B030BD28461EF042FC82
:10790000F5E728461EF03EFC0446F0E708B50246BF
:10791000FFF78CFB10B1032806D008BDBDE8084076
:1079200002F23C4000F064BEBDE8084010461EF084
:1079300061BF00000B4610B411462BB1032B09D0D8
:1079400000205DF8044B70475DF8044B00F23C40AA
:1079500000F064BE5DF8044B1EF05CBC13B5044639
:10796000FFF764FB0A46014620460192FFF7E2FF5B
:1079700070B9084B019A1B68DB6A93F89C0038B118
:1079800094F80C13204602B0BDE81040FFF7D2BFB8
:1079900002B010BD5826002037B504460D4640F20F
:1079A000B25200F5067101A813F0CCF82946204622
:1079B0001EF04EFC94F80C33032B054610D148B151
:1079C00004F583612046FFF7C9FF84F828042046A8
:1079D00000F0A4FD01A813F0D7F8284603B030BD8D
:1079E0000025F7E770B590F87C32DB0786B00446D7
:1079F0000D460CD402F0E0FF437C242202FB03007E
:107A0000D0ED0B7AF1EE677AC5ED007A3BE002A883
:107A100005F0FCFE01A92046FFF7FAFAE8B90FF0DD
:107A20006DFB94F94432022B0646E3D1FEF7E8FEE3
:107A30000228DFD996F8C4029FED147AB02303FB25
:107A40000066D4F87032D6F8B0209B1A07EE903A50
:107A5000F8EEE77A67EE877AD6E702A92046FFF7C5
:107A60007DFF0028DBD0D4F87022039BDFED076A8E
:107A70009DED017A9B1A07EE903AF8EEE77AA7EEB1
:107A8000E67A85ED007A06B070BD00BF0AD7233CC8
:107A9000F0B50C4687B000F50671064640F6863212
:107AA00001A813F04FF8A36853B9E36843B96368BA
:107AB00033B9002701A813F067F8384607B0F0BDC6
:107AC000204605F079FF0028F3D094E80F0002ADBE
:107AD00085E80F000021284605F030FF0746002802
:107AE000E7D096F87C32DB0704D440F069FE192118
:107AF00040F0A2FD95E80F0006F51B7C8CE80F0016
:107B000096F87C3243F0010386F87C32304600F070
:107B100005FD49F02FFC46214AF026F849F02AFCE1
:107B200045214AF021F8054BA2681B68DB6A1A61FF
:107B3000E2685A6162689A61BCE700BF582600207B
:107B400038B5144B1B68DD6A2B6804465B68284611
:107B50009847F0B12B690BB96A69D2B1C4F8743295
:107B60006B69C4F87832A969002204F51B7005F02E
:107B700053FE94F87C3223F0030343F0030384F8AC
:107B80007C3249F0F7FBBDE83840034A062142F059
:107B900019BD38BD58260020D03D0B0810B588B05F
:107BA00004460593FFF742FA0328059B4FF00000B7
:107BB0000AD10690079006A802900B9801900A98A7
:107BC000009020461EF0B6FB08B010BD38B5044644
:107BD000FEF7B0FA0546D0B194F80C33032B03D06E
:107BE00095F84E41204638BD20461EF0FBFAFF288E
:107BF0000446F5D001462846FEF740F90028EFD0AC
:107C000021462846FEF73EF80028E9D0EAE7044678
:107C1000E8E7000008B590F80C33032B05D016F008
:107C20005FF990F9EB04C0B208BD1EF00FFA431CD7
:107C3000F9D1F4E708B590F80C3383B1032B03D1E5
:107C4000BDE808401EF0FAB93FF00CF940F6ED42ED
:107C50004FF480113FF0BEF84FF0FF3008BD1846DA
:107C6000FCE7000090F80C33032B01D11FF046B85D
:107C70007047000090F80C33032B01D11EF0C2B8FE
:107C8000704700001EF048B910B5044621F000F915
:107C90002046FEF7E7FB2046BDE81040FEF7E8BCB3
:107CA00090F80C330BB1032B01D11FF0A3B80020C7
:107CB0007047000030B500F5757304460D460FCBD4
:107CC00085E80F0094F8E40330BD00007FB5054659
:107CD00068460E4605F09AFD95F87C32DB0703D422
:107CE0000024204604B070BD69462846FFF7E2FF35
:107CF00004460028F4D0694605F51B7005F06CFFBA
:107D000086ED000AC6ED010AEBE70000D0F88033EB
:107D10000B6090F87C037047D0F888330B6090F8C4
:107D20008503704730B500F5677304460D460FCBE9
:107D300085E80F0094F8AC0330BD000030B500F5C5
:107D4000836304460D460FCB85E80F0094F82804A2
:107D500030BD000010B500F22C4203460C4607CAA5
:107D600084E8070093F8380410BD00002DE9F043C3
:107D70002DED028B8BB005460E461746FFF726FF0A
:107D8000014680462846FFF7ADFB0446002848D050
:107D9000FEF7D0F94146FEF7B3F886ED000A95F9F3
:107DA0003032002B3ADD0FF0A9F9FEF729FD01284A
:107DB00034D90FF0A3F990F8C432D5EDDE7ADFEDB7
:107DC0005D8A96ED000AB02202FB030095F930327D
:107DD000D0ED2F0A07EE103AF4EEE87AB8EEC77A43
:107DE000F1EE10FAB7EE008AB8BFF0EE487A37EE3F
:107DF000201A20EE270A70EEC70A40F2B63016F0BD
:107E0000BFFDD5EDDE7AF4EEE87AF1EE10FAB8BFF8
:107E1000F0EE487A80EE277A86ED007A01233B70F7
:107E200003E095F8083333B9387020460BB0BDEC49
:107E3000028BBDE8F08395F80C334FF00009CDF8C4
:107E40000490CDF80890CDF80C9043B1032B10D0DE
:107E5000CDF81090CDF81490CDF818907CB902238D
:107E60003B703246414605F23C4001F0ABFB044614
:107E7000DBE701A928461EF0A9F90446E8E795F8D2
:107E80000C33002BEBD004A92846FFF763FF044610
:107E90000028E4D001A904A819F086FC07A8CDEDBC
:107EA000080A8DED091A8DED070A1AF091F804A859
:107EB000B0EE408A1AF08CF895F93032002B30DDA4
:107EC00007EE903AF8EEE77A4FF47F7070EE670AAB
:107ED00037EE801AF5EEC00AF1EE10FA48BFDFED7A
:107EE000160AF4EE410AF1EE10FAB0EE480AC8BFE5
:107EF000B0EE601A16F044FDB0EE408AD5EDDE7AA1
:107F00009FED0C7AF4EEC77AF1EE10FAB7EE007A34
:107F1000B8BFF0EE477A88EE277A032386ED007A21
:107F20007DE7B5EEC08AF1EE10FA48BF9FED028AF8
:107F3000E4E700BF000000340000000010B5044674
:107F4000FFF768FE84F80D032046FFF763FE84F810
:107F50000E032046FFF75EFE84F80F032046FFF76E
:107F600069FE04F55A7184F810032046FEF71AFFE3
:107F700084F8740300F0F2FA04F5617284EDDE0A0D
:107F800004F560712046FFF7F1FE04F5627184F894
:107F90007C032046FEF722FF04F5637184F8850315
:107FA0002046FEF74FFF04F5677184F898032046DA
:107FB000FEF768FF04F56C7184F8AC032046FFF708
:107FC00021FA04F5707184F8BC032046FFF7E8F944
:107FD00004F5757184F8D0032046FEF7BBFE04F566
:107FE0007A7184F8E4032046FFF7BAF984F8F803BD
:107FF0002046FEF771FF04F5806384EDFF0A2046FA
:10800000C3ED000AFEF788FF04F2044383ED000A83
:1080100004F2144204F581612046FFF79BFA04F54F
:1080200083612046FFF79AFC04F22C4184F828046F
:108030002046FEF791FF84F8380410BD37B50D4691
:10804000044600F0FFF81DB915F04AFF14F032FDA8
:108050004FF4BE7204F5067101A812F073FD94F896
:1080600069322BB92046FFF76BFD012384F8693292
:10807000224B1D68A86A03689B6998472046FEF753
:10808000A1FD2046FEF726FE204600F079FA2046A4
:10809000FFF780F8286B30B10368D4EDD20ADB68B3
:1080A00094EDD10A9847D4F8100208B16FF0B4FDEE
:1080B000204600F07DF82046FEF7C6FF94F8903287
:1080C00084F80C0383420ED084F8900298B10C4DD2
:1080D0000C4B032808BF1D4649F04CF90A4A2B46B1
:1080E000062142F06FFA2046FFF728FF01A812F0A0
:1080F0004BFD03B030BD054DEEE700BF5826002014
:10810000ABF50A08773D0B08E83D0B087C3D0B08F2
:10811000D0EDDE7A9FED057AF4EEC77AF1EE10FA33
:10812000B7EE000AA8BFB0EE670A7047000000343F
:10813000014B1868704700BFB08800204FF0FF3037
:108140007047000001207047704700000020704712
:108150000020704770470000704700000020704703
:1081600000207047002070470020704700207047B3
:108170000020704700207047012070470368D3F843
:108180009430184700207047002070470020704747
:108190000020704700207047002070470020704783
:1081A0000020704700207047002070477047000093
:1081B0007047000008B515F093FE90F8EC0408BD78
:1081C00008B515F08DFE90F8EB0408BD30B52DED27
:1081D000028B9FED1A1ADFED1A0A91ED000A87B0A3
:1081E00005462D200C468DED011ACDED000A16F046
:1081F000C7FB9DED011ADDED000AF0EE408A2E204E
:1082000094ED010A16F0BCFB9DED011ADDED000AAC
:10821000B0EE408A2F2094ED020A16F0B1FB03A9BC
:1082200005F52570CDED038A8DED048A8DED050AE7
:1082300037F006FE07B0BDEC028B30BDC2B8323E4F
:10824000C2B832BE10B504466DF084F9D4F8F432E9
:108250001BB1C21AB2F57A7F12D30A4A1268D26AE7
:1082600092F89C2002B15BB9C4F8F40294F8314250
:1082700015F036FE80F8E24406F080FB80F82540D9
:1082800010BD00BF582600202DE9F0432DED028BD4
:1082900091ED007AD1ED037A87B08DED047AB0EEDE
:1082A000C77AB5EEC07AF1EE10FADDE91087DDF895
:1082B0004C90CDED057A0C4615461E4606DCF0EED8
:1082C000E77AF5EEC07AF1EE10FA02DD04A819F0B3
:1082D0000FF86B20B7EE001AFFEE000A9DED050ABD
:1082E00016F04EFB6C2089ED000AB7EE001AFFEE87
:1082F000000A9DED040A16F043FB04A888ED000A6D
:1083000018F052FFB7EE008A002852D00023C9F8B7
:10831000003088ED008AD4ED067A67EEA77AF4EE95
:10832000C87AF1EE10FA4ADB0023336085ED008A4B
:10833000DFED3F0A96ED000A7C20B7EE001A16F03A
:108340001FFB86ED000A95ED000A7D20B7EE001AAE
:10835000FFEE000A16F014FB85ED000AD4ED067A54
:10836000129BDFED346AF1EE677AC3ED007A96ED89
:10837000007AF0EEC77AF4EEE67AF1EE10FA2BD539
:1083800003AB02AA01A9204617F068FB9DED018A04
:10839000B0EE480A8FF01CF885ED000AB0EE480AEE
:1083A0008FF06CF987ED000A07B0BDEC028BBDE8D9
:1083B000F08304A818F0E4FE0028A7D1ABE738EE5C
:1083C000670A16F00DFA86ED000A94ED087AC7EEFA
:1083D000007AC5ED007AABE794ED076AC6EE077A3E
:1083E000C7ED007A96ED007AB0EEC77AB4EEE67A81
:1083F000F1EE10FAC4D495ED007ADFED0F6AB0EE1D
:10840000C76AB4EE666AF1EE10FAB9DCB4EE477AE8
:10841000F1EE10FAB4D6B0EEE77AB4EE667AF1EE89
:1084200010FAADDCF4EE677AF1EE10FABCD7A7E7EC
:108430000000000000000034FFFF7F7F1FB500F543
:108440001773039300F51673029300F515730193E8
:1084500000F51473009300F5127200F5137300F524
:108460004871FFF711FF05B05DF804FB9FED156A39
:1084700090ED817ADFED146AD0ED837A27EE067AEB
:1084800067EE867A27EE267A67EEA67ABDEEC77A81
:10849000FDEEE77A80ED7E7A90ED827A27EE067A1D
:1084A00017EE903A27EE267A002BB8BF03F50C435F
:1084B000BDEEC77AB8BFA03380ED7F7AC0F8003236
:1084C000704700BFE02E65420000C842D0ED946ABC
:1084D000D1ED010AD0ED977A91ED007A20EEA70A4E
:1084E00066EEA00AA7EE260A84B0E7EE670A04B09B
:1084F00070470000D0ED946AD1ED010AD0ED977A73
:1085000091ED007A27EEE00A66EEA00AA7EE260AB1
:1085100084B0E7EE270A04B0704700001FB50E4B89
:108520001B680446B3B1684605F070F969462046F9
:10853000FFF704FC20B16A4600212046FEF770F8E0
:1085400094F87C32DB0705D504F51B720121204627
:10855000FEF766F804B010BD6C8B002008B502F081
:108560002BFABDE8084001F0B9BD000010B580F855
:10857000F81204466CF0EEFFC4F8FC0210BD0000D7
:1085800010B590F8F832044653B16CF0E3FFD4F81C
:10859000FC32C01AB0F57A7F84BF002384F8F83229
:1085A00094F8003353B16CF0D5FFD4F80433C01AFB
:1085B000B0F57A7F84BF002384F8003310BD00003B
:1085C00000F5B6700B4607C883E807000120704726
:1085D0000023C0F89C30C0F89830C0F89430C0F840
:1085E000A830C0F8A430C0F8A030C0F8AC30704754
:1085F00070470000024B0B604FF07C5313607047D4
:10860000000048427047000008B50B4600F1280101
:10861000184618F08DF8012008BD000010B500F5CF
:10862000C0700C460FC884E80F00204605F0DEF845
:1086300030B1FFF77DFD00F51B700FC884E80F0017
:10864000204605F0D3F880F00100C0B210BD000054
:1086500010B5044605F012FC204610BD10B5D0F848
:10866000783104465BB16CF075FFD4F87831C01AEC
:1086700041F28833984294BF0020012010BD0120B0
:10868000FCE7000013B5009303680192D3F8903023
:108690009847DDE90021044628B90448044B0068E6
:1086A000C06A12F02DFC204602B010BD58260020F2
:1086B000803D0B0813B504460191FDF73BFD23688F
:1086C000019A1B6D014608B190F84E11204602B088
:1086D000BDE810401847000030B585B00023019375
:1086E0000293039303680D46DB6D01A99847044686
:1086F00020B1039B2B60204605B030BD02F05CF931
:10870000417C01F027FE04460028F4D002F054F921
:1087100001F086FDB1EE400A85ED000AEBE70000AE
:1087200090ED007ADFED0F7AB0EEC77AB4EEE77A1B
:10873000F1EE10FA14D590ED017AB0EEC77AB4EEEE
:10874000E77AF1EE10FA0BD590ED027AB0EEC77A27
:10875000B4EEE77AF1EE10FA4CBF0120002070472A
:10876000002070470000003410B5FDF7E3FC04461C
:1087700058B190F84E11FDF785FA30B194F84E11CA
:108780002046BDE81040FDF779BB002010BD000079
:1087900038B50D460EF0B2FC0446FEF731F802285B
:1087A00081BF94F8C402B02303FB0040D43089BFDA
:1087B00007C8002085E80700012038BD2DE9F043F7
:1087C0002DED028B8FB003680025DB6C03950495BB
:1087D00005950695029502A904469847064638B1C4
:1087E000FFF7BCFEDDED027A27EE800A8DED020A6E
:1087F0000EF084FCFEF704F80746002E50D0DDEDA5
:10880000027AD4ED6A6A94ED6B7A23680B9527EEB1
:10881000877A67EEA67A8DED097ACDED0A7A0C9506
:108820000D959B6C0BA9204609AD98470BA92846CE
:1088300018F014FC012F8DED030ACDED040A40F26F
:10884000B3800EF05BFC90F8C432DFED5B7AB025AC
:1088500005FB030090ED308A28EE278AB0EE480A27
:108860008EF0B6FDF0EE408AB0EE480A8EF006FFBC
:10887000CDED0B8A8DED0C0A0EF040FC90F8C43261
:1088800005FB030090ED2F0A0BA818F007FC09ADBB
:108890008DED050ACDED060A05A896BB03C885E057
:1088A0000128CED89DED020AB5EEC00AF1EE10FA0D
:1088B0007FDD07AED4F8AC21D4F8A831079230465A
:1088C000089318F015FC23680B950C950D959B6C7F
:1088D0000BA920469847DDED077A9DED0B7A77EEE0
:1088E000877A9DED0C7ACDED077ADDED087A77EE8B
:1088F000877A09ABCDED087A96E8030083E8030098
:1089000049E0236993ED000AB7EE008A38EE408A09
:1089100018F0C4FB04F5C8798DED090A4846B0EE9D
:10892000480ACDED0A0A18F0B9FB0BA92846CDED8F
:108930000C0A8DED0B0A18F091FB04F5D07603AF0D
:10894000C4ED650A314684ED640A384618F096FB9A
:1089500004F5CC788DED090A4046B0EE480ACDED1D
:108960000A0A18F09BFB0BA928468DED0B0ACDEDEA
:108970000C0A18F073FB97E8030084ED660AC4ED57
:10898000670A86E803004946404618F067FB8DED0C
:10899000090ACDED0A0A9DED090ADDED0A0A0FB0BC
:1089A000BDEC028BBDE8F083DDE9030185E803003F
:1089B000F1E709950A95EEE735FA8E3C10B590F887
:1089C0004213044605F0F4FB7C23C0B203FB0044D1
:1089D000D4F8A00010BD0000044B026F1B68DB6AD6
:1089E0005A60426F9A60826FDA60704758260020A2
:1089F000F0B58FB0044615F073FA00230293039389
:108A0000049390F8EB1401AB02AA054614F020F988
:108A100004F19407D8B39DED010AB5EEC00AF1EE5A
:108A200010FA34DD02A818F0E5FE04F1B00684ED7A
:108A30002C0AC4ED2D0A84ED2E1A3946304618F062
:108A4000E9FE04F17C01304618F098FE04F188013B
:108A500005A88DED050ACDED060A8DED071A18F073
:108A60008DFE08A88DED080A9DED010ACDED090ADD
:108A70008DED0A1A18F0AEFE0BA904F128008DED59
:108A80000B0ACDED0C0A8DED0D1A17F093F895F841
:108A9000EB040C2303FB0050394600F55C7018F022
:108AA0006DFE84ED2C0AC4ED2D0A84ED2E1A0FB054
:108AB000F0BD00002DE9F047824B00251F682DED29
:108AC000028BC0F89C50C0F89850C0F89450C0F881
:108AD0008450C0F88050C567C0F89050C0F88C50E2
:108AE000C0F88850C0F8B850C0F8B450C0F8B050C2
:108AF0000446F86A03688AB05B680E46984704F13A
:108B00002809002854D06CF025FD42F20F739842DA
:108B10004ED8FB6A9FED6C8A93ED010A84ED1C0A26
:108B2000D3ED020AC4ED1D0A93ED031A484684ED05
:108B30001E1A16F033FF48F01DFCD4ED1E7A67EEC6
:108B4000887A054617EE900AF3F7D6FCD4ED1D7A25
:108B500067EE887ACDE9040117EE900AF3F7CCFCB2
:108B6000D4ED1C7A67EE887ACDE9020117EE900AFF
:108B7000F3F7C2FC554ACDE900010621284641F031
:108B800021FD94ED1E8AB0EE480A8EF021FC84EDA2
:108B90006B0AB0EE480A8EF071FD84ED6A0A6CF043
:108BA000D9FCC4F87C010AB0BDEC028BBDE8F087AB
:108BB000A6B194ED1C0AB4EE400AF1EE10FA0DD6FF
:108BC000D4ED1D0AF4EE600AF1EE10FA06D694ED2B
:108BD0001E1AB4EE411AF1EE10FA52D715F080F9D0
:108BE00090F8EC344FF00C0A0AFB030303F5007312
:108BF000074693E8070007AE86E807004FF0150820
:108C0000B2EE028AF2EE068A304619F0E1F9B4EECD
:108C1000C80AF1EE10FA38D508F1FF3818F0FF084D
:108C20003CD1304619F0D4F9F1EE047AB4EEE70AFB
:108C3000F1EE10FA43DD9DED090ADDED087A9DEDB8
:108C4000078A20EE000AA7EEA70A8EF02DFFF0EEAD
:108C5000400AB0EE480A8EF0DDFDDDED090A84ED34
:108C60001D0A9DED080AF1EE600AB1EE400A8EF091
:108C7000D1FD84ED1C0A9FED161AD4ED1D0A94ED6A
:108C80001C0A484616F08AFE7BE7304619F0A0F928
:108C9000B4EEE80AF1EE10FABEDCC2E7384613F093
:108CA00027FE384613F006FF97F8EC340AFB0373EF
:108CB00003F5007393E8070086E80700A4E725673B
:108CC0006567D8E758260020E02E6542003F0B0874
:108CD000000000000021FFF7EDBE000037B504469C
:108CE00008461546019119F073F9B7EE007AC7EE00
:108CF000007AB4F8DC3001980133A4F8DC3094ED4C
:108D0000367A37EE277A84ED367AB0EE007AF4EED2
:108D1000C77AF1EE10FA06D5B6EE007AF4EEC77A0D
:108D2000F1EE10FA0DDC9FED0E7AF4EEC77AF1EE5B
:108D300010FA13D59FED0B7AF4EEC77AF1EE10FA24
:108D40000CDDB0EE670A18F045FD012085ED000A44
:108D5000C5ED010A85ED021A03B030BD0020FBE726
:108D600000247449BD37863570B52DED028B00F1B6
:108D7000280600F134058AB029460446304618F02A
:108D8000A5FDB6EE008A20EE088A2846B0EE480A15
:108D900018F020FD07A93046CDED080A8DED091A1F
:108DA0008DED070A18F000FD30468DED010AB0EE9A
:108DB000480ACDED020A8DED031A18F00BFD07A944
:108DC00028468DED070ACDED080A8DED091A18F039
:108DD000EBFC04A901A88DED040ACDED050A8DED8B
:108DE000061A18F087FD324601A920468DED070AC4
:108DF000CDED080A8DED091AFFF770FF58B96CF038
:108E0000A9FB0121C4F878012046FFF753FE0AB000
:108E1000BDEC028B70BD2A4604A92046FFF75EFF19
:108E20000028ECD004F1400207A92046FFF756FFC6
:108E30000028E4D0EBE7000030B52DED028B0D46A5
:108E400083B091F842130446284605F0B1F9C1B247
:108E50007C2000FB0151903104F1280016F02EFC1B
:108E600068468DED000ACDED010A18F0C3F9DFED7B
:108E70001C7AB4EEE70AF1EE10FA05D59FED190A57
:108E800003B0BDEC028B30BD684618F031FA68467D
:108E900018F08AF90028F1D1284694ED488A05F0A7
:108EA000FBFAF0EE400AB0EE480A15F065FC80B916
:108EB000284605F0F1FA84ED480AB0EE408A8EF0BB
:108EC00087FA84ED490AB0EE480A8EF0D7FB84EDAC
:108ED0004A0A04F59271684618F034F9D0E700BFE9
:108EE00000000034000000009FED0C7AB4EEC70AC9
:108EF000F1EE10FA0BD4DFED0A7AB4EEE70AF1EEE8
:108F000010FA07DCC0EE077AB0EE670A7047F7EE9A
:108F1000007AF9E7F2EE047AF6E700BFF3665F3F06
:108F200058A00B4108B51C3018F064F9F1EE007A36
:108F3000B4EEE70AF1EE10FA9DBFF1EE027A37EED9
:108F4000C00ADFED047A9FED040A98BF20EE270ADD
:108F500008BD00BFCDCC4C3ECDCCCC3D08B583691F
:108F600093F9000038B10EF0C9F8FDF749FC01286B
:108F700094BF0020012008BDF8B52DED028B0546F9
:108F800005F0FCFC05F0F8FB0446B8B3FFF7D0F899
:108F900090F8093393B32846FFF7E0FF064668B31D
:108FA0000EF0ACF890F8C432B02707FB030090ED48
:108FB0002F7AF0EE087AB4EEE77AF1EE10FA1DD4CB
:108FC00095ED1E8A0EF09AF890F8C432DFED1E7A05
:108FD00007FB030090ED300A98EE270A15F050FCCD
:108FE000DFED1A7AB0EEC00AB4EEE70AF1EE10FA3D
:108FF00008DC6CF0AFFA3446C5F86801BDEC028BB2
:109000002046F8BD05F5B67018F0E2FFB0EE408AD4
:109010000EF074F890F8C4329FED0D7A07FB03034D
:10902000D3ED2F7A67EE877AB4EEE78AF1EE10FA85
:10903000DFD56CF08FFAD5F86841001BB0F5FA6FF8
:109040008CBF00240124D9E7E02E654200003442A1
:10905000CDCC4C3F10B50A4B1B68DB6A93F89C30B3
:1090600004465BB96CF076FAD4F87C31C01A44F649
:109070001F6398428CBF0020012010BD0020FCE738
:1090800058260020F8B52DED068B04460EF036F874
:10909000054605F073FC064608F05CF9002840F030
:1090A000AA802046FFF768FF002800F0A78030461E
:1090B000FFF784FCD4F8E830984200F0188130467D
:1090C000FFF77CFCD4F8E830DFED8E7AC31A08EEA7
:1090D000903AF8EE688A304668EEA78AFFF76EFC91
:1090E00094F8BC30C4F8E800F3B9304605F056FBFC
:1090F000D0B104F1280796F842233946304605F0EE
:10910000CFF9D4ED1D0AB0EE401A384694ED1C0A92
:1091100016F044FC0023C4F89030C4F88C30C4F836
:109120008830012384F8BC3020463146FFF784FEA6
:1091300095F8C40205EB0015B0EE408A2B6FC4F819
:10914000EC3004F1B000D4ED129A18F041FF6368DE
:10915000DFED6D7A93ED007AB4EEE77AF1EE10FA76
:1091600068EE299AB0EE40AA01D5C3ED007A2046F8
:10917000B0EE4A0AFFF7B8FE636820EE299A93ED35
:10918000000A29EE009AFFF7CDFE29EE009A20464C
:1091900084ED249AFFF75EFF38B1D4ED247AB2EE65
:1091A000007A67EE877AC4ED247AF0EE007AF4EE66
:1091B000E78AF1EE10FA10D5DFED547AB4EEE7AAA3
:1091C000F1EE10FA09D5DFED527A69EEA79AD4EDE7
:1091D0002A7AE9EEA87AC4ED2A7A9FED4E0A94ED38
:1091E000397ADFED4D7AB0EEC88A28EE008AA7EE14
:1091F000278A84ED398ABDEC068BF8BDFEF798FF0F
:1092000090F80933002B72D02046FFF7A7FE002804
:109210006DD095F8C42205EB0213196FD4F8EC3029
:109220008B4264D0B02606FB025292ED2F7AF0EE0C
:10923000087AB4EEE77AF1EE10FA58DBCB1AC4F8EC
:10924000EC1008EE903A95F8C4329FED341A94ED84
:109250001E0ADFED337A06FB0353D3ED309A69EE35
:10926000819AF8EE688A39EEC00A68EEA78A15F08E
:1092700073FBB0EE409A8EF001FA94F8BC30B0EE79
:10928000408AF3B1F3EE047AF4EEE78AF1EE10FAD5
:1092900017DC95F8C40206FB005595ED2F7AF2EE27
:1092A000027AB4EEE77AF1EE10FAFFF64AAFDFED9C
:1092B0001D7AB0EEC99AB4EEE79AF1EE10FAFFF615
:1092C00040AF9FED198AD4ED1D0A94ED1C0AB0EE53
:1092D000691A04F1280016F061FB012384ED248A49
:1092E00084ED238A84ED228A84F8BC3029E7BDEC22
:1092F000068B04F188009FED0D0ABDE8F84018F0D8
:10930000BDBA00BFBD378635CDCC4C3DC2B8B23EEC
:109310000AD7233CCDCC4C3ECDCC4C3F35FA8E3CCD
:109320006F12833A1904863F00000000EC51783F29
:1093300030B50C2303FB010101F1C003144693E88F
:1093400007008BB004AD85E8070094E8070083E8C8
:1093500007002846FFF7E4F907AB58B194E8070087
:1093600083E807009DED070ADDED080A9DED091A67
:109370000BB030BD95E80700F2E70000F0B52DED29
:10938000028BD0F830318B60D0F83431CB6085B0AF
:1093900004460D4601F010FB06460DF0AFFEA36932
:1093A00093F90030022B07464BD1FDF729FA02282A
:1093B00047D997F8C432B02202FB0373D3F8B01038
:1093C0000022284604F028FAD4ED500A94ED4F0A02
:1093D000284604F01BFD94F8443163B36CF0BAF8EE
:1093E0009FED228A97F8C4128DED018A01AA0646E4
:1093F00038460CF007FFD4F838019FED1D0A361AE5
:1094000007EE906AF8EE677A4FF4876027EE800ADD
:10941000B6EE001AF0EE480A15F0B2FADDED017A68
:1094200030EE270A04F584708DED010A17F036FE40
:10943000284604F0EBFC94F8440105B0BDEC028B27
:10944000F0BD707C242303FB006696ED0B8AFEF7CB
:109450006FFED0ED9C7A9FED077AF8EEE77AE8EEA2
:10946000077AFDEEE77A17EE901AA9E700000000F0
:109470006F12833A0000C842F8B5036F0B60436F68
:109480004B60836F8B6000F14C050E46074601F17F
:109490000C040FCD0FC40FCD0FC42B68236007F150
:1094A000B00207CA06F1300383E8070007F194020F
:1094B00007CA06F13C0383E8070007F11C0207CA4C
:1094C00006F1480383E8070006F160013846FFF71C
:1094D00055FF86F87000F8BD30B589B0044668467F
:1094E0000D4604F093F969462046FFF797F818B93E
:1094F0000024204609B030BD04A804F087F92046B6
:1095000004A9FFF73BFF04460028F1D004A96846F0
:1095100004F0D4FB85ED000AC5ED010A85ED021AC1
:10952000E7E700001FB500230C4601A90193029351
:109530000393FFF7D1FF08B1039B236004B010BD74
:1095400030B585B001AD00230C4629460193029346
:109550000393FFF7C1FF034618B195E8030084E8C1
:109560000300184605B030BDF8B506460F4615464F
:10957000FCF7E0FD044690B13946FCF783FB70B17F
:1095800020463946FCF77AFC044640B1FCF7D2FD90
:109590003946FCF7B5FC85ED000A2046F8BDFEF71C
:1095A000C7FD90F8083343B13046FFF7D7FC0446B7
:1095B00018B1D6F864312B60EFE7D6F864312B6030
:1095C0000024EAE770B52DED048B1646FFF7CCFFBB
:1095D000054670B3FEF7ACFD90F930424CB30DF088
:1095E0008DFDFDF70DF9012823D9E4B207EE904A6D
:1095F000B8EE678A0DF082FD90F8C43296ED009ABD
:10960000B02202FB0300D0ED2F8AFEF7A7FF38EE51
:10961000281A78EEC80A40F2614029EE000A15F0D7
:10962000AFF9B0EE408AFEF799FFC8EE007AC6EDBA
:10963000007ABDEC048B284670BD000008B505F02B
:109640009DF9BDE8084005F097B8000010B5044644
:1096500018F06CF950B904F10C0018F067F928B94A
:1096600004F11800BDE8104018F060B9012010BDE9
:1096700038B500F1280504462846FFF7E7FF28B172
:1096800020460121BDE83840FFF714BAD4ED107A26
:10969000B7EE007AF4EEC77AF1EE10FA06D5BFEE17
:1096A000007AF4EEC77AF1EE10FA12DC2046FFF7EA
:1096B0005BFB2846FFF7CAFF0028E1D1D4ED107A02
:1096C000B2EE047AF0EEE77AF4EEC77AF1EE10FA31
:1096D000D6DC38BD10B5044618F07AFC2046BDE84B
:1096E000104018F0DFB800002DE9F04F2DED028B8F
:1096F000A3B000270446B0EE408A0A970B970C9758
:10970000FFF7C0FC14F0ECFB04F1F00B05465E46DD
:109710004FF0000804F1280A95F8F131022B5FFAA6
:1097200088F1A8BF02238B423AD92846019112F052
:10973000FDFF019980B310AB13AA28461397149725
:10974000159713F0E3FA9DED100AB5EEC00AF1EE9D
:1097500010FA21DD13A818F04DF81CA950468DED24
:109760001C0ACDED1D0A8DED1E1A15F04BFF16A833
:109770008DED160AB0EE480ACDED170A8DED181AD8
:1097800018F028F81CA930468DED1C0ACDED1D0AF5
:109790008DED1E1A18F03EF808F101080C36BBE7F3
:1097A00095F8EC140C2303FB015101F500715046B0
:1097B00015F028FF84ED070A94ED450AC4ED080A68
:1097C00030EE088A84ED091A84ED458A0DF096FC86
:1097D0000646FEF7ADFC90F8093302932046FFF7EA
:1097E000BDFB80B13046FDF70BF802280BD996F887
:1097F000C4226169B02303FB026391F9001093F85E
:10980000D200884261DA94ED457ADFEDCB7AB4EE8E
:10981000E77AF1EE10FA61D494ED598AFEF7A4FFCD
:1098200038B1FCF787FC90F84E11FCF769FBB0EEFD
:10983000408A236C626BA16A1E93B0EE480A1CA892
:109840001D921C9117F0C6FF04F5B6710AA88DEDA4
:109850000A0ACDED0B0A8DED0C1A17F0DBFF6BF049
:1098600079FE0023019084F82C312046FFF776FB27
:10987000002869D096F8C422B02302FB0332324498
:109880005268C4F8302196F8C42202FB03333344F3
:109890009B68C4F834316BF05DFE0123C4F83801D5
:1098A000C4F83C71C4F8407184F84431D4F81831DC
:1098B000002B5CD1019BC4F818310AAB93E8070078
:1098C00004F5847484E8070008E006EB0212126FC6
:1098D00001920199D4F818218A4204D123B0BDEC39
:1098E000028BBDE8F08FD43393E8070094F82C3155
:1098F0000DF1280C8CE807001BB904F5847383E88C
:1099000007000123604684F82C3104F5B67117F086
:109910004BFF1CA904F14C008DED1C0ACDED1D0A76
:109920008DED1E1A15F09CFEB5EEC00AF1EE10FA90
:109930008DED1C0AD8BF9FED810ACDED1D0A8DED7E
:109940001E1A84ED590A90E794ED457AD4ED4F7ACA
:10995000DDED0A6AE6EE877ADDED0B6AC4ED4F7A3B
:10996000D4ED507AE7EE267AC4ED507A9EE7D4ED36
:10997000457A734B0D97F5EEC07AF1EE10FA0E971B
:109980000F93ABD99FED6F7A94F82C3167EE877AFD
:10999000B7EE007AC7EE278A1BB9029B002B00F0B6
:1099A000C380E36804F584710AA893ED008A17F078
:1099B000FBFE28EE888A8DED1C0A1CA8B0EE480A32
:1099C000CDED1D0A8DED1E1A17F004FF16A90DA886
:1099D0008DED160ACDED170A8DED181A17F01AFF46
:1099E0000DA8FFF777FE0DA817F0BAFF20B16BF0B6
:1099F000B1FDC4F8780171E701231822002116A8EF
:109A0000039390F001F9182200211CA890F0FCF8B3
:109A10009FED4A8A05F20E530DF170084FF00009D0
:109A20004FF0FF37059395F8F131022B1A465FFA94
:109A300089F1A8BF02228A4240F296808B420491AB
:109A40006BD9059B13F80930002B66D0B0EE680A7D
:109A5000584617F013FFDDE90331002B66D00C22C6
:109A600022AB02FB0933A3F11802049220465A46A6
:109A70000693FFF75DFC069B03ED060A049BC3ED0E
:109A8000010A83ED021A4046FEF74AFE002844D13F
:109A90004046FFF71FFE404617F062FF00283CD10A
:109AA0000C2303FB09F222AB134407920DA9A3F187
:109AB000300240460492069317F01CFF069B03ED0C
:109AC0000C0A049B0DA9C3ED010A83ED021A40465E
:109AD00017F0FCFE22AB079A03EB890303ED1A0A89
:109AE00016AB981818F074FA7A1C04D0B4EEC08A39
:109AF000F1EE10FA03DD4FFA89F7B0EE408A22AB9F
:109B000003EB870353ED1A7AF5EE407AF1EE10FA83
:109B1000F7EE007A48BFB0EE678A09F1010908F153
:109B20000C080BF10C0B7EE7029B66E79BE8070035
:109B300088E80700A7E700BFCDCC4C3E000000003E
:109B4000000080BF0AE81C41CDCC4C3ECDCC4C3F40
:109B5000CDCC4C3D920A06BF920A063FC2B8B23E37
:109B6000728A0E3C5B8218397B1C3FF440AF84F84C
:109B70001C712046FFF700FA60B12046FFF7EEF9AE
:109B8000002840F0348122AA0C2303FB0723002283
:109B900043F8282C16AA07EB470895F8EB3402EB9C
:109BA000880895F8F0219A4240F23C812B4493F8C2
:109BB0000C35002B00F0368195F8EC3495F8F12146
:109BC0009A4240F22F812B4493F80E35002B00F07F
:109BD00029810C2322AA4146504603FB072715F092
:109BE0003FFD07ED0C0A47ED0B0A07ED0A1A404648
:109BF00017F09CFE002840F02181404617F0B0FE8F
:109C0000002840F01B815FED307A94ED387A28EE21
:109C1000278A5FED327AA7EE278A04F1B00084ED3F
:109C2000388A18F0D5F9A3685FED377A93ED007A9A
:109C3000B4EEE77AF1EE10FAB0EE408A00F102815C
:109C40002046B0EE480AFFF74FF9404617F0C2FD34
:109C5000A3688DED130ACDED140A8DED151A93ED61
:109C6000000A13A817F0B6FD204684ED1F0AC4EDC4
:109C7000200A84ED211AFFF7EDF928B1B2EE000AAF
:109C800004F17C0017F0FAFD029BB3B33046FCF7F9
:109C9000B7FD012831D996F8C402B02303FB006652
:109CA00096ED2F7AF0EE087AB4EEE77AF1EE10FA3C
:109CB00023D595F8EC040C2303FB005595ED807A31
:109CC000F1EE0C7AB4EEE77AF1EE10FA15DBD4ED92
:109CD0001D7A1FED607AF4EEC77AF1EE10FA0CDD12
:109CE0001FED637AF4EEC77AF1EE10FA05D5B6EE01
:109CF000000A04F17C0017F0C1FD5FED687AB4EE54
:109D0000E78AF1EE10FA22D51FED6B0A404617F0F4
:109D100061FD10A88DED100A94ED450ACDED110AF4
:109D20008DED121A17F056FD13A904F1A0008DED68
:109D3000130ACDED140A8DED151A17F06BFDD4ED55
:109D40002B7A94ED457A77EE877AC4ED2B7A94EDF1
:109D50002B7AF1EE047AB4EEE77AF1EE10FA4FF0D6
:109D600000053BDB14F0BCF85FED827A94ED2B1A12
:109D700094ED280A21EE271A40F2C530F1EE410A8F
:109D80008DED031ACDED020A14F0FAFD9DED031AD4
:109D9000DDED020A84ED280A40F2C63094ED290A6E
:109DA00014F0EEFD9DED031ADDED020A84ED290AA3
:109DB00040F2C73094ED2A0A14F0E2FD04F1A0014C
:109DC00084ED2A0A04F1940017F024FDC4F8A85089
:109DD000C4F8A450C4F8A050C4F8AC501822002114
:109DE00004F1F0008FF010FFC4F8145162E5E3684D
:109DF000F7EE000A93ED000A14F0BEFC00283FF4D1
:109E0000C2AE94ED1C0AB0EEC00A8DF037FC0C23F4
:109E100022AA03FB072353ED0A7A27EE800A03EDFB
:109E20000A0AB7E60C2322AA03FB0727002347F8F8
:109E3000283C47F82C3C47F8303CD8E62046FFF752
:109E400017FCD4E5C3ED007AFAE600BF2DE9F04D2A
:109E50002DED048B9EB0044614F042F800F59F638C
:109E6000D3ED007A90ED7F8AF4EE487AF1EE10FAA5
:109E700048BFB0EE678ADFED5C7AB4EEE78AF1EEB8
:109E800010FA0DDD1822002104F1F0008FF0BCFE65
:109E90000023C4F814311EB0BDEC048BBDE8F08D76
:109EA0002046FEF7A5FD2046FEF75EFFB0EE480A0D
:109EB0002046FFF719FC2046FFF7DAFBFEF738F9DA
:109EC00014AD00F5347204F1280114A815F018FC43
:109ED0000FCD04F14C060FC60FCD0FC62B683360B3
:109EE00004F1740204F1780304F1700104F14C00F0
:109EF00015F0B4FD94ED1E8AB0EE480A8DF068FAB4
:109F000084ED6B0AB0EE480A8DF0B8FB204684ED74
:109F10006A0AFEF761FDFEF70BF904F5C071FDF763
:109F20000DFF6BF017FBD4F8B031C31A632BB2D915
:109F3000C4F8B0013EF044FC9FED2C9A05466BF04E
:109F400011FBD4ED1C7A67EE897A074617EE900A6A
:109F50000E46F2F7D1FAD4ED1D7A67EE897A824681
:109F600017EE900A8B46F2F7C7FA94ED1E0A20EE20
:109F7000090A41EC180B14F06DFCD4F8740110EED2
:109F8000108AF2F7B9FACDE91201D4F87001F2F7AC
:109F9000B3FACDE91001D4F86C01F2F7ADFACDE9CE
:109FA0000E01D4F8E400F2F7A7FACDE90C01D4F8D9
:109FB000E000F2F7A1FACDE90A014046F2F79CFA77
:109FC0000B4B01930B4B0093CDE908018DED068BF4
:109FD000CDE904ABCDE90276074B084A084928468B
:109FE0003EF090F957E700BFCDCC4C3EE02E6542E5
:109FF000653F0B086F3F0B082C3F0B08363F0B08E3
:10A000007C3D0B0808B52DED048BB0EE609AF0EEA8
:10A01000408A00F011F9B0EE408A89EE280A8DF0EE
:10A0200063FCDFED0B7A20EE270A8DF0F5FBDFED08
:10A03000097A38EE278ADFED087A28EE278AF7EECC
:10A04000007A37EEC00A28EE000ABDEC048B08BD8A
:10A0500041D3423E33938843A1D81943FFF7D2BF7F
:10A0600008B52DED048B9FED189AF0EEE07AF4EE32
:10A07000C97AF1EE10FAF0EE408AB0EE608A1ED492
:10A0800000F0DAF8DFED117A9FED117A70EE277AA1
:10A090009FED100AE8EEC77A9FED0F7A27EE800A4F
:10A0A000C8EE007A87EE270AB4EEC90AF1EE10FA7C
:10A0B00005DBBDEC048BBDE808408DF0F5BCBDECC4
:10A0C000048BB7EE000A08BD0000003433938843C8
:10A0D000F4FDD43B48A18F43CDCC9C3F427CD0EDD6
:10A0E000257A242101FB020292ED0B0AD2ED090A26
:10A0F00030EE270AFFF7B4BF38B52DED088BDFED42
:10A1000021AA9FED21AA9FED21BA0546B0EE409A03
:10A11000F0EE609AB0EE408A1524013CA4B25CB324
:10A12000F0EE490A2846B0EE480AFFF76BFFF0EE62
:10A13000490A70EE698A284638EE2A0AFFF762FF5C
:10A14000B0EEE87A70EE697AB4EECA7AF1EE10FAFF
:10A1500077EEE87A10D468EEAA8A40F2631088EEAF
:10A16000A70AB0EE4B1A38EE400AF0EE4A0A14F095
:10A1700007FCB0EE408AD0E7B0EE480ABDEC088B91
:10A1800038BD00BFCDCCCC3D0AD7233C0024744958
:10A19000002343608360C360036143618361C361E3
:10A1A000002380F82030704790F82020531CDBB249
:10A1B000062B80F8203000EB820288BF002382ED5E
:10A1C000010A88BF80F82030704700004FF0FF334D
:10A1D00010B543610E4BC0F8A8300023044680F848
:10A1E000C830A830FFF7D4FF0A4BC4F8A83004F5F4
:10A1F00086706AF079FB084B08491C60204634F0F1
:10A20000EFFED4F89030C4F89430204610BD00BF63
:10A210008C410B089C410B08B48800202C420B0891
:10A2200008B5A8303FF0F2FADFED027A20EE270AF7
:10A2300008BD00BF00007A4490ED3C0ADFED057ACE
:10A24000B0EEC07AB4EEE77AF1EE10FA48BF90EDC6
:10A250003D0A70470000003473B5D0F8A4300446BE
:10A260000E4663B16BF076F9D4F8A430C01A42F20E
:10A270000F73984203D894ED280A02B070BD114BB9
:10A280001D687DB195F84E112846FBF7F7FD48B1E2
:10A2900095F84E1101AA2846FBF7A8FB10B19DEDD9
:10A2A000010AEAE7242101FB064494ED0A0ADFEDE6
:10A2B000067AB4EEE70AF1EE10FA58BFB0EE670A7C
:10A2C000DBE700BFAC88002000000C4208B561B19C
:10A2D0000378022B02D906486BF00AF95A1C027067
:10A2E00000EB83004160012008BD0846FCE700BF89
:10A2F00054400B082DE9F84305460E4691460024CC
:10A3000000F13C082B78A34211DD00234A46314678
:10A31000012010F071FA242363430746002158F806
:10A32000030010F079FA874204D00134EAE70020F4
:10A33000BDE8F8830120FBE7054B1B682BB14169A1
:10A340004A1C02D018463EF005BA0020704700BFF4
:10A350006C8B002002290BD8242303FB010191F808
:10A36000390030B191F83A0018B191F83B007047CC
:10A37000002070472DE9F04704466BF0EBF8D4F865
:10A38000F86042F21073861B9E4288BFC4F8F80042
:10A3900000274FF0240942F2107A237CFDB2AB4231
:10A3A0001CD929462046FFF7D5FF70B109FB0548A7
:10A3B00098ED0D0AD8ED097AD4ED250A30EE270A7A
:10A3C0002046FFF799FE88ED0C0A564504D909FB93
:10A3D0000540303034F0DCFF0137DEE7617C204699
:10A3E000FFF73AFF84ED3D0ABDE8F08770B50446FB
:10A3F00086B06BF0AFF8D4F89830C31AB3F57A7F13
:10A4000005464FD3344B94ED257A1B68DFED336A54
